 SwiGobi

 Timestamp is 5400392c (Fri Aug 29 16:26:20 2014)

 Preferred load address is 10000000

 Start         Length     Name                   Class
 0001:00000000 00015b04H .text                   CODE
 0001:00015b04 0000004cH .text$yc                CODE
 0001:00015b50 00000010H .text$yd                CODE
 0002:00000000 0000ceddH .rdata                  DATA
 0002:0000cee0 00000072H .rdata$debug            DATA
 0002:0000cf54 000000ccH .xdata                  DATA
 0002:0000d020 0000003cH .idata$2                DATA
 0002:0000d05c 00000014H .idata$3                DATA
 0002:0000d070 0000020cH .idata$4                DATA
 0002:0000d27c 000002c4H .idata$6                DATA
 0002:0000d540 0000035fH .edata                  DATA
 0003:00000000 0000020cH .idata$5                DATA
 0003:0000020c 00000004H .CRT$XCA                DATA
 0003:00000210 00000004H .CRT$XCAA               DATA
 0003:00000214 00000004H .CRT$XCU                DATA
 0003:00000218 00000004H .CRT$XCZ                DATA
 0003:0000021c 00000004H .CRT$XIA                DATA
 0003:00000220 00000004H .CRT$XIZ                DATA
 0003:00000224 00000004H .CRT$XPA                DATA
 0003:00000228 00000004H .CRT$XPZ                DATA
 0003:0000022c 00000004H .CRT$XTA                DATA
 0003:00000230 00000004H .CRT$XTZ                DATA
 0003:00000238 0000032cH .data                   DATA
 0003:00000568 00001490H .bss                    DATA
 0004:00000000 000009b8H .pdata                  DATA
 0005:00000000 00000058H .rsrc$01                DATA
 0005:00000060 000003f0H .rsrc$02                DATA

  Address         Publics by Value              Rva+Base       Lib:Object

 0000:00000000       ___safe_se_handler_table   00000000     <absolute>
 0000:00000000       ___safe_se_handler_count   00000000     <absolute>
 0001:00000000       ??1CCEPowerControl@@QAA@XZ 10001000 f   CEPowerControl.obj
 0001:000000a0       ?NotifyDeviceRemoved@CCEPowerControl@@QAAXXZ 100010a0 f   CEPowerControl.obj
 0001:000000f4       ?WaitForSingleObjectReset@CCEPowerControl@@QAAKPAXK@Z 100010f4 f   CEPowerControl.obj
 0001:00000178       ?ProcessPowerNotification@CCEPowerControl@@AAAXPAX@Z 10001178 f   CEPowerControl.obj
 0001:00000260       ?MonitorSystemPowerState@CCEPowerControl@@QAAXXZ 10001260 f   CEPowerControl.obj
 0001:000007a4       ?ThreadFunc@@YAKPAX@Z      100017a4 f   CEPowerControl.obj
 0001:000007b8       ??0CCEPowerControl@@QAA@P6AHHHPAX@ZH00@Z 100017b8 f   CEPowerControl.obj
 0001:00000934       ??0CircularBuffer@@QAA@XZ  10001934 f   circularbuffer.obj
 0001:00000950       ?Write@CircularBuffer@@QAAHPAEI@Z 10001950 f   circularbuffer.obj
 0001:00000ae8       ?Write@CircularBuffer@@QAAHPAEI0I@Z 10001ae8 f   circularbuffer.obj
 0001:00000cf0       ?HasData@CircularBuffer@@QAAHXZ 10001cf0 f   circularbuffer.obj
 0001:00000d34       ?DataBytesInBuffer@CircularBuffer@@QAAKXZ 10001d34 f   circularbuffer.obj
 0001:00000d6c       ?ResetBuffer@CircularBuffer@@QAAXXZ 10001d6c f   circularbuffer.obj
 0001:00000da4       ?Read@CircularBuffer@@QAAHPAEIPAI@Z 10001da4 f   circularbuffer.obj
 0001:00000f7c       ?Init@CircularBuffer@@QAAXIH@Z 10001f7c f   circularbuffer.obj
 0001:0000101c       ?GetBufferSize@CircularBuffer@@QAAKXZ 1000201c f   circularbuffer.obj
 0001:00001024       ?DeInit@CircularBuffer@@QAAXXZ 10002024 f   circularbuffer.obj
 0001:00001078       ??1CircularBuffer@@QAA@XZ  10002078 f   circularbuffer.obj
 0001:00001084       ?LogCritical@@YAXPA_WZZ    10002084 f i commdevice.obj
 0001:000010e4       ??0CommDevice@@QAA@PB_W@Z  100020e4 f   commdevice.obj
 0001:00001274       ??1CommDevice@@UAA@XZ      10002274 f   commdevice.obj
 0001:00001300       ?ReOpen@CommDevice@@QAAKXZ 10002300 f   commdevice.obj
 0001:000013e0       ?CardRemovedNotify@CommDevice@@AAAXH@Z 100023e0 f   commdevice.obj
 0001:00001444       ?SetHostJustResumedEvent@CommDevice@@QAAXXZ 10002444 f   commdevice.obj
 0001:0000147c       ?DevicePowerNotify@@YAHHHPAX@Z 1000247c f   commdevice.obj
 0001:0000152c       ??_GCommDevice@@UAAPAXI@Z  1000252c f i commdevice.obj
 0001:0000152c       ??_ECommDevice@@UAAPAXI@Z  1000252c f i commdevice.obj
 0001:00001558       ?Open@CommDevice@@QAAKKKH@Z 10002558 f   commdevice.obj
 0001:00001830       ?Close@CommDevice@@QAAHH@Z 10002830 f   commdevice.obj
 0001:00001b08       ?Read@CommDevice@@QAAKPAXK@Z 10002b08 f   commdevice.obj
 0001:00001d6c       ?Write@CommDevice@@QAAKPBXK@Z 10002d6c f   commdevice.obj
 0001:00001ff4       ?IoControl@CommDevice@@QAAHKPAEK0KPAK@Z 10002ff4 f   commdevice.obj
 0001:00002374       ?DeInitPowerControl@CommDevice@@QAAXXZ 10003374 f   commdevice.obj
 0001:000023dc       ?WMP_Init@@YAKPB_WPBX@Z    100033dc f   commentry.obj
 0001:0000242c       ?WMP_Deinit@@YAHK@Z        1000342c f   commentry.obj
 0001:0000245c       ?WMP_Open@@YAKKKK@Z        1000345c f   commentry.obj
 0001:0000247c       ?WMP_Close@@YAHK@Z         1000347c f   commentry.obj
 0001:000024a8       ?WMP_Read@@YAKKPAXK@Z      100034a8 f   commentry.obj
 0001:000024ac       ?WMP_Write@@YAKKPBXK@Z     100034ac f   commentry.obj
 0001:000024b0       ?WMP_Seek@@YAKKJG@Z        100034b0 f   commentry.obj
 0001:000024c4       ?WMP_PowerUp@@YAXK@Z       100034c4 f   commentry.obj
 0001:000024c8       ?WMP_IOControl@@YAHKKPAEK0KPAK@Z 100034c8 f   commentry.obj
 0001:000024f4       ??0CtlTransaction@@QAA@XZ  100034f4 f i CtlService.obj
 0001:00002524       ??0CtlService@@QAA@XZ      10003524 f   CtlService.obj
 0001:000025ac       ??1CtlService@@UAA@XZ      100035ac f   CtlService.obj
 0001:000025f0       ?Initialize@CtlService@@QAA_NPAUQMI_CHANNEL@@@Z 100035f0 f   CtlService.obj
 0001:0000262c       ?Shutdown@CtlService@@QAAXXZ 1000362c f   CtlService.obj
 0001:00002680       ?HandleTransactionResponse@CtlService@@IAAXPAEG@Z 10003680 f   CtlService.obj
 0001:00002708       ?ReadNotify@CtlService@@QAAXPAEG@Z 10003708 f   CtlService.obj
 0001:00002724       ?NewTransactionId@CtlService@@IAAEXZ 10003724 f   CtlService.obj
 0001:0000275c       ?AddToOutstandingList@CtlService@@IAAXPAVCtlTransaction@@@Z 1000375c f   CtlService.obj
 0001:00002790       ?RemoveFromOutstandingList@CtlService@@IAAXPAVCtlTransaction@@@Z 10003790 f   CtlService.obj
 0001:000027c8       ?AddToFreeList@CtlService@@QAAXPAVCtlTransaction@@@Z 100037c8 f   CtlService.obj
 0001:000027fc       ?GetFromFreeList@CtlService@@QAAPAVCtlTransaction@@XZ 100037fc f   CtlService.obj
 0001:00002838       ??_GCtlService@@UAAPAXI@Z  10003838 f i CtlService.obj
 0001:00002838       ??_ECtlService@@UAAPAXI@Z  10003838 f i CtlService.obj
 0001:0000285c       ?ProcessSynchronousTransaction@CtlService@@QAAHPAVCtlTransaction@@GK@Z 1000385c f   CtlService.obj
 0001:000029e0       ??0QmiTransaction@@QAA@XZ  100039e0 f i DmsService.obj
 0001:00002a1c       ??1CtlTransaction@@QAA@XZ  10003a1c f i CtlService.obj
 0001:00002a1c       ??1QmiTransaction@@QAA@XZ  10003a1c f i DmsService.obj
 0001:00002a24       ??0DmsService@@QAA@XZ      10003a24 f   DmsService.obj
 0001:00002ab0       ??1DmsService@@UAA@XZ      10003ab0 f   DmsService.obj
 0001:00002af8       ?Initialize@DmsService@@QAA_NPAUQMI_CHANNEL@@E@Z 10003af8 f   DmsService.obj
 0001:00002b3c       ?HandleTransactionResponse@DmsService@@IAAXPAEG@Z 10003b3c f   DmsService.obj
 0001:00002bd4       ?ReadNotify@DmsService@@QAAXPAEG@Z 10003bd4 f   DmsService.obj
 0001:00002bf0       ?NewTransactionId@DmsService@@IAAGXZ 10003bf0 f   DmsService.obj
 0001:00002bf0       ?NewTransactionId@WdsService@@IAAGXZ 10003bf0 f   WdsService.obj
 0001:00002c2c       ?AddToOutstandingList@WdsService@@IAAXPAVQmiTransaction@@@Z 10003c2c f   WdsService.obj
 0001:00002c2c       ?AddToOutstandingList@DmsService@@IAAXPAVQmiTransaction@@@Z 10003c2c f   DmsService.obj
 0001:00002c60       ?GetFromFreeList@WdsService@@QAAPAVQmiTransaction@@XZ 10003c60 f   WdsService.obj
 0001:00002c60       ?GetFromFreeList@DmsService@@QAAPAVQmiTransaction@@XZ 10003c60 f   DmsService.obj
 0001:00002c9c       ??_EDmsService@@UAAPAXI@Z  10003c9c f i DmsService.obj
 0001:00002c9c       ??_GDmsService@@UAAPAXI@Z  10003c9c f i DmsService.obj
 0001:00002cc0       ?ProcessSynchronousTransaction@DmsService@@QAAHPAVQmiTransaction@@GK@Z 10003cc0 f   DmsService.obj
 0001:00002dec       ?PMInitialize@@YAHXZ       10003dec f   pmcommon.obj
 0001:00002dec       ?WrpCheckForHang@@YAEPAX@Z 10003dec f   wrpcard.obj
 0001:00002df4       ?WrpShutDown@@YAXPAX@Z     10003df4 f   wrpcard.obj
 0001:00002df4       ?WrpPnPEventNotify@@YAXPAXW4_NDIS_DEVICE_PNP_EVENT@@0K@Z 10003df4 f   wrpcard.obj
 0001:00002df4       ?WMP_PowerDown@@YAXK@Z     10003df4 f   commentry.obj
 0001:00002df4       ?PMShutdown@@YAXPAUsAdapterConfig@@@Z 10003df4 f   pmcommon.obj
 0001:00002df8       ?time4PPPLog@@YAEPAK@Z     10003df8 f   PPP4pcap.obj
 0001:00002e88       ??1CPPP4pcap@@QAA@XZ       10003e88 f   PPP4pcap.obj
 0001:00002ec4       ?WriteLogFile@CPPP4pcap@@QAAKKPBXK@Z 10003ec4 f   PPP4pcap.obj
 0001:00003064       ?WriteNewTime@CPPP4pcap@@QAAKK@Z 10004064 f   PPP4pcap.obj
 0001:00003130       ??0CPPP4pcap@@QAA@K@Z      10004130 f   PPP4pcap.obj
 0001:000031dc       ?qlIsListEmpty@@YAEPAU_LIST_ENTRY@@@Z 100041dc f   qlmanage.obj
 0001:000031f8       ?qlremovenext_signalnotempty@@YAPAU_LIST_ENTRY@@PAU1@PAU_NDIS_SPIN_LOCK@@PAU_NDIS_EVENT@@@Z 100041f8 f   qlmanage.obj
 0001:0000325c       ?qlinserttail_signalnotempty@@YAXPAU_LIST_ENTRY@@PAU_NDIS_SPIN_LOCK@@0PAU_NDIS_EVENT@@@Z 1000425c f   qlmanage.obj
 0001:000032b8       ?RetrieveVersionInfo@@YAHPAU_QMICTL_GET_VERSION_RESP_MSG@@@Z 100042b8 f   qmi.obj
 0001:00003528       ?GetQMIVersions@@YAHXZ     10004528 f   qmi.obj
 0001:00003600       ?GetClientID@@YAHW4_QMI_SERVICE_TYPE@@PAEPAW4_QMI_ERROR_CODE_TYPE@@@Z 10004600 f   qmi.obj
 0001:000036f4       ?ReleaseClientID@@YAHW4_QMI_SERVICE_TYPE@@E@Z 100046f4 f   qmi.obj
 0001:000037ec       ?DmsGetDeviceManufacturer@@YAHPADH@Z 100047ec f   qmi.obj
 0001:000038c4       ?DmsGetDeviceMsisdn@@YAHPADH@Z 100048c4 f   qmi.obj
 0001:0000399c       ?WdsSetEventReportIndicationCallback@@YAXP6AXPAXPAEG@Z0@Z 1000499c f   qmi.obj
 0001:000039b4       ?WdsSetEventReportAsync@@YAHHP6AXPAXPAEG@Z0@Z 100049b4 f   qmi.obj
 0001:00003aa4       ?WdsSetGetPacketServiceStatusIndicationCallbackCallback@@YAXP6AXPAXPAEG@Z0@Z 10004aa4 f   qmi.obj
 0001:00003abc       ?WdsGetCurrentChannelRate@@YAHPAK000@Z 10004abc f   qmi.obj
 0001:00003c0c       ?SendQMIMessage@@YAKPAUQMI_CHANNEL@@PAEGEW4_QMI_SERVICE_TYPE@@@Z 10004c0c f   qmi.obj
 0001:00003ca8       ?ConfigPowerSaveSetting@@YAHKGEPAGPAW4_QMI_ERROR_CODE_TYPE@@@Z 10004ca8 f   qmi.obj
 0001:00003e44       ?SetPowerSaveMode@@YAHK@Z  10004e44 f   qmi.obj
 0001:00003f50       ?QMI_Init@@YAPAXPB_WPBX@Z  10004f50 f   qmicom.obj
 0001:00004034       ?QMI_Open@@YAPAXPAXKK@Z    10005034 f   qmicom.obj
 0001:000044ac       ?QMI_Close@@YAHPAUQMI_OPEN_INFO@@@Z 100054ac f   qmicom.obj
 0001:00004684       ?QMI_Deinit@@YAHPAUQMI_PORT_MDD@@@Z 10005684 f   qmicom.obj
 0001:00004708       ?QMI_Read@@YAKPAXPAEK@Z    10005708 f   qmicom.obj
 0001:000048a8       ?QMI_Write@@YAKPAXPAEK@Z   100058a8 f   qmicom.obj
 0001:00004a4c       ?EvaluateEventFlag@@YAXPAUQMI_PORT_MDD@@K@Z 10005a4c f   qmicom.obj
 0001:00004a4c       ?EvaluateEventFlag@@YAXPAUVSP_PORT_MDD@@K@Z 10005a4c f   swicom.obj
 0001:00004b4c       ?QmiWaitCommEvent@@YAHPAUQMI_OPEN_INFO@@PAKPAU_OVERLAPPED@@@Z 10005b4c f   qmicom.obj
 0001:000050bc       ?ProcessClientMsg@@YAXPAUQMI_OPEN_INFO@@PAEK@Z 100060bc f   qmicom.obj
 0001:00005114       ?QMI_IOControl@@YAHPAUQMI_OPEN_INFO@@KPAEK1KPAK@Z 10006114 f   qmicom.obj
 0001:00005844       ??0RilOutContextPool@@QAA@XZ 10006844 f   RilOutContextPool.obj
 0001:00005908       ??1RilOutContextPool@@UAA@XZ 10006908 f   RilOutContextPool.obj
 0001:00005944       ?SetContextId@RilOutContextPool@@QAAXK@Z 10006944 f   RilOutContextPool.obj
 0001:00005950       ?SetStatusCallback@RilOutContextPool@@QAAXP6AXPAXPAUrilndisstatus_tag@@@Z0@Z 10006950 f   RilOutContextPool.obj
 0001:00005960       ?Allocate@RilOutContextPool@@QAAPAURilOutContext@@XZ 10006960 f   RilOutContextPool.obj
 0001:00005a64       ?Free@RilOutContextPool@@QAAXPAURilOutContext@@@Z 10006a64 f   RilOutContextPool.obj
 0001:00005b3c       ?AddToPendingList@RilOutContextPool@@QAAXPAURilOutContext@@@Z 10006b3c f   RilOutContextPool.obj
 0001:00005b90       ?RemoveFromToPendingList@RilOutContextPool@@QAAPAURilOutContext@@XZ 10006b90 f   RilOutContextPool.obj
 0001:00005bfc       ??_GRilOutContextPool@@UAAPAXI@Z 10006bfc f i RilOutContextPool.obj
 0001:00005bfc       ??_ERilOutContextPool@@UAAPAXI@Z 10006bfc f i RilOutContextPool.obj
 0001:00005c20       ??0RilPacketPool@@QAA@XZ   10006c20 f   RilPacketPool.obj
 0001:00005cd0       ?SetContextId@RilPacketPool@@QAAXK@Z 10006cd0 f   RilPacketPool.obj
 0001:00005d00       ?Allocate@RilPacketPool@@QAAPAUrilndispacket_tag@@XZ 10006d00 f   RilPacketPool.obj
 0001:00005d90       ?Free@RilPacketPool@@QAAXPAUrilndispacket_tag@@@Z 10006d90 f   RilPacketPool.obj
 0001:00005de4       ??_ERilPacketPool@@UAAPAXI@Z 10006de4 f i RilPacketPool.obj
 0001:00005de4       ??_GRilPacketPool@@UAAPAXI@Z 10006de4 f i RilPacketPool.obj
 0001:00005e28       ?SWD_Init@@YAPAXPB_WPBX@Z  10006e28 f   swdcom.obj
 0001:00005f68       ?SWD_Open@@YAPAXPAXKK@Z    10006f68 f   swdcom.obj
 0001:00006074       ?SWD_Close@@YAHPAUSWD_OPEN_INFO@@@Z 10007074 f   swdcom.obj
 0001:0000615c       ?SWD_Deinit@@YAHPAUSWD_MDD@@@Z 1000715c f   swdcom.obj
 0001:000061dc       ?SWD_IOControl@@YAHPAUSWD_OPEN_INFO@@KPAEK1KPAK@Z 100071dc f   swdcom.obj
 0001:00006438       ?ReadDWORDValue@@YAJPAUHKEY__@@PB_W1PAK@Z 10007438 f   swicom.obj
 0001:000064a4       ?WriteDWORDValue@@YAJPAUHKEY__@@PB_W1K@Z 100074a4 f   swicom.obj
 0001:00006530       ?ReadStrValue@@YAJPAUHKEY__@@PB_W1QA_WK@Z 10007530 f   swicom.obj
 0001:000065b0       ?WriteStrValue@@YAJPAUHKEY__@@PB_W1QA_WK@Z 100075b0 f   swicom.obj
 0001:00006634       DllMain                    10007634 f   swicom.obj
 0001:00006734       ?dumpBytesData@@YAXKPA_WPAEK@Z 10007734 f   swicom.obj
 0001:000069b0       ?initDefaultDCB@@YAXPAU_DCB@@@Z 100079b0 f   swicom.obj
 0001:00006a24       ?initDefaultCommProp@@YAXPAU_COMMPROP@@@Z 10007a24 f   swicom.obj
 0001:00006aac       ?IsSystemCleanBooting@@YAHXZ 10007aac f   swicom.obj
 0001:00006afc       ?SWI_Init@@YAPAXPB_WPBX@Z  10007afc f   swicom.obj
 0001:00006c00       ?PortStatusIsOpen@@YAEPAUVSP_OPEN_INFO@@H@Z 10007c00 f   swicom.obj
 0001:00006c74       ?PortStatusOpen@@YAXPAUVSP_OPEN_INFO@@@Z 10007c74 f   swicom.obj
 0001:00006cb0       ?PortStatusClose@@YAXPAUVSP_OPEN_INFO@@@Z 10007cb0 f   swicom.obj
 0001:00006cf8       ?SWI_Open@@YAPAXPAXKK@Z    10007cf8 f   swicom.obj
 0001:00007300       ?SWI_Close@@YAHPAUVSP_OPEN_INFO@@@Z 10008300 f   swicom.obj
 0001:0000768c       ?SWI_Deinit@@YAHPAUVSP_PORT_MDD@@@Z 1000868c f   swicom.obj
 0001:00007720       ?SWI_Read@@YAKPAXPAEK@Z    10008720 f   swicom.obj
 0001:00007874       ?SWI_Write@@YAKPAXPAEK@Z   10008874 f   swicom.obj
 0001:00007a6c       ?SWI_Seek@@YAKPAXJK@Z      10008a6c f   swicom.obj
 0001:00007a6c       ?QMI_Seek@@YAKPAXJK@Z      10008a6c f   qmicom.obj
 0001:00007a6c       ?SWD_Seek@@YAKPAXJK@Z      10008a6c f   swdcom.obj
 0001:00007a6c       ?SWD_Read@@YAKPAXPAEK@Z    10008a6c f   swdcom.obj
 0001:00007a6c       ?SWD_Write@@YAKPAXPAEK@Z   10008a6c f   swdcom.obj
 0001:00007a74       ?SWI_PowerDown@@YAHPAX@Z   10008a74 f   swicom.obj
 0001:00007a74       ?SWI_PowerUp@@YAHPAX@Z     10008a74 f   swicom.obj
 0001:00007a84       ?DbgPrintEventMask@@YAXK@Z 10008a84 f   swicom.obj
 0001:00007c44       ?VspSetSerialStatusState@@YAXPAUVSP_PORT_MDD@@EEEEG@Z 10008c44 f   swicom.obj
 0001:00007d60       ?VspAddToReadQueue@@YAEPAUVSP_PORT_MDD@@PAEK@Z 10008d60 f   swicom.obj
 0001:00007f08       ?VspWaitCommEvent@@YAHPAUVSP_OPEN_INFO@@PAKPAU_OVERLAPPED@@@Z 10008f08 f   swicom.obj
 0001:00008768       ?SWI_IOControl@@YAHPAUVSP_OPEN_INFO@@KPAEK1KPAK@Z 10009768 f   swicom.obj
 0001:00008f4c       ?GetAvailStoreMem@@YAKXZ   10009f4c f   swiroutines.obj
 0001:00008f7c       ?GetMemUsed@@YAKXZ         10009f7c f   swiroutines.obj
 0001:00008fa8       ?OpenInModemBulkPipe10@@YAPAXU_USB_ENDPOINT_DESCRIPTOR@@@Z 10009fa8 f   swiroutines.obj
 0001:00008fa8       ?OpenOutModemBulkPipe11@@YAPAXU_USB_ENDPOINT_DESCRIPTOR@@@Z 10009fa8 f   swiroutines.obj
 0001:00009018       ?OpenInterruptModemPipe1@@YAPAXU_USB_ENDPOINT_DESCRIPTOR@@@Z 1000a018 f   swiroutines.obj
 0001:0000907c       ?SWIUSBPowerControl@@YAHHHPAH@Z 1000a07c f   swiroutines.obj
 0001:00009180       ?SWICreateMemory@@YAPAEK@Z 1000a180 f   swiroutines.obj
 0001:00009240       ?SWIFreeMemory@@YAXPAE@Z   1000a240 f   swiroutines.obj
 0001:00009340       ?IsQMIChannelBusy@@YAHXZ   1000a340 f   swiroutines.obj
 0001:000093a4       ?HwIsModemBusy@@YAEPAU_SW_MODEM@@@Z 1000a3a4 f   swiroutines.obj
 0001:0000945c       ?EnsurePortResumed@@YAHK@Z 1000a45c f   swiroutines.obj
 0001:0000952c       ?GetDescriptor@@YAHEEGPAEGPAK@Z 1000a52c f   swiroutines.obj
 0001:00009618       ?HandleInvalidModem@@YAXGG@Z 1000a618 f   swiroutines.obj
 0001:00009634       ?SendSyncGPSCommand@@YAHPAUVSP_PORT_MDD@@W4_GPS_CMD@@@Z 1000a634 f   swiroutines.obj
 0001:00009758       ?DoSendInitControlRequests@@YAHKKH@Z 1000a758 f   swiroutines.obj
 0001:00009a64       ?SendInitControlRequests@@YAHKKH@Z 1000aa64 f   swiroutines.obj
 0001:00009af8       ?SendHostToInterfaceCommandSync@@YAHPAU_USB_DEVICE_REQUEST@@PAEKK@Z 1000aaf8 f   swiroutines.obj
 0001:00009c5c       ?UsbGetMuxMode@@YAHPAW4_MUX_INSTANCE_STATE@@@Z 1000ac5c f   swiroutines.obj
 0001:00009d08       ?UsbSetMuxMode@@YAHPAU_MUX_MODE_PARAMETERS@@@Z 1000ad08 f   swiroutines.obj
 0001:00009d9c       ?UsbSetNmxMode@@YAHXZ      1000ad9c f   swiroutines.obj
 0001:00009de8       ?UsbGetNMEAMode@@YAHPAG@Z  1000ade8 f   swiroutines.obj
 0001:00009e34       ?UsbSetNMEAMode@@YAHG@Z    1000ae34 f   swiroutines.obj
 0001:00009e80       ?UsbSetHostSleepPowerState@@YAHG@Z 1000ae80 f   swiroutines.obj
 0001:00009fc8       ?TransferCompletionRoutine@@YAKPAX@Z 1000afc8 f   swiusb.obj
 0001:00009fec       ?DispatchQMIMsg@@YAXPAEG@Z 1000afec f   swiusb.obj
 0001:0000a24c       ?QMIThread@@YAXPAPAX@Z     1000b24c f   swiusb.obj
 0001:0000a684       ?StartQMIThreads@@YAXXZ    1000b684 f   swiusb.obj
 0001:0000a6d0       ?InitializeQMIChannel@@YAHE@Z 1000b6d0 f   swiusb.obj
 0001:0000a880       ?CleanupQMIChannel@@YAXXZ  1000b880 f   swiusb.obj
 0001:0000aa38       ?CleanupDirectIpChannel@@YAXXZ 1000ba38 f   swiusb.obj
 0001:0000ac04       ?StartDmsService@@YAHXZ    1000bc04 f   swiusb.obj
 0001:0000ad50       ?StopDmsService@@YAXXZ     1000bd50 f   swiusb.obj
 0001:0000ada8       ?StartWdsService@@YAHXZ    1000bda8 f   swiusb.obj
 0001:0000aef4       ?StopWdsService@@YAXXZ     1000bef4 f   swiusb.obj
 0001:0000af44       ?SWIResetPipe@@YAHPBU_USB_FUNCS@@PAX@Z 1000bf44 f   swiusb.obj
 0001:0000af98       ?CreateRegistryPath@@YAXPA_WKPBU_USB_DRIVER_SETTINGS@@@Z 1000bf98 f   swiusb.obj
 0001:0000b0c4       ?SetDeviceStateActive@@YAXH@Z 1000c0c4 f   swiusb.obj
 0001:0000b128       ?SetUSBActivityEvent@@YAXXZ 1000c128 f   swiusb.obj
 0001:0000b160       ?SetDeviceStateInActive@@YAXH@Z 1000c160 f   swiusb.obj
 0001:0000b510       ?RilNdisReceivePacketDone@@YAXQAUrilndispacket_tag@@@Z 1000c510 f   swiusb.obj
 0001:0000b528       ?RilNdisSendPacket@@YAXQAUrilndispacket_tag@@@Z 1000c528 f   swiusb.obj
 0001:0000b698       ?processMsmSerialState@@YAXPAU_SW_MODEM@@PADK@Z 1000c698 f   swiusb.obj
 0001:0000c358       ?DisplayMemoryStatus@@YAXXZ 1000d358 f   swiusb.obj
 0001:0000c3a4       ?USBDeviceNotifications@@YAHPAXKPAPAK111@Z 1000d3a4 f   swiusb.obj
 0001:0000c9c4       ?WMWdsGetPacketServiceStatusInd@@YAXPAXPAEG@Z 1000d9c4 f   swiusb.obj
 0001:0000c9e8       USBInstallDriver           1000d9e8 f   swiusb.obj
 0001:0000ca04       ?GetDeviceInstalledEvent@@YAPAXXZ 1000da04 f   swiusb.obj
 0001:0000ca14       ?HookUsbToAdapter@@YAXPAUsAdapterConfig@@@Z 1000da14 f   swiusb.obj
 0001:0000ca70       ?HelpResumingOS@@YAKPAPAX@Z 1000da70 f   swiusb.obj
 0001:0000ca94       ?ActivityThread@@YAXPAPAX@Z 1000da94 f   swiusb.obj
 0001:0000f134       ?InitializeDirectIpChannel@@YAHPBU_USB_INTERFACE@@PA_W@Z 10010134 f   swiusb.obj
 0001:0000f81c       USBDeviceAttach            1001081c f   swiusb.obj
 0001:00011210       ??0WdsService@@QAA@XZ      10012210 f   WdsService.obj
 0001:000112ac       ??1WdsService@@UAA@XZ      100122ac f   WdsService.obj
 0001:000112f4       ?SetEventReportIndicationCallback@WdsService@@QAAXP6AXPAXPAEG@Z0@Z 100122f4 f   WdsService.obj
 0001:00011300       ?SetGetPacketServiceStatusIndicationCallbackCallback@WdsService@@QAAXP6AXPAXPAEG@Z0@Z 10012300 f   WdsService.obj
 0001:0001130c       ?Initialize@WdsService@@QAA_NPAUQMI_CHANNEL@@E@Z 1001230c f   WdsService.obj
 0001:00011350       ?Shutdown@WdsService@@QAAXXZ 10012350 f   WdsService.obj
 0001:00011350       ?Shutdown@DmsService@@QAAXXZ 10012350 f   DmsService.obj
 0001:000113a4       ?HandleTransactionIndication@WdsService@@IAAXPAEG@Z 100123a4 f   WdsService.obj
 0001:00011418       ?RemoveFromOutstandingList@WdsService@@IAAXPAVQmiTransaction@@@Z 10012418 f   WdsService.obj
 0001:00011418       ?RemoveFromOutstandingList@DmsService@@IAAXPAVQmiTransaction@@@Z 10012418 f   DmsService.obj
 0001:00011450       ?AddToFreeList@WdsService@@QAAXPAVQmiTransaction@@@Z 10012450 f   WdsService.obj
 0001:00011450       ?AddToFreeList@DmsService@@QAAXPAVQmiTransaction@@@Z 10012450 f   DmsService.obj
 0001:00011484       ??_EWdsService@@UAAPAXI@Z  10012484 f i WdsService.obj
 0001:00011484       ??_GWdsService@@UAAPAXI@Z  10012484 f i WdsService.obj
 0001:000114a8       ?ProcessSynchronousTransaction@WdsService@@QAAHPAVQmiTransaction@@GK@Z 100124a8 f   WdsService.obj
 0001:0001159c       ?ProcessAsynchronousTransaction@WdsService@@QAAHPAVQmiTransaction@@GP6AXPAXPAEG@Z1@Z 1001259c f   WdsService.obj
 0001:0001165c       ?HandleTransactionResponse@WdsService@@IAAXPAEG@Z 1001265c f   WdsService.obj
 0001:00011720       ?ReadNotify@WdsService@@QAAXPAEG@Z 10012720 f   WdsService.obj
 0001:00011864       ?WrpHalt@@YAXPAX@Z         10012864 f   wrp.obj
 0001:00011954       ?WrpInitialize@@YAHPAHPAIPAW4_NDIS_MEDIUM@@IPAX3@Z 10012954 f   wrp.obj
 0001:00011c2c       ?DriverEntry@@YAJPAU_CEDRIVER_OBJECT@@PAU_UNICODE_STRING@@@Z 10012c2c f   wrp.obj
 0001:00011dc4       ?WrpSend@@YAHPAXPAU_NDIS_PACKET@@I@Z 10012dc4 f   wrpcard.obj
 0001:00011e20       ?WrpIndicateReceive@@YAXPAUsAdapterConfig@@PAEI@Z 10012e20 f   wrpcard.obj
 0001:00011edc       ?WrpTransferData@@YAHPAU_NDIS_PACKET@@PAIPAX2II@Z 10012edc f   wrpcard.obj
 0001:0001202c       ?WrpReset@@YAHPAEPAX@Z     1001302c f   wrpcard.obj
 0001:00012058       ?WrpBuildLinearEthPacket@@YAEPAU_NDIS_PACKET@@PAEPAI@Z 10013058 f   wrpcard.obj
 0001:00012120       ?WrpIndicateSendComplete@@YAXPAUsAdapterConfig@@PAU_NDIS_PACKET@@E@Z 10013120 f   wrpcard.obj
 0001:000121a0       ?WrpQmiShutdown@@YAXPAUsAdapterConfig@@@Z 100131a0 f   wrpcard.obj
 0001:000121c0       ?WrpWdsSetEventReportResp@@YAXPAXPAEG@Z 100131c0 f   wrpcard.obj
 0001:000121d8       ?WrpWdsEventReportInd@@YAXPAXPAEG@Z 100131d8 f   wrpcard.obj
 0001:00012358       ?WrpReconfigTimerDpc@@YAXPAX000@Z 10013358 f   wrpcard.obj
 0001:000123c4       ?WrpWdsGetPacketServiceStatusInd@@YAXPAXPAEG@Z 100133c4 f   wrpcard.obj
 0001:00012558       ?WrpQmiInitialize@@YAEPAUsAdapterConfig@@@Z 10013558 f   wrpcard.obj
 0001:00012658       ?WrpGetDriverBlock@@YAPAUDRIVER_BLOCK@@XZ 10013658 f   wrpdata.obj
 0001:00012664       ?WrpSetAdapterPointer@@YAXPAUsAdapterConfig@@@Z 10013664 f   wrpdata.obj
 0001:00012674       ?WrpSetCardCount@@YAXE@Z   10013674 f   wrpdata.obj
 0001:00012684       ?WrpGetCardCount@@YAKXZ    10013684 f   wrpdata.obj
 0001:00012694       ?WrpSetReset@@YAXPAUsAdapterConfig@@E@Z 10013694 f   wrpdata.obj
 0001:0001269c       ?WrpGetReset@@YAEPAUsAdapterConfig@@@Z 1001369c f   wrpdata.obj
 0001:000126a4       ?WrpAllocateMemory@@YAHPAUsAdapterConfig@@PAPAXIPBD@Z 100136a4 f   wrpmemory.obj
 0001:000126bc       ?WrpFreeMemory@@YAXPAUsAdapterConfig@@PAXIPBD@Z 100136bc f   wrpmemory.obj
 0001:000126dc       ?OidToNameStr@@YAPADK@Z    100136dc f   wrpoid.obj
 0001:00012ffc       ?WrpQueryInfo@@YAHPAXK0KPAK1@Z 10013ffc f   wrpoid.obj
 0001:00013810       ?WrpSetInfo@@YAHPAXK0KPAK1@Z 10014810 f   wrpoid.obj
 0001:00013a64       ?OpenRegistry@@YAXPAHPAPAX1@Z 10014a64 f   wrpregistry.obj
 0001:00013a8c       ?CloseRegistry@@YAXPAPAX@Z 10014a8c f   wrpregistry.obj
 0001:00013aa4       ?ReadRegistry@@YAXPAHPAPAU_NDIS_CONFIGURATION_PARAMETER@@PAPAXPAU_UNICODE_STRING@@W4_NDIS_PARAMETER_TYPE@@@Z 10014aa4 f   wrpregistry.obj
 0001:00013acc       ?ConvertMacAddress@@YAEPAU_NDIS_CONFIGURATION_PARAMETER@@PAE@Z 10014acc f   wrpregistry.obj
 0001:00013bf4       NdisReleaseSpinLock        10014bf4 f   ndis:NDIS.dll
 0001:00013c04       NdisAcquireSpinLock        10014c04 f   ndis:NDIS.dll
 0001:00013c14       NdisResetEvent             10014c14 f   ndis:NDIS.dll
 0001:00013c24       NdisSetEvent               10014c24 f   ndis:NDIS.dll
 0001:00013c34       NdisDeregisterAdapter      10014c34 f   ndis:NDIS.dll
 0001:00013c44       NdisRegisterAdapter        10014c44 f   ndis:NDIS.dll
 0001:00013c54       NdisWriteErrorLogEntry     10014c54 f   ndis:NDIS.dll
 0001:00013c64       NdisFreeSpinLock           10014c64 f   ndis:NDIS.dll
 0001:00013c74       NdisMDeregisterAdapterShutdownHandler 10014c74 f   ndis:NDIS.dll
 0001:00013c84       NdisMSleep                 10014c84 f   ndis:NDIS.dll
 0001:00013c94       NdisFreeEvent              10014c94 f   ndis:NDIS.dll
 0001:00013ca4       NdisWaitEvent              10014ca4 f   ndis:NDIS.dll
 0001:00013cb4       NdisCancelTimer            10014cb4 f   ndis:NDIS.dll
 0001:00013cc4       NdisMSetAttributesEx       10014cc4 f   ndis:NDIS.dll
 0001:00013cd4       NdisMRegisterAdapterShutdownHandler 10014cd4 f   ndis:NDIS.dll
 0001:00013ce4       NdisInitializeTimer        10014ce4 f   ndis:NDIS.dll
 0001:00013cf4       NdisInitializeEvent        10014cf4 f   ndis:NDIS.dll
 0001:00013d04       NdisAllocateSpinLock       10014d04 f   ndis:NDIS.dll
 0001:00013d14       NdisTerminateWrapper       10014d14 f   ndis:NDIS.dll
 0001:00013d24       NdisMRegisterMiniport      10014d24 f   ndis:NDIS.dll
 0001:00013d34       NdisInitializeWrapper      10014d34 f   ndis:NDIS.dll
 0001:00013d44       NdisQueryPacket            10014d44 f   ndis:NDIS.dll
 0001:00013d54       NdisSetTimer               10014d54 f   ndis:NDIS.dll
 0001:00013d64       NdisAllocateMemoryWithTag  10014d64 f   ndis:NDIS.dll
 0001:00013d74       NdisFreeMemory             10014d74 f   ndis:NDIS.dll
 0001:00013d84       NdisOpenConfiguration      10014d84 f   ndis:NDIS.dll
 0001:00013d94       NdisCloseConfiguration     10014d94 f   ndis:NDIS.dll
 0001:00013da4       NdisReadConfiguration      10014da4 f   ndis:NDIS.dll
 0001:00013db4       NdisUnicodeStringToAnsiString 10014db4 f   ndis:NDIS.dll
 0001:00013dc4       htons                      10014dc4 f   ws2:WS2.dll
 0001:00013dd4       htonl                      10014dd4 f   ws2:WS2.dll
 0001:00013de4       EventModify                10014de4 f   coredll:COREDLL.dll
 0001:00013df4       CloseMsgQueue              10014df4 f   coredll:COREDLL.dll
 0001:00013e04       DeleteCriticalSection      10014e04 f   coredll:COREDLL.dll
 0001:00013e14       LeaveCriticalSection       10014e14 f   coredll:COREDLL.dll
 0001:00013e24       CloseHandle                10014e24 f   coredll:COREDLL.dll
 0001:00013e34       NKDbgPrintfW               10014e34 f   coredll:COREDLL.dll
 0001:00013e44       WaitForSingleObject        10014e44 f   coredll:COREDLL.dll
 0001:00013e54       EnterCriticalSection       10014e54 f   coredll:COREDLL.dll
 0001:00013e64       Sleep                      10014e64 f   coredll:COREDLL.dll
 0001:00013e74       GetTickCount               10014e74 f   coredll:COREDLL.dll
 0001:00013e84       GetLastError               10014e84 f   coredll:COREDLL.dll
 0001:00013e94       ReadMsgQueue               10014e94 f   coredll:COREDLL.dll
 0001:00013ea4       memset                     10014ea4 f   coredll:COREDLL.dll
 0001:00013eb4       WaitForMultipleObjects     10014eb4 f   coredll:COREDLL.dll
 0001:00013ec4       CeSetThreadPriority        10014ec4 f   coredll:COREDLL.dll
 0001:00013ed4       RequestPowerNotifications  10014ed4 f   coredll:COREDLL.dll
 0001:00013ee4       CreateMsgQueue             10014ee4 f   coredll:COREDLL.dll
 0001:00013ef4       InitializeCriticalSection  10014ef4 f   coredll:COREDLL.dll
 0001:00013f04       CreateThread               10014f04 f   coredll:COREDLL.dll
 0001:00013f14       CreateEventW               10014f14 f   coredll:COREDLL.dll
 0001:00013f24       memcpy                     10014f24 f   coredll:COREDLL.dll
 0001:00013f34       vswprintf                  10014f34 f   coredll:COREDLL.dll
 0001:00013f44       SetCommMask                10014f44 f   coredll:COREDLL.dll
 0001:00013f54       ??3@YAXPAX@Z               10014f54 f   coredll:COREDLL.dll
 0001:00013f64       SetCommState               10014f64 f   coredll:COREDLL.dll
 0001:00013f74       CreateFileW                10014f74 f   coredll:COREDLL.dll
 0001:00013f84       swprintf                   10014f84 f   coredll:COREDLL.dll
 0001:00013f94       ??2@YAPAXI@Z               10014f94 f   coredll:COREDLL.dll
 0001:00013fa4       GetCommModemStatus         10014fa4 f   coredll:COREDLL.dll
 0001:00013fb4       EscapeCommFunction         10014fb4 f   coredll:COREDLL.dll
 0001:00013fc4       SetLastError               10014fc4 f   coredll:COREDLL.dll
 0001:00013fd4       ReadFile                   10014fd4 f   coredll:COREDLL.dll
 0001:00013fe4       WriteFile                  10014fe4 f   coredll:COREDLL.dll
 0001:00013ff4       DeviceIoControl            10014ff4 f   coredll:COREDLL.dll
 0001:00014004       ??_L@YAXPAXIHP6AX0@Z1@Z    10015004 f   coredll:COREDLL.dll
 0001:00014014       ??_M@YAXPAXIHP6AX0@Z@Z     10015014 f   coredll:COREDLL.dll
 0001:00014024       SystemTimeToFileTime       10015024 f   coredll:COREDLL.dll
 0001:00014034       GetSystemTime              10015034 f   coredll:COREDLL.dll
 0001:00014044       FlushFileBuffers           10015044 f   coredll:COREDLL.dll
 0001:00014054       SetFilePointer             10015054 f   coredll:COREDLL.dll
 0001:00014064       RegCloseKey                10015064 f   coredll:COREDLL.dll
 0001:00014074       RegDeleteValueW            10015074 f   coredll:COREDLL.dll
 0001:00014084       RegOpenKeyExW              10015084 f   coredll:COREDLL.dll
 0001:00014094       wsprintfW                  10015094 f   coredll:COREDLL.dll
 0001:000140a4       wcslen                     100150a4 f   coredll:COREDLL.dll
 0001:000140b4       strncpy                    100150b4 f   coredll:COREDLL.dll
 0001:000140c4       __C_specific_handler       100150c4 f   coredll:COREDLL.dll
 0001:000140d4       InterlockedExchange        100150d4 f   coredll:COREDLL.dll
 0001:000140e4       LocalAlloc                 100150e4 f   coredll:COREDLL.dll
 0001:000140f4       LocalFree                  100150f4 f   coredll:COREDLL.dll
 0001:00014104       RegQueryValueExW           10015104 f   coredll:COREDLL.dll
 0001:00014114       RegSetValueExW             10015114 f   coredll:COREDLL.dll
 0001:00014124       RegCreateKeyExW            10015124 f   coredll:COREDLL.dll
 0001:00014134       wcsncat                    10015134 f   coredll:COREDLL.dll
 0001:00014144       _snwprintf                 10015144 f   coredll:COREDLL.dll
 0001:00014154       rand                       10015154 f   coredll:COREDLL.dll
 0001:00014164       wcscat                     10015164 f   coredll:COREDLL.dll
 0001:00014174       FindClose                  10015174 f   coredll:COREDLL.dll
 0001:00014184       FindFirstFileW             10015184 f   coredll:COREDLL.dll
 0001:00014194       _wcsicmp                   10015194 f   coredll:COREDLL.dll
 0001:000141a4       GetStoreInformation        100151a4 f   coredll:COREDLL.dll
 0001:000141b4       GlobalMemoryStatus         100151b4 f   coredll:COREDLL.dll
 0001:000141c4       HeapAlloc                  100151c4 f   coredll:COREDLL.dll
 0001:000141d4       GetProcessHeap             100151d4 f   coredll:COREDLL.dll
 0001:000141e4       VirtualAlloc               100151e4 f   coredll:COREDLL.dll
 0001:000141f4       HeapFree                   100151f4 f   coredll:COREDLL.dll
 0001:00014204       VirtualFree                10015204 f   coredll:COREDLL.dll
 0001:00014214       IsBadReadPtr               10015214 f   coredll:COREDLL.dll
 0001:00014224       TerminateThread            10015224 f   coredll:COREDLL.dll
 0001:00014234       StringCchCatW              10015234 f   coredll:COREDLL.dll
 0001:00014244       StringCchPrintfW           10015244 f   coredll:COREDLL.dll
 0001:00014254       DeactivateDevice           10015254 f   coredll:COREDLL.dll
 0001:00014264       SetSystemPowerState        10015264 f   coredll:COREDLL.dll
 0001:00014274       wcsstr                     10015274 f   coredll:COREDLL.dll
 0001:00014284       _wcslwr                    10015284 f   coredll:COREDLL.dll
 0001:00014294       GetSystemPowerState        10015294 f   coredll:COREDLL.dll
 0001:000142a4       ActivateDeviceEx           100152a4 f   coredll:COREDLL.dll
 0001:000142b4       SystemParametersInfoW      100152b4 f   coredll:COREDLL.dll
 0001:000142c4       MultiByteToWideChar        100152c4 f   coredll:COREDLL.dll
 0001:000142d4       wcscpy                     100152d4 f   coredll:COREDLL.dll
 0001:000142e4       wcscmp                     100152e4 f   coredll:COREDLL.dll
 0001:000142f4       memcmp                     100152f4 f   coredll:COREDLL.dll
 0001:00014304       strlen                     10015304 f   coredll:COREDLL.dll
 0001:00014314       sprintf                    10015314 f   coredll:COREDLL.dll
 0001:00014324       __security_check_cookie    10015324     corelibc:armsecgs.obj
 0001:00014338       __gsfailure                10015338     corelibc:armsecgs.obj
 0001:0001437c       _onexit                    1001537c f   corelibc:onexit.obj
 0001:00014428       atexit                     10015428 f   corelibc:onexit.obj
 0001:00014448       _DllMainCRTStartup         10015448 f   corelibc:pegdmain.obj
 0001:000144e0       __security_init_cookie     100154e0 f   corelibc:seccinit.obj
 0001:00014530       _cinit                     10015530 f   corelibc:crt0dat.obj
 0001:000146a0       _cexit                     100156a0 f   corelibc:crt0dat.obj
 0001:000146bc       __GSHandlerCheckCommon     100156bc f   LIBCMT:gshandler.obj
 0001:00014704       __GSHandlerCheck           10015704 f   LIBCMT:gshandler.obj
 0001:0001473c       __FrameUnwindToState       1001573c f   LIBCMT:frame_ce.obj
 0001:00014ab4       ?_DestructExceptionObject@@YAXPAUEHExceptionRecord@@E@Z 10015ab4 f   LIBCMT:frame_ce.obj
 0001:00014b20       ?_OffsetToAddress@@YAPAXHPAKK@Z 10015b20 f   LIBCMT:frame_ce.obj
 0001:00014b6c       ?FindFrameInfo@@YAPAU_FrameInfo@@PAK@Z 10015b6c f   LIBCMT:frame_ce.obj
 0001:00014bac       ?FindCatchFrameInfo@@YAPAU_FrameInfo@@PAK@Z 10015bac f   LIBCMT:frame_ce.obj
 0001:00014bec       ?_GetRangeOfTrysToCheck@@YAPBU_s_TryBlockMapEntry@@PBU_s_FuncInfo@@HHPAI1@Z 10015bec f   LIBCMT:frame_ce.obj
 0001:000155f8       __InternalCxxFrameHandler  100165f8 f   LIBCMT:frame_ce.obj
 0001:00015750       __CxxFrameHandler3         10016750 f   LIBCMT:frame_ce.obj
 0001:00015788       __GSHandlerCheck_EH        10016788 f   LIBCMT:gshandlereh.obj
 0001:0001581c       GetCRTStorage              1001681c f   LIBCMT:corecrt.obj
 0001:000158e8       _CallSettingFrame          100168e8     LIBCMT:handlers_arm.obj
 0001:0001592c       ?FindFrameForUnwind@@YAPAKPAKPBU_s_FuncInfo@@@Z 1001692c f   LIBCMT:mdframe_arm.obj
 0001:00015974       ?FindCatchFrame@@YAPAKPAKK@Z 10016974 f   LIBCMT:mdframe_arm.obj
 0001:000159c0       ?AdjustFrameForCatch@@YAPAKPAKPBU_s_FuncInfo@@@Z 100169c0 f   LIBCMT:mdframe_arm.obj
 0001:000159f8       ?GetCurrentState@@YAHPAKPAU_DISPATCHER_CONTEXT@@PBU_s_FuncInfo@@@Z 100169f8 f   LIBCMT:ehstate_arm_mips.obj
 0001:00015a54       __report_gsfailure         10016a54 f   coredll:COREDLL.dll
 0001:00015a64       LocalReAlloc               10016a64 f   coredll:COREDLL.dll
 0001:00015a74       LocalSize                  10016a74 f   coredll:COREDLL.dll
 0001:00015a84       __security_gen_cookie      10016a84 f   coredll:COREDLL.dll
 0001:00015a94       strcmp                     10016a94 f   coredll:COREDLL.dll
 0001:00015aa4       ?terminate@std@@YAXXZ      10016aa4 f   coredll:COREDLL.dll
 0001:00015ab4       memmove                    10016ab4 f   coredll:COREDLL.dll
 0001:00015ac4       TlsCall                    10016ac4 f   coredll:COREDLL.dll
 0001:00015ad4       TlsSetValue                10016ad4 f   coredll:COREDLL.dll
 0001:00015ae4       TlsGetValue                10016ae4 f   coredll:COREDLL.dll
 0001:00015af4       InterlockedCompareExchange 10016af4 f   coredll:COREDLL.dll
 0002:00000020       ??_C@_1GE@FFDGHJLP@?$AAC?$AAC?$AAE?$AAP?$AAo?$AAw?$AAe?$AAr?$AAC?$AAo?$AAn?$AAt?$AAr?$AAo?$AAl?$AA?5?$AAm?$AA_?$AAh?$AAM?$AAo?$AAn?$AAi?$AAt?$AAo?$AAr?$AAT?$AAh?$AAr?$AAe?$AAa?$AAd@ 10017020     CEPowerControl.obj
 0002:00000088       ??_C@_1FA@GOPBKAMB@?$AA?$CF?$AAs?$AA?3?$AA?7?$AAI?$AAg?$AAn?$AAo?$AAr?$AAe?$AA?5?$AAM?$AAe?$AAs?$AAs?$AAa?$AAg?$AAe?$AA?5?$AAt?$AAo?$AAo?$AA?5?$AAs?$AAh?$AAo?$AAr?$AAt?$AA?3?$AA?5?$AA?$CF?$AAd@ 10017088     CEPowerControl.obj
 0002:000000d8       ??_C@_1DK@EHLMGLMA@?$AAP?$AAB?$AAT?$AA_?$AAR?$AAE?$AAS?$AAU?$AAM?$AAE?$AA?0?$AA?5?$AAt?$AAi?$AAc?$AAk?$AAC?$AAo?$AAu?$AAn?$AAt?$AA?5?$AA?$DN?$AA?5?$AA?$CF?$AAd?$AA?$AN?$AA?6?$AA?$AA@ 100170d8     CEPowerControl.obj
 0002:00000114       ??_C@_1DK@OGBDJKCH@?$AAU?$AAn?$AAh?$AAa?$AAn?$AAd?$AAl?$AAe?$AAd?$AA?5?$AAP?$AAo?$AAw?$AAe?$AAr?$AA?5?$AAM?$AAe?$AAs?$AAs?$AAa?$AAg?$AAe?$AA?3?$AA?$CF?$AAd?$AA?$AN?$AA?6?$AA?$AA@ 10017114     CEPowerControl.obj
 0002:00000150       ??_C@_1EC@HGHJEAP@?$AAP?$AAr?$AAo?$AAc?$AAe?$AAs?$AAs?$AAi?$AAn?$AAg?$AA?5?$AAp?$AAo?$AAw?$AAe?$AAr?$AA?5?$AAn?$AAo?$AAt?$AAi?$AAf?$AAi?$AAc?$AAa?$AAt?$AAi?$AAo?$AAn?$AAs?$AA?$AN?$AA?6@ 10017150     CEPowerControl.obj
 0002:00000194       ??_C@_1DA@PJJNJDEO@?$AAR?$AAe?$AAa?$AAd?$AAM?$AAs?$AAg?$AAQ?$AAu?$AAe?$AAu?$AAe?$AA?3?$AA?5?$AAE?$AAR?$AAR?$AAO?$AAR?$AA?3?$AA?$CF?$AAd?$AA?6?$AA?$AA@ 10017194     CEPowerControl.obj
 0002:000001c8       ??_C@_1NM@IPHMFOJK@?$AAC?$AAE?$AAP?$AAo?$AAw?$AAe?$AAr?$AAC?$AAo?$AAn?$AAt?$AAr?$AAo?$AAl?$AA?3?$AAM?$AAo?$AAn?$AAi?$AAt?$AAo?$AAr?$AAS?$AAy?$AAs?$AAt?$AAe?$AAm?$AAP?$AAo?$AAw?$AAe@ 100171c8     CEPowerControl.obj
 0002:000002a8       ??_C@_1IK@HBIOAECJ@?$AAC?$AAE?$AAP?$AAo?$AAw?$AAe?$AAr?$AAC?$AAo?$AAn?$AAt?$AAr?$AAo?$AAl?$AA?3?$AAW?$AAa?$AAi?$AAt?$AA?5?$AAd?$AAu?$AAr?$AAi?$AAn?$AAg?$AA?5?$AAD?$AAE?$AAV?$AAI?$AAC@ 100172a8     CEPowerControl.obj
 0002:00000338       ??_C@_1II@IDIFPKKM@?$AAC?$AAE?$AAP?$AAo?$AAw?$AAe?$AAr?$AAC?$AAo?$AAn?$AAt?$AAr?$AAo?$AAl?$AA?3?$AAW?$AAa?$AAi?$AAt?$AA?5?$AAd?$AAu?$AAr?$AAi?$AAn?$AAg?$AA?5?$AAD?$AAE?$AAV?$AAI?$AAC@ 10017338     CEPowerControl.obj
 0002:000003c0       ??_C@_1NO@EACPHDBD@?$AAC?$AAE?$AAP?$AAo?$AAw?$AAe?$AAr?$AAC?$AAo?$AAn?$AAt?$AAr?$AAo?$AAl?$AA?3?$AAT?$AAh?$AAr?$AAe?$AAa?$AAd?$AA?5?$AAl?$AAo?$AAo?$AAp?$AA?3?$AA?5?$AAN?$AAo?$AAt?$AAi@ 100173c0     CEPowerControl.obj
 0002:000004a0       ??_C@_1BAO@NHGFFGBD@?$AAC?$AAE?$AAP?$AAo?$AAw?$AAe?$AAr?$AAC?$AAo?$AAn?$AAt?$AAr?$AAo?$AAl?$AA?3?$AAm?$AA_?$AAd?$AAw?$AAL?$AAa?$AAs?$AAt?$AAD?$AAe?$AAv?$AAi?$AAc?$AAe?$AAR?$AAe?$AAs@ 100174a0     CEPowerControl.obj
 0002:000005b0       ??_C@_1BBO@GAGCALEB@?$AAC?$AAE?$AAP?$AAo?$AAw?$AAe?$AAr?$AAC?$AAo?$AAn?$AAt?$AAr?$AAo?$AAl?$AA?3?$AAU?$AAS?$AAB?$AA?5?$AAd?$AAe?$AAv?$AAi?$AAc?$AAe?$AA?5?$AAd?$AAi?$AAd?$AAn?$AA?8?$AAt@ 100175b0     CEPowerControl.obj
 0002:000006d0       ??_C@_1BMC@IOFFFKCL@?$AAC?$AAE?$AAP?$AAo?$AAw?$AAe?$AAr?$AAC?$AAo?$AAn?$AAt?$AAr?$AAo?$AAl?$AA?3?$AAd?$AAw?$AAW?$AAa?$AAi?$AAt?$AAR?$AAe?$AAs?$AAu?$AAl?$AAt?$AAN?$AAe?$AAg?$AAa?$AAt@ 100176d0     CEPowerControl.obj
 0002:00000898       ??_C@_1BEA@LOJFFOJB@?$AAC?$AAE?$AAP?$AAo?$AAw?$AAe?$AAr?$AAC?$AAo?$AAn?$AAt?$AAr?$AAo?$AAl?$AA?3?$AAC?$AAo?$AAu?$AAl?$AAd?$AAn?$AA?8?$AAt?$AA?5?$AAs?$AAe?$AAe?$AA?5?$AAd?$AAe?$AAv?$AAi@ 10017898     CEPowerControl.obj
 0002:000009d8       ??_C@_1BAM@JPACNBAA@?$AAC?$AAE?$AAP?$AAo?$AAw?$AAe?$AAr?$AAC?$AAo?$AAn?$AAt?$AAr?$AAo?$AAl?$AA?3?$AAT?$AAh?$AAr?$AAe?$AAa?$AAd?$AA?5?$AAl?$AAo?$AAo?$AAp?$AA?3?$AA?5?$AAN?$AAo?$AAt?$AAi@ 100179d8     CEPowerControl.obj
 0002:00000ae8       ??_C@_1BBC@JPEJOJDE@?$AAC?$AAE?$AAP?$AAo?$AAw?$AAe?$AAr?$AAC?$AAo?$AAn?$AAt?$AAr?$AAo?$AAl?$AA?3?$AA?5?$AAH?$AAa?$AAn?$AAd?$AAl?$AAi?$AAn?$AAg?$AA?5?$AAP?$AAo?$AAr?$AAt?$AA?5?$AAR?$AAe@ 10017ae8     CEPowerControl.obj
 0002:00000c00       ??_C@_1OI@NGLLBKKN@?$AAC?$AAE?$AAP?$AAo?$AAw?$AAe?$AAr?$AAC?$AAo?$AAn?$AAt?$AAr?$AAo?$AAl?$AA?3?$AAT?$AAh?$AAr?$AAe?$AAa?$AAd?$AA?5?$AAl?$AAo?$AAo?$AAp?$AA?0?$AA?5?$AAp?$AAr?$AAo?$AAc@ 10017c00     CEPowerControl.obj
 0002:00000ce8       ??_C@_1OA@BGNNMBHN@?$AAC?$AAE?$AAP?$AAo?$AAw?$AAe?$AAr?$AAC?$AAo?$AAn?$AAt?$AAr?$AAo?$AAl?$AA?3?$AA?5?$AAT?$AAi?$AAc?$AAk?$AA?5?$AAc?$AAo?$AAu?$AAn?$AAt?$AA?5?$AAj?$AAu?$AAs?$AAt?$AA_@ 10017ce8     CEPowerControl.obj
 0002:00000dc8       ??_C@_1HO@CDNJAJLO@?$AAC?$AAE?$AAP?$AAo?$AAw?$AAe?$AAr?$AAC?$AAo?$AAn?$AAt?$AAr?$AAo?$AAl?$AA?3?$AAB?$AAo?$AAt?$AAh?$AA?5?$AAD?$AAe?$AAv?$AAi?$AAc?$AAe?$AA?5?$AAA?$AAr?$AAr?$AAi?$AAv@ 10017dc8     CEPowerControl.obj
 0002:00000e48       ??_C@_1GC@JLILFAHH@?$AAC?$AAE?$AAP?$AAo?$AAw?$AAe?$AAr?$AAC?$AAo?$AAn?$AAt?$AAr?$AAo?$AAl?$AA?3?$AAT?$AAh?$AAr?$AAe?$AAa?$AAd?$AA?5?$AAb?$AAe?$AAg?$AAi?$AAn?$AA?3?$AA?5?$AAN?$AAo?$AAt@ 10017e48     CEPowerControl.obj
 0002:00000eb0       ??_C@_1GA@CHKBDOHF@?$AAC?$AAE?$AAP?$AAo?$AAw?$AAe?$AAr?$AAC?$AAo?$AAn?$AAt?$AAr?$AAo?$AAl?$AA?3?$AAT?$AAh?$AAr?$AAe?$AAa?$AAd?$AA?5?$AAb?$AAe?$AAg?$AAi?$AAn?$AA?3?$AA?5?$AAN?$AAo?$AAt@ 10017eb0     CEPowerControl.obj
 0002:00000f10       ??_C@_1II@LGHEKFO@?$AAC?$AAE?$AAP?$AAo?$AAw?$AAe?$AAr?$AAC?$AAo?$AAn?$AAt?$AAr?$AAo?$AAl?$AA?3?$AAI?$AAn?$AAv?$AAa?$AAl?$AAi?$AAd?$AA?5?$AAu?$AAs?$AAa?$AAg?$AAe?$AA?4?$AA?5?$AAS?$AAt@ 10017f10     CEPowerControl.obj
 0002:00000f98       ??_C@_1FK@HPDAFKGO@?$AAF?$AAa?$AAi?$AAl?$AA?5?$AAt?$AAo?$AA?5?$AAC?$AAr?$AAe?$AAa?$AAt?$AAe?$AA?5?$AAm?$AA_?$AAh?$AAR?$AAe?$AAa?$AAd?$AA?5?$AAm?$AAs?$AAg?$AA?5?$AAq?$AAu?$AAe?$AAu?$AAe@ 10017f98     CEPowerControl.obj
 0002:00000ff8       ??_C@_1HC@BKFMJEPM@?$AAF?$AAa?$AAi?$AAl?$AA?5?$AAt?$AAo?$AA?5?$AAr?$AAe?$AAg?$AAi?$AAs?$AAt?$AAe?$AAr?$AA?5?$AAf?$AAo?$AAr?$AA?5?$AAP?$AAB?$AAT?$AA_?$AAR?$AAE?$AAS?$AAU?$AAM?$AAE?$AA?5@ 10017ff8     CEPowerControl.obj
 0002:0000106c       ??_C@_1DK@PFMIPBAF@?$AAa?$AAc?$AAt?$AAi?$AAv?$AAe?$AAl?$AAo?$AAw?$AA_?$AAs?$AAw?$AAi?$AAm?$AAd?$AAm?$AAr?$AAe?$AAs?$AAe?$AAt?$AA_?$AAs?$AAi?$AAg?$AAn?$AAa?$AAl?$AA?$AA@ 1001806c     CEPowerControl.obj
 0002:000010a8       ??_C@_1GG@INDIPEOO@?$AAW?$AAr?$AAi?$AAt?$AAe?$AA?3?$AA?5?$AAb?$AAi?$AAg?$AA?5?$AAp?$AAr?$AAo?$AAb?$AAl?$AAe?$AAm?$AA?4?$AA?5?$AAR?$AAe?$AAa?$AAd?$AA?5?$AAi?$AAs?$AA?5?$AAf?$AAa?$AAs?$AAt@ 100180a8     circularbuffer.obj
 0002:00001110       ??_C@_1HO@FLKDCNCC@?$AA?$CK?$AA?$CK?$AA?$CK?$AA?$CC?$AAE?$AAN?$AAD?$AA?$CC?$AA?5?$AAn?$AAo?$AAt?$AA?5?$AAd?$AAe?$AAt?$AAe?$AAc?$AAt?$AAe?$AAd?$AA?4?$AA?5?$AAC?$AAi?$AAr?$AAc?$AAu?$AAl?$AAa?$AAr?$AA?5@ 10018110     circularbuffer.obj
 0002:00001190       ??_C@_1NE@PICEGIJP@?$AA?$CK?$AA?$CK?$AA?$CK?$AAC?$AAi?$AAr?$AAc?$AAu?$AAl?$AAa?$AAr?$AA?5?$AAb?$AAu?$AAf?$AAf?$AAe?$AAr?$AA?5?$AAo?$AAv?$AAe?$AAr?$AAf?$AAl?$AAo?$AAw?$AA?5?$AAm?$AA_?$AAn?$AAA@ 10018190     circularbuffer.obj
 0002:00001268       ??_C@_1NO@EKCOMFAH@?$AA?$CK?$AA?$CK?$AA?$CK?$AAC?$AAi?$AAr?$AAc?$AAu?$AAl?$AAa?$AAr?$AA?5?$AAb?$AAu?$AAf?$AAf?$AAe?$AAr?$AA?5?$AAo?$AAv?$AAe?$AAr?$AAf?$AAl?$AAo?$AAw?$AA?5?$AAm?$AA_?$AAn?$AAA@ 10018268     circularbuffer.obj
 0002:00001348       ??_C@_1GE@LJJLCDGE@?$AAR?$AAe?$AAa?$AAd?$AA?3?$AA?5?$AAb?$AAi?$AAg?$AA?5?$AAp?$AAr?$AAo?$AAb?$AAl?$AAe?$AAm?$AA?4?$AA?5?$AAR?$AAe?$AAa?$AAd?$AA?5?$AAi?$AAs?$AA?5?$AAf?$AAa?$AAs?$AAt?$AAe@ 10018348     circularbuffer.obj
 0002:000013b0       ??_C@_1IE@LHDGJNPM@?$AAN?$AAo?$AA?5?$AAm?$AAo?$AAr?$AAe?$AA?5?$AAm?$AAe?$AAm?$AAo?$AAr?$AAy?$AA?5?$AAf?$AAo?$AAr?$AA?5?$AAc?$AAr?$AAe?$AAa?$AAt?$AAi?$AAn?$AAg?$AA?5?$AAc?$AAi?$AAr?$AAc@ 100183b0     circularbuffer.obj
 0002:00001434       ??_C@_15JNBOKNOG@?$AA?$AN?$AA?6?$AA?$AA@ 10018434     commdevice.obj
 0002:0000143c       ??_C@_1BG@PCNLLPJI@?$AAA?$AAC?$AA_?$AAE?$AAJ?$AAE?$AAC?$AAT?$AAE?$AAD?$AA?$AA@ 1001843c     commdevice.obj
 0002:00001454       ??_C@_1BI@DJOGOGFO@?$AAA?$AAC?$AA_?$AAI?$AAN?$AAS?$AAE?$AAR?$AAT?$AAE?$AAD?$AA?$AA@ 10018454     commdevice.obj
 0002:00001470       ??_C@_1FO@IMNIACHN@?$AAF?$AAa?$AAi?$AAl?$AA?5?$AAt?$AAo?$AA?5?$AAr?$AAe?$AAa?$AAd?$AA?5?$AAI?$AAn?$AAd?$AAe?$AAx?$AA?5?$AAf?$AAr?$AAo?$AAm?$AA?5?$AAt?$AAh?$AAe?$AAB?$AAu?$AAi?$AAl?$AAt@ 10018470     commdevice.obj
 0002:000014d0       ??_C@_1EG@NPNBLLHL@?$AAP?$AAo?$AAr?$AAt?$AA?5?$AAi?$AAn?$AAd?$AAe?$AAx?$AA?5?$AAi?$AAs?$AA?5?$AA?$FL?$AAW?$AAM?$AAP?$AA?5?$AA?$DN?$AA?5?$AA?$CF?$AAd?$AA?0?$AA?5?$AAS?$AAW?$AAI?$AA?5?$AA?$DN?$AA?5?$AA?$CF@ 100184d0     commdevice.obj
 0002:00001518       ??_C@_1M@EENNDIOJ@?$AAI?$AAn?$AAd?$AAe?$AAx?$AA?$AA@ 10018518     commdevice.obj
 0002:00001524       ??_C@_1BC@PMPEPIHB@?$AAS?$AAW?$AAI?$AAI?$AAn?$AAd?$AAe?$AAx?$AA?$AA@ 10018524     commdevice.obj
 0002:00001538       ??_C@_1GG@BOBNACNC@?$AAF?$AAa?$AAi?$AAl?$AA?5?$AAt?$AAo?$AA?5?$AAr?$AAe?$AAa?$AAd?$AA?5?$AAt?$AAh?$AAe?$AAB?$AAu?$AAi?$AAl?$AAt?$AAI?$AAn?$AAK?$AAe?$AAy?$AAP?$AAa?$AAt?$AAh?$AA?5?$AAf@ 10018538     commdevice.obj
 0002:000015a0       ??_7CommDevice@@6B@        100185a0     commdevice.obj
 0002:000015a4       ??_C@_17KACEIPNC@?$AAK?$AAe?$AAy?$AA?$AA@ 100185a4     commdevice.obj
 0002:000015b0       ??_C@_1GK@BLANJEIC@?$AAW?$AAM?$AAP?$AA?$CF?$AAd?$AA?5?$AAR?$AAe?$AAO?$AAp?$AAe?$AAn?$AA?3?$AA?5?$AAU?$AAn?$AAb?$AAl?$AAo?$AAc?$AAk?$AA?5?$AAI?$AAO?$AAC?$AAT?$AAL?$AA?5?$AAw?$AAi?$AAt?$AAh@ 100185b0     commdevice.obj
 0002:00001620       ??_C@_1FO@NMLNDHD@?$AAW?$AAM?$AAP?$AA?$CF?$AAd?$AA?5?$AAR?$AAe?$AAO?$AAp?$AAe?$AAn?$AA?9?$AA?$DO?$AAS?$AAe?$AAt?$AAC?$AAo?$AAm?$AAm?$AAM?$AAa?$AAs?$AAk?$AA?5?$AAf?$AAa?$AAi?$AAl?$AAe?$AAd@ 10018620     commdevice.obj
 0002:00001680       ??_C@_1GO@LLCBOIDK@?$AAW?$AAM?$AAP?$AA?$CF?$AAd?$AA?5?$AAR?$AAe?$AAO?$AAp?$AAe?$AAn?$AA?5?$AAa?$AAb?$AAo?$AAu?$AAt?$AA?5?$AAt?$AAo?$AA?5?$AAS?$AAe?$AAt?$AAC?$AAo?$AAm?$AAm?$AAM?$AAa?$AAs@ 10018680     commdevice.obj
 0002:000016f0       ??_C@_1GK@GBPGEFFD@?$AAF?$AAa?$AAi?$AAl?$AA?5?$AAR?$AAe?$AAO?$AAp?$AAe?$AAn?$AA?5?$AAW?$AAM?$AAP?$AA?$CF?$AAd?$AA?5?$AAb?$AAe?$AAc?$AAa?$AAu?$AAs?$AAe?$AA?5?$AAm?$AA_?$AAb?$AAG?$AAo?$AAO@ 100186f0     commdevice.obj
 0002:00001760       ??_C@_1FO@PAKHDLDE@?$AAS?$AAe?$AAt?$AA?5?$AAm?$AA_?$AAh?$AAD?$AAe?$AAv?$AAi?$AAc?$AAe?$AAJ?$AAu?$AAs?$AAt?$AAR?$AAe?$AAs?$AAu?$AAm?$AAe?$AAd?$AAE?$AAv?$AAe?$AAn?$AAt?$AA?5?$AA?$DN?$AA?5@ 10018760     commdevice.obj
 0002:000017c0       ??_C@_1EI@GDPOIHHM@?$AAC?$AAo?$AAm?$AAm?$AAD?$AAe?$AAv?$AAi?$AAc?$AAe?$AA?5?$AAC?$AAo?$AAu?$AAl?$AAd?$AA?5?$AAn?$AAo?$AAt?$AA?5?$AAs?$AAe?$AAe?$AA?5?$AAD?$AAA?$AA?5?$AAi?$AAn?$AA?5?$AAt@ 100187c0     commdevice.obj
 0002:00001808       ??_C@_1GM@LGGHIDNG@?$AAW?$AAM?$AAP?$AA?$CF?$AAd?$AA?5?$AAi?$AAs?$AA?5?$AAN?$AAO?$AAT?$AA?5?$AAr?$AAe?$AAa?$AAd?$AAy?$AA?5?$AAt?$AAo?$AA?5?$AAc?$AAo?$AAm?$AAm?$AAu?$AAn?$AAi?$AAc?$AAa?$AAt@ 10018808     commdevice.obj
 0002:00001878       ??_C@_1EG@EKBNBMB@?$AAW?$AAM?$AAP?$AA?$CF?$AAd?$AA?5?$AAc?$AAo?$AAm?$AAm?$AAu?$AAn?$AAi?$AAc?$AAa?$AAt?$AAi?$AAo?$AAn?$AA?5?$AAr?$AAe?$AAa?$AAd?$AAi?$AAn?$AAe?$AAs?$AAs?$AA?5?$AA?$DN?$AA?5@ 10018878     commdevice.obj
 0002:000018c0       ??_C@_1DM@FBAPKGPA@?$AAW?$AAM?$AAP?$AA?$CF?$AAd?$AA?5?$AAi?$AAs?$AA?5?$AAr?$AAe?$AAa?$AAd?$AAy?$AA?5?$AAt?$AAo?$AA?5?$AAc?$AAo?$AAm?$AAm?$AAu?$AAn?$AAi?$AAc?$AAa?$AAt?$AAe?$AA?$AA@ 100188c0     commdevice.obj
 0002:00001958       ??_C@_1JG@ILBNLMLF@?$AAC?$AAo?$AAm?$AAm?$AAD?$AAe?$AAv?$AAi?$AAc?$AAe?$AA?3?$AA?3?$AAO?$AAp?$AAe?$AAn?$AA?5?$AAf?$AAa?$AAi?$AAl?$AAe?$AAd?$AA?5?$AAb?$AAc?$AAo?$AAs?$AA?5?$AAm?$AA_?$AAd@ 10018958     commdevice.obj
 0002:000019f0       ??_C@_1EG@GKDDFDAN@?$AAW?$AAM?$AAP?$AA?$CF?$AAd?$AA?5?$AAO?$AAp?$AAe?$AAn?$AA?5?$AAe?$AAr?$AAr?$AA?5?$AA?$DN?$AA?5?$AA?$CF?$AAd?$AA?0?$AA?5?$AAr?$AAe?$AAt?$AAr?$AAy?$AAC?$AAn?$AAt?$AA?5?$AA?$DN?$AA?5@ 100189f0     commdevice.obj
 0002:00001a38       ??_C@_1CK@MJMJPDJF@?$AAW?$AAM?$AAP?$AA?$CF?$AAd?$AA?5?$AAO?$AAp?$AAe?$AAn?$AA?5?$AAs?$AAu?$AAc?$AAc?$AAe?$AAe?$AAd?$AAe?$AAd?$AA?$AA@ 10018a38     commdevice.obj
 0002:00001a64       ??_C@_1O@OCAHMOCM@?$AAS?$AAW?$AAI?$AA?$CF?$AAd?$AA?3?$AA?$AA@ 10018a64     commdevice.obj
 0002:00001a78       ??_C@_1EG@MKKLBDPE@?$AAP?$AAP?$AAP?$AA4?$AAc?$AAa?$AAp?$AA?5?$AAf?$AAo?$AAr?$AA?5?$AAp?$AAo?$AAr?$AAt?$AA?5?$AAn?$AAu?$AAm?$AAb?$AAe?$AAr?$AA?5?$AA?$CF?$AAd?$AA?5?$AAc?$AAr?$AAe?$AAa?$AAt@ 10018a78     commdevice.obj
 0002:00001ac0       ??_C@_1DE@IPPHJDLK@?$AAm?$AA_?$AAe?$AAD?$AAa?$AAt?$AAa?$AAL?$AAo?$AAg?$AA?5?$AAf?$AAo?$AAr?$AA?5?$AAW?$AAM?$AAP?$AA?$CF?$AAd?$AA?5?$AA?$DN?$AA?5?$AA?$CF?$AAd?$AA?$AA@ 10018ac0     commdevice.obj
 0002:00001af4       ??_C@_1O@FHLFJINA@?$AAS?$AAS?$AA_?$AAL?$AAo?$AAg?$AA?$AA@ 10018af4     commdevice.obj
 0002:00001b04       ??_C@_1CA@LKDEBJIA@?$AAG?$AAo?$AAO?$AAn?$AAO?$AAv?$AAe?$AAr?$AAS?$AAu?$AAs?$AAp?$AAe?$AAn?$AAd?$AA?$AA@ 10018b04     commdevice.obj
 0002:00001b24       ??_C@_1BM@BFCLBFKH@?$AAW?$AAM?$AAP?$AA?$CF?$AAd?$AA?5?$AAc?$AAl?$AAo?$AAs?$AAe?$AAd?$AA?$CB?$AA?$AA@ 10018b24     commdevice.obj
 0002:00001b40       ??_C@_1IO@JCBLENE@?$AAR?$AAe?$AAO?$AAp?$AAe?$AAn?$AA?5?$AAW?$AAM?$AAP?$AA?$CF?$AAd?$AA?5?$AAp?$AAa?$AAs?$AAs?$AAe?$AAd?$AA?5?$AAb?$AAu?$AAt?$AA?5?$AAC?$AAL?$AAR?$AAD?$AAT?$AAR?$AA?5?$AAf@ 10018b40     commdevice.obj
 0002:00001bd0       ??_C@_1HI@BAJPCNBC@?$AAW?$AAM?$AAP?$AA?$CF?$AAd?$AA?5?$AAF?$AAo?$AAr?$AAc?$AAe?$AA?5?$AAC?$AAL?$AAR?$AAD?$AAT?$AAR?$AA?5?$AAw?$AAo?$AAr?$AAk?$AAs?$AA?5?$AAa?$AAr?$AAo?$AAu?$AAn?$AAd?$AA?0@ 10018bd0     commdevice.obj
 0002:00001c48       ??_C@_1JO@CHJFLLCJ@?$AAD?$AAT?$AAR?$AA?5?$AAd?$AAr?$AAo?$AAp?$AAp?$AAe?$AAd?$AA?4?$AA?5?$AAM?$AAo?$AAd?$AAe?$AAm?$AA?5?$AAs?$AAt?$AAi?$AAl?$AAl?$AA?5?$AAi?$AAn?$AA?5?$AAa?$AA?5?$AAd?$AAa@ 10018c48     commdevice.obj
 0002:00001ce8       ??_C@_1KG@FCAKMMCN@?$AAD?$AAT?$AAR?$AA?5?$AAd?$AAr?$AAo?$AAp?$AAp?$AAe?$AAd?$AA?4?$AA?5?$AAM?$AAo?$AAd?$AAe?$AAm?$AA?5?$AAs?$AAt?$AAi?$AAl?$AAl?$AA?5?$AAi?$AAn?$AA?5?$AAa?$AA?5?$AAd?$AAa@ 10018ce8     commdevice.obj
 0002:00001d90       ??_C@_1CM@PJBODCMP@?$AAW?$AAM?$AAP?$AA?$CF?$AAd?$AA?5?$AAC?$AAL?$AAR?$AAD?$AAT?$AAR?$AA?5?$AAn?$AAo?$AAr?$AAm?$AAa?$AAl?$AAl?$AAy?$AA?$AA@ 10018d90     commdevice.obj
 0002:00001dc0       ??_C@_1HK@CLCNBPLF@?$AAD?$AAo?$AAn?$AA?8?$AAt?$AA?5?$AAf?$AAa?$AAk?$AAe?$AA?5?$AAI?$AAn?$AAs?$AAe?$AAr?$AAt?$AAC?$AAa?$AAr?$AAd?$AAE?$AAv?$AAe?$AAn?$AAt?$AA?5?$AAs?$AAi?$AAn?$AAc?$AAe@ 10018dc0     commdevice.obj
 0002:00001e40       ??_C@_1EM@PEGFNJPI@?$AAP?$AAu?$AAl?$AAs?$AAe?$AA?5?$AAI?$AAn?$AAs?$AAe?$AAr?$AAt?$AAC?$AAa?$AAr?$AAd?$AAE?$AAv?$AAe?$AAn?$AAt?$AA?0?$AA?5?$AAt?$AAi?$AAc?$AAk?$AAC?$AAo?$AAu?$AAn?$AAt@ 10018e40     commdevice.obj
 0002:00001e90       ??_C@_1EK@KFLOCNFD@?$AAP?$AAu?$AAl?$AAs?$AAe?$AA?5?$AAE?$AAj?$AAe?$AAc?$AAt?$AAC?$AAa?$AAr?$AAd?$AAE?$AAv?$AAe?$AAn?$AAt?$AA?0?$AA?5?$AAt?$AAi?$AAc?$AAk?$AAC?$AAo?$AAu?$AAn?$AAt?$AA?5@ 10018e90     commdevice.obj
 0002:00001edc       ??_C@_1DE@FOMFACKO@?$AAC?$AAl?$AAo?$AAs?$AAe?$AA?5?$AAW?$AAM?$AAP?$AA?$CF?$AAd?$AA?0?$AA?5?$AAb?$AAS?$AAi?$AAl?$AAe?$AAn?$AAt?$AA?5?$AA?$DN?$AA?5?$AA?$CF?$AAd?$AA?$AA@ 10018edc     commdevice.obj
 0002:00001f10       ??_C@_1FA@LBDOLEHK@?$AAW?$AAM?$AAP?$AA?$CF?$AAd?$AA?5?$AAR?$AAe?$AAa?$AAd?$AAf?$AAi?$AAl?$AAe?$AA?5?$AAS?$AAt?$AAe?$AAp?$AA?5?$AA4?$AA?5?$AA?$CI?$AA1?$AAs?$AAt?$AA?5?$AAb?$AAy?$AAt?$AAe?$AA?5@ 10018f10     commdevice.obj
 0002:00001f60       ??_C@_1FA@IIEHLGLO@?$AAW?$AAM?$AAP?$AA?$CF?$AAd?$AA?5?$AAc?$AAa?$AAl?$AAl?$AAs?$AA?5?$AAC?$AAl?$AAo?$AAs?$AAe?$AA?5?$AA?$CI?$AAF?$AAA?$AAL?$AAS?$AAE?$AA?$CJ?$AA?5?$AAf?$AAr?$AAo?$AAm?$AA?5?$AAR@ 10018f60     commdevice.obj
 0002:00001fb0       ??_C@_1FG@KAHDLMAB@?$AAW?$AAM?$AAP?$AA?$CF?$AAd?$AA?5?$AAR?$AAe?$AAa?$AAd?$AAf?$AAi?$AAl?$AAe?$AA?5?$AA?$CI?$AAb?$AA?$FL?$AA5?$AA?0?$AA6?$AA?0?$AA7?$AA?$FN?$AA?5?$AA?$DN?$AA?5?$AA0?$AAx?$AA?$CF?$AAx?$AA?5@ 10018fb0     commdevice.obj
 0002:00002008       ??_C@_1EI@LILONOFL@?$AAW?$AAM?$AAP?$AA?$CF?$AAd?$AA?5?$AAR?$AAe?$AAa?$AAd?$AA?5?$AAf?$AAa?$AAi?$AAl?$AA?5?$AAb?$AAc?$AAo?$AAs?$AA?5?$AAi?$AAn?$AAv?$AAa?$AAl?$AAi?$AAd?$AA?5?$AAh?$AAa?$AAn@ 10019008     commdevice.obj
 0002:00002050       ??_C@_1IG@GALBFLCB@?$AAW?$AAM?$AAP?$AA?$CF?$AAd?$AA?5?$AAm?$AA_?$AAh?$AAD?$AAe?$AAv?$AAi?$AAc?$AAe?$AAJ?$AAu?$AAs?$AAt?$AAR?$AAe?$AAs?$AAu?$AAm?$AAe?$AAd?$AAE?$AAv?$AAe?$AAn?$AAt?$AA?5@ 10019050     commdevice.obj
 0002:000020d8       ??_C@_1FG@OJACNNJ@?$AAW?$AAM?$AAP?$AA?$CF?$AAd?$AA?5?$AAC?$AAa?$AAl?$AAl?$AA?5?$AAC?$AAa?$AAr?$AAd?$AAR?$AAe?$AAm?$AAo?$AAv?$AAe?$AAd?$AAN?$AAo?$AAt?$AAi?$AAf?$AAy?$AA?5?$AAf?$AAr?$AAo@ 100190d8     commdevice.obj
 0002:00002130       ??_C@_1CM@HNPGMACN@?$AAW?$AAM?$AAP?$AA?$CF?$AAd?$AA?5?$AAR?$AAe?$AAa?$AAd?$AAf?$AAi?$AAl?$AAe?$AA?5?$AAS?$AAt?$AAe?$AAp?$AA?5?$AA3?$AA?$AA@ 10019130     commdevice.obj
 0002:0000215c       ??_C@_1CM@MFEKKHEI@?$AAW?$AAM?$AAP?$AA?$CF?$AAd?$AA?5?$AAR?$AAe?$AAa?$AAd?$AAf?$AAi?$AAl?$AAe?$AA?5?$AAS?$AAt?$AAe?$AAp?$AA?5?$AA2?$AA?$AA@ 1001915c     commdevice.obj
 0002:00002188       ??_C@_0BB@KOGIBMHK@CommDevice?3?3Read?$AA@ 10019188     commdevice.obj
 0002:000021a0       ??_C@_1JC@KMBKCBGN@?$AAW?$AAM?$AAP?$AA?$CF?$AAd?$AA?5?$AAm?$AA_?$AAh?$AAD?$AAe?$AAv?$AAi?$AAc?$AAe?$AAJ?$AAu?$AAs?$AAt?$AAR?$AAe?$AAs?$AAu?$AAm?$AAe?$AAd?$AAE?$AAv?$AAe?$AAn?$AAt?$AA?5@ 100191a0     commdevice.obj
 0002:00002234       ??_C@_1CM@NHPPAIKG@?$AAW?$AAM?$AAP?$AA?$CF?$AAd?$AA?5?$AAR?$AAe?$AAa?$AAd?$AAf?$AAi?$AAl?$AAe?$AA?5?$AAS?$AAt?$AAe?$AAp?$AA?5?$AA1?$AA?$AA@ 10019234     commdevice.obj
 0002:00002260       ??_C@_1FC@GBCLDLKB@?$AAW?$AAM?$AAP?$AA?$CF?$AAd?$AA?5?$AAW?$AAr?$AAi?$AAt?$AAe?$AAf?$AAi?$AAl?$AAe?$AA?5?$AAS?$AAt?$AAe?$AAp?$AA?5?$AA5?$AA?5?$AA?$CI?$AA1?$AAs?$AAt?$AA?5?$AAb?$AAy?$AAt?$AAe@ 10019260     commdevice.obj
 0002:000022b4       ??_C@_1CO@NADAHMKB@?$AAW?$AAM?$AAP?$AA?$CF?$AAd?$AA?5?$AAW?$AAr?$AAi?$AAt?$AAe?$AAf?$AAi?$AAl?$AAe?$AA?5?$AAS?$AAt?$AAe?$AAp?$AA?5?$AA4?$AA?$AA@ 100192b4     commdevice.obj
 0002:000022e8       ??_C@_1FC@EMGAOJGI@?$AAW?$AAM?$AAP?$AA?$CF?$AAd?$AA?5?$AAc?$AAa?$AAl?$AAl?$AAs?$AA?5?$AAC?$AAl?$AAo?$AAs?$AAe?$AA?5?$AA?$CI?$AAF?$AAA?$AAL?$AAS?$AAE?$AA?$CJ?$AA?5?$AAf?$AAr?$AAo?$AAm?$AA?5?$AAW@ 100192e8     commdevice.obj
 0002:00002340       ??_C@_1FI@HOLLHOKA@?$AAW?$AAM?$AAP?$AA?$CF?$AAd?$AA?5?$AAW?$AAr?$AAi?$AAt?$AAe?$AAf?$AAi?$AAl?$AAe?$AA?5?$AA?$CI?$AAb?$AA?$FL?$AA5?$AA?0?$AA6?$AA?0?$AA7?$AA?$FN?$AA?5?$AA?$DN?$AA?5?$AA0?$AAx?$AA?$CF?$AAx@ 10019340     commdevice.obj
 0002:00002398       ??_C@_1EK@MIDNAKDB@?$AAW?$AAM?$AAP?$AA?$CF?$AAd?$AA?5?$AAW?$AAr?$AAi?$AAt?$AAe?$AA?5?$AAf?$AAa?$AAi?$AAl?$AA?5?$AAb?$AAc?$AAo?$AAs?$AA?5?$AAi?$AAn?$AAv?$AAa?$AAl?$AAi?$AAd?$AA?5?$AAh?$AAa@ 10019398     commdevice.obj
 0002:000023e8       ??_C@_1GC@BNIFPIHP@?$AAW?$AAM?$AAP?$AA?$CF?$AAd?$AA?5?$AAC?$AAa?$AAl?$AAl?$AA?5?$AAC?$AAa?$AAr?$AAd?$AAR?$AAe?$AAm?$AAo?$AAv?$AAe?$AAd?$AAN?$AAo?$AAt?$AAi?$AAf?$AAy?$AA?5?$AAf?$AAr?$AAo@ 100193e8     commdevice.obj
 0002:0000244c       ??_C@_1CO@ENOHEEBI@?$AAW?$AAM?$AAP?$AA?$CF?$AAd?$AA?5?$AAW?$AAr?$AAi?$AAt?$AAe?$AAf?$AAi?$AAl?$AAe?$AA?5?$AAS?$AAt?$AAe?$AAp?$AA?5?$AA3?$AA?$AA@ 1001944c     commdevice.obj
 0002:0000247c       ??_C@_1CO@PFFLCDHN@?$AAW?$AAM?$AAP?$AA?$CF?$AAd?$AA?5?$AAW?$AAr?$AAi?$AAt?$AAe?$AAf?$AAi?$AAl?$AAe?$AA?5?$AAS?$AAt?$AAe?$AAp?$AA?5?$AA2?$AA?$AA@ 1001947c     commdevice.obj
 0002:000024ac       ??_C@_0BC@PDGLDOGC@CommDevice?3?3Write?$AA@ 100194ac     commdevice.obj
 0002:000024c0       ??_C@_1CO@OHOOIMJD@?$AAW?$AAM?$AAP?$AA?$CF?$AAd?$AA?5?$AAW?$AAr?$AAi?$AAt?$AAe?$AAf?$AAi?$AAl?$AAe?$AA?5?$AAS?$AAt?$AAe?$AAp?$AA?5?$AA1?$AA?$AA@ 100194c0     commdevice.obj
 0002:000024f0       ??_C@_1HM@PICDBDBB@?$AAW?$AAM?$AAP?$AA?$CF?$AAd?$AA?5?$AAI?$AAo?$AAC?$AAo?$AAn?$AAt?$AAr?$AAo?$AAl?$AA?5?$AAd?$AAw?$AAC?$AAo?$AAd?$AAe?$AA?5?$AA?$DN?$AA?5?$AA0?$AAx?$AA?$CF?$AAx?$AA?5?$AAs?$AAt@ 100194f0     commdevice.obj
 0002:00002570       ??_C@_1HA@KPKCJCDJ@?$AAW?$AAM?$AAP?$AA?$CF?$AAd?$AA?5?$AAd?$AAe?$AAt?$AAe?$AAc?$AAt?$AAs?$AA?5?$AAD?$AAC?$AAD?$AA?5?$AAd?$AAr?$AAo?$AAp?$AA?4?$AA?5?$AAE?$AAx?$AAp?$AAe?$AAc?$AAt?$AA?5?$AAu@ 10019570     commdevice.obj
 0002:000025e0       ??_C@_1EM@DLKONMLD@?$AAW?$AAM?$AAP?$AA?$CF?$AAd?$AA?5?$AAc?$AAa?$AAl?$AAl?$AAs?$AA?5?$AAC?$AAl?$AAo?$AAs?$AAe?$AA?5?$AA?$CI?$AAF?$AAA?$AAL?$AAS?$AAE?$AA?$CJ?$AA?5?$AAf?$AAr?$AAo?$AAm?$AA?5?$AAi@ 100195e0     commdevice.obj
 0002:00002630       ??_C@_1EK@CGKJMGOP@?$AAW?$AAM?$AAP?$AA?$CF?$AAd?$AA?5?$AAI?$AAO?$AAC?$AAT?$AAL?$AA?5?$AAf?$AAa?$AAi?$AAl?$AA?5?$AAb?$AAc?$AAo?$AAs?$AA?5?$AAi?$AAn?$AAv?$AAa?$AAl?$AAi?$AAd?$AA?5?$AAh?$AAa@ 10019630     commdevice.obj
 0002:00002680       ??_C@_1FC@MCHMGPFN@?$AAW?$AAM?$AAP?$AA?$CF?$AAd?$AA?5?$AAC?$AAa?$AAl?$AAl?$AA?5?$AAC?$AAa?$AAr?$AAd?$AAR?$AAe?$AAm?$AAo?$AAv?$AAe?$AAd?$AAN?$AAo?$AAt?$AAi?$AAf?$AAy?$AA?5?$AAf?$AAr?$AAo@ 10019680     commdevice.obj
 0002:000026d8       ??_C@_1JK@FBCDAJKF@?$AAW?$AAM?$AAP?$AA?$CF?$AAd?$AA?5?$AAI?$AAo?$AAC?$AAo?$AAn?$AAt?$AAr?$AAo?$AAl?$AA?5?$AAd?$AAw?$AAC?$AAo?$AAd?$AAe?$AA?5?$AA?$DN?$AA?5?$AA0?$AAx?$AA?$CF?$AAx?$AA?0?$AA?5?$AAr@ 100196d8     commdevice.obj
 0002:00002778       ??_C@_1GE@IIFHLNLJ@?$AAW?$AAM?$AAP?$AA?$CF?$AAd?$AA?5?$AAI?$AAo?$AAC?$AAo?$AAn?$AAt?$AAr?$AAo?$AAl?$AA?5?$AAd?$AAw?$AAC?$AAo?$AAd?$AAe?$AA?5?$AA?$DN?$AA?5?$AA0?$AAx?$AA?$CF?$AAx?$AA?5?$AAs?$AAt@ 10019778     commdevice.obj
 0002:000027dc       ??_C@_1CO@INPDBHCE@?$AAW?$AAM?$AAP?$AA?$CF?$AAd?$AA?5?$AAI?$AAo?$AAC?$AAo?$AAn?$AAt?$AAr?$AAo?$AAl?$AA?5?$AAs?$AAt?$AAe?$AAp?$AA?5?$AA2?$AA?$AA@ 100197dc     commdevice.obj
 0002:0000280c       ??_C@_0BG@FJIADCGC@CommDevice?3?3IoControl?$AA@ 1001980c     commdevice.obj
 0002:00002824       ??_C@_1CO@JPEGLIMK@?$AAW?$AAM?$AAP?$AA?$CF?$AAd?$AA?5?$AAI?$AAo?$AAC?$AAo?$AAn?$AAt?$AAr?$AAo?$AAl?$AA?5?$AAs?$AAt?$AAe?$AAp?$AA?5?$AA1?$AA?$AA@ 10019824     commdevice.obj
 0002:00002888       ??_C@_1EA@FDCHOEII@?$AAU?$AAp?$AAp?$AAe?$AAr?$AA?5?$AAl?$AAa?$AAy?$AAe?$AAr?$AA?5?$AAc?$AAa?$AAl?$AAl?$AAs?$AA?5?$AAW?$AAM?$AAP?$AA_?$AAC?$AAl?$AAo?$AAs?$AAe?$AA?3?$AA?5?$AA?$AN?$AA?6?$AA?$AA@ 10019888     commentry.obj
 0002:000028c8       ??_7CtlService@@6B@        100198c8     CtlService.obj
 0002:000028d0       ??_C@_1JO@LOAJJPBB@?$AAS?$AAW?$AA?5?$AAG?$AAo?$AAb?$AAi?$AA?3?$AA?5?$AAF?$AAa?$AAi?$AAl?$AAe?$AAd?$AA?5?$AAt?$AAo?$AA?5?$AAs?$AAe?$AAn?$AAd?$AA?5?$AAo?$AAu?$AAt?$AA?5?$AAd?$AAa?$AAt?$AAa@ 100198d0     CtlService.obj
 0002:00002970       ??_C@_1KG@IIJHHHIP@?$AAS?$AAW?$AA?5?$AAG?$AAo?$AAb?$AAi?$AA?3?$AA?5?$AAG?$AAe?$AAt?$AA?5?$AAs?$AAy?$AAn?$AAc?$AAh?$AAr?$AAo?$AAn?$AAo?$AAu?$AAs?$AA?5?$AAt?$AAr?$AAa?$AAn?$AAs?$AAa?$AAc@ 10019970     CtlService.obj
 0002:00002a18       ??_C@_1LE@LIKDKBKH@?$AAS?$AAW?$AA?5?$AAG?$AAo?$AAb?$AAi?$AA?3?$AA?5?$AAW?$AAa?$AAi?$AAt?$AA?5?$AAf?$AAo?$AAr?$AA?5?$AAs?$AAy?$AAn?$AAc?$AAh?$AAr?$AAo?$AAn?$AAo?$AAu?$AAs?$AA?5?$AAt?$AAr@ 10019a18     CtlService.obj
 0002:00002ad0       ??_C@_1KM@LOKPGGJG@?$AAS?$AAW?$AA?5?$AAG?$AAo?$AAb?$AAi?$AA?3?$AA?5?$AAW?$AAa?$AAi?$AAt?$AA?5?$AAf?$AAo?$AAr?$AA?5?$AAs?$AAy?$AAn?$AAc?$AAh?$AAr?$AAo?$AAn?$AAo?$AAu?$AAs?$AA?5?$AAt?$AAr@ 10019ad0     CtlService.obj
 0002:00002b80       ??_C@_1IG@INBLMGLN@?$AAS?$AAW?$AA?5?$AAG?$AAo?$AAb?$AAi?$AA?3?$AA?5?$AAW?$AAa?$AAi?$AAt?$AA?5?$AAf?$AAo?$AAr?$AA?5?$AAs?$AAy?$AAn?$AAc?$AAh?$AAr?$AAo?$AAn?$AAo?$AAu?$AAs?$AA?5?$AAt?$AAr@ 10019b80     CtlService.obj
 0002:00002c08       ??_7DmsService@@6B@        10019c08     DmsService.obj
 0002:00002c0c       ??_C@_1DC@BJECNHMD@?$AAL?$AAo?$AAg?$AAF?$AAi?$AAl?$AAe?$AA?5?$AA?$DN?$AA?5?$AA?$CF?$AAs?$AA?5?$AAn?$AAo?$AAt?$AA?5?$AAo?$AAp?$AAe?$AAn?$AAn?$AAe?$AAd?$AA?$AA@ 10019c0c     PPP4pcap.obj
 0002:00002c40       ??_C@_1CC@MPMOLEGG@?$AAS?$AAS?$AA_?$AAL?$AAo?$AAg?$AAP?$AAo?$AAr?$AAt?$AA?$CF?$AAd?$AA?4?$AAb?$AAi?$AAn?$AA?$AA@ 10019c40     PPP4pcap.obj
 0002:00002c68       ??_C@_1FO@NNBIDDD@?$AAS?$AAW?$AA?5?$AAG?$AAo?$AAb?$AAi?$AA?3?$AA?5?$AAS?$AAe?$AAr?$AAv?$AAi?$AAc?$AAe?$AA?5?$AAt?$AAy?$AAp?$AAe?$AA?3?$AA?5?$AA0?$AAx?$AA?$CF?$AAx?$AA?0?$AA?5?$AAV?$AAe?$AAr@ 10019c68     qmi.obj
 0002:00002cc8       ??_C@_1O@MMGGCPIE@?$AA0?$AAx?$AA?$CF?$AA0?$AA2?$AAX?$AA?$AA@ 10019cc8     qmi.obj
 0002:00002cd8       ??_C@_1M@NDGNLFMH@?$AA?$CF?$AAd?$AA?4?$AA?$CF?$AAd?$AA?$AA@ 10019cd8     qmi.obj
 0002:00002ce4       ??_C@_1O@GMFEIALK@?$AA0?$AAx?$AA?$CF?$AA0?$AA2?$AAx?$AA?$AA@ 10019ce4     qmi.obj
 0002:00002cf4       ??_C@_1CG@FJLIKHGJ@?$AAS?$AAW?$AAG?$AAo?$AAb?$AAi?$AAQ?$AAM?$AAI?$AA?2?$AAS?$AAe?$AAr?$AAv?$AAi?$AAc?$AAe?$AAs?$AA?$AA@ 10019cf4     qmi.obj
 0002:00002d1c       ??_C@_1DK@DFOPCCDF@?$AAS?$AAo?$AAf?$AAt?$AAw?$AAa?$AAr?$AAe?$AA?2?$AAS?$AAi?$AAe?$AAr?$AAr?$AAa?$AA?5?$AAW?$AAi?$AAr?$AAe?$AAl?$AAe?$AAs?$AAs?$AA?5?$AAI?$AAn?$AAc?$AA?$AA@ 10019d1c     qmi.obj
 0002:00002d58       ??_C@_1M@DFKENGJN@?$AA?$CF?$AAs?$AA?2?$AA?$CF?$AAs?$AA?$AA@ 10019d58     qmi.obj
 0002:00002d68       ??_C@_1GI@LMEIIMCM@?$AAS?$AAW?$AA?5?$AAG?$AAo?$AAb?$AAi?$AA?3?$AA?5?$AAF?$AAa?$AAi?$AAl?$AAe?$AAd?$AA?5?$AAt?$AAo?$AA?5?$AAg?$AAe?$AAt?$AA?5?$AAQ?$AAM?$AAI?$AA?5?$AAv?$AAe?$AAr?$AAs?$AAi@ 10019d68     qmi.obj
 0002:00002dd0       ??_C@_1IO@PIFFEINC@?$AAS?$AAW?$AA?5?$AAG?$AAo?$AAb?$AAi?$AA?3?$AA?5?$AAF?$AAa?$AAi?$AAl?$AAe?$AAd?$AA?5?$AAt?$AAo?$AA?5?$AAg?$AAe?$AAt?$AA?5?$AAa?$AA?5?$AAf?$AAr?$AAe?$AAe?$AA?5?$AAt?$AAr@ 10019dd0     qmi.obj
 0002:00002e60       ??_C@_1KG@OFBGKIIM@?$AAS?$AAW?$AA?5?$AAG?$AAo?$AAb?$AAi?$AA?5?$AA?9?$AA?5?$AAG?$AAe?$AAt?$AAC?$AAl?$AAi?$AAe?$AAn?$AAt?$AAI?$AAD?$AA?3?$AA?5?$AAF?$AAa?$AAi?$AAl?$AAe?$AAd?$AA?5?$AAt?$AAo@ 10019e60     qmi.obj
 0002:00002f08       ??_C@_1HA@FFOICHGM@?$AAS?$AAW?$AA?5?$AAG?$AAo?$AAb?$AAi?$AA?5?$AA?9?$AA?5?$AAR?$AAe?$AAl?$AAe?$AAa?$AAs?$AAe?$AAC?$AAl?$AAi?$AAe?$AAn?$AAt?$AAI?$AAD?$AA?5?$AA?$CF?$AAd?$AA?0?$AA?5?$AAp?$AAr@ 10019f08     qmi.obj
 0002:00002f78       ??_C@_1HA@ENOJKJFH@?$AAS?$AAW?$AA?5?$AAG?$AAo?$AAb?$AAi?$AA?5?$AA?9?$AA?5?$AAR?$AAe?$AAl?$AAe?$AAa?$AAs?$AAe?$AAC?$AAl?$AAi?$AAe?$AAn?$AAt?$AAI?$AAD?$AA?5?$AA?$CF?$AAd?$AA?3?$AA?5?$AAF?$AAa@ 10019f78     qmi.obj
 0002:00002fe8       ??_C@_1HM@HGMENFLC@?$AAS?$AAW?$AA?5?$AAG?$AAo?$AAb?$AAi?$AA?5?$AA?9?$AA?5?$AAD?$AAm?$AAs?$AAG?$AAe?$AAt?$AAD?$AAe?$AAv?$AAi?$AAc?$AAe?$AAM?$AAa?$AAn?$AAu?$AAf?$AAa?$AAc?$AAt?$AAu?$AAr@ 10019fe8     qmi.obj
 0002:00003068       ??_C@_1HA@CAHENCKM@?$AAS?$AAW?$AA?5?$AAG?$AAo?$AAb?$AAi?$AA?5?$AA?9?$AA?5?$AAD?$AAm?$AAs?$AAG?$AAe?$AAt?$AAD?$AAe?$AAv?$AAi?$AAc?$AAe?$AAM?$AAs?$AAi?$AAs?$AAd?$AAn?$AA?3?$AA?5?$AAF?$AAa@ 1001a068     qmi.obj
 0002:000030d8       ??_C@_1FI@HHNAEICA@?$AAS?$AAW?$AA?5?$AAG?$AAo?$AAb?$AAi?$AA?5?$AA?9?$AA?5?$AAW?$AAd?$AAs?$AAS?$AAe?$AAt?$AAE?$AAv?$AAe?$AAn?$AAt?$AAR?$AAe?$AAp?$AAo?$AAr?$AAt?$AAA?$AAs?$AAy?$AAn?$AAc@ 1001a0d8     qmi.obj
 0002:00003130       ??_C@_1FM@JGCKCLBE@?$AAS?$AAW?$AA?5?$AAG?$AAo?$AAb?$AAi?$AA?5?$AA?9?$AA?5?$AAW?$AAd?$AAs?$AAG?$AAe?$AAt?$AAC?$AAu?$AAr?$AAr?$AAe?$AAn?$AAt?$AAC?$AAh?$AAa?$AAn?$AAn?$AAe?$AAl?$AAR?$AAa@ 1001a130     qmi.obj
 0002:00003190       ??_C@_1IA@JMCLNLDK@?$AAS?$AAW?$AA?5?$AAG?$AAo?$AAb?$AAi?$AA?5?$AA?9?$AA?5?$AAW?$AAd?$AAs?$AAG?$AAe?$AAt?$AAC?$AAu?$AAr?$AAr?$AAe?$AAn?$AAt?$AAC?$AAh?$AAa?$AAn?$AAn?$AAe?$AAl?$AAR?$AAa@ 1001a190     qmi.obj
 0002:00003210       ??_C@_1FG@KMOMDCDF@?$AAS?$AAW?$AA?5?$AAG?$AAo?$AAb?$AAi?$AA?5?$AA?9?$AA?5?$AAC?$AAo?$AAn?$AAf?$AAi?$AAg?$AAP?$AAo?$AAw?$AAe?$AAr?$AAS?$AAa?$AAv?$AAe?$AAS?$AAe?$AAt?$AAt?$AAi?$AAn?$AAg@ 1001a210     qmi.obj
 0002:00003268       ??_C@_1HM@FPMEPOEH@?$AAS?$AAW?$AA?5?$AAG?$AAo?$AAb?$AAi?$AA?5?$AA?9?$AA?5?$AAC?$AAo?$AAn?$AAf?$AAi?$AAg?$AAP?$AAo?$AAw?$AAe?$AAr?$AAS?$AAa?$AAv?$AAe?$AAS?$AAe?$AAt?$AAt?$AAi?$AAn?$AAg@ 1001a268     qmi.obj
 0002:000032e8       ??_C@_1GK@LACCHLKJ@?$AAS?$AAW?$AA?5?$AAG?$AAo?$AAb?$AAi?$AA?5?$AA?9?$AA?5?$AAS?$AAe?$AAt?$AAP?$AAo?$AAw?$AAe?$AAr?$AAS?$AAa?$AAv?$AAe?$AAM?$AAo?$AAd?$AAe?$AA?5?$AAp?$AAr?$AAo?$AAc?$AAe@ 1001a2e8     qmi.obj
 0002:00003358       ??_C@_1GK@OHHNKGFB@?$AAS?$AAW?$AA?5?$AAG?$AAo?$AAb?$AAi?$AA?5?$AA?9?$AA?5?$AAS?$AAe?$AAt?$AAP?$AAo?$AAw?$AAe?$AAr?$AAS?$AAa?$AAv?$AAe?$AAM?$AAo?$AAd?$AAe?$AA?5?$AAF?$AAa?$AAi?$AAl?$AAe@ 1001a358     qmi.obj
 0002:000033c8       ??_C@_1EM@LPGEDGFC@?$AAS?$AAW?$AA?5?$AAG?$AAo?$AAb?$AAi?$AA?5?$AA?9?$AA?5?$AAS?$AAe?$AAt?$AAP?$AAo?$AAw?$AAe?$AAr?$AAS?$AAa?$AAv?$AAe?$AAM?$AAo?$AAd?$AAe?$AA?5?$AAs?$AAu?$AAc?$AAc?$AAe@ 1001a3c8     qmi.obj
 0002:00003418       ??_C@_1FA@HHDNHHCK@?$AAS?$AAW?$AA?5?$AAG?$AAo?$AAb?$AAi?$AA?5?$AA?9?$AA?5?$AAS?$AAe?$AAt?$AAP?$AAo?$AAw?$AAe?$AAr?$AAS?$AAa?$AAv?$AAe?$AAM?$AAo?$AAd?$AAe?$AA?5?$AAi?$AAn?$AAi?$AAt?$AA?5@ 1001a418     qmi.obj
 0002:00003468       ??_C@_1II@NDGLMOLI@?$AAF?$AAa?$AAi?$AAl?$AAe?$AAd?$AA?5?$AAt?$AAo?$AA?5?$AAc?$AAr?$AAe?$AAa?$AAt?$AAe?$AA?5?$AAe?$AAv?$AAe?$AAn?$AAt?$AAs?$AA?5?$AAf?$AAo?$AAr?$AA?5?$AAp?$AAM?$AAd?$AAd@ 1001a468     qmicom.obj
 0002:000034f0       ??_C@_1IG@FPJHLIFE@?$AAE?$AAr?$AAr?$AAo?$AAr?$AA?5?$AAa?$AAl?$AAl?$AAo?$AAc?$AAa?$AAt?$AAi?$AAn?$AAg?$AA?5?$AAm?$AAe?$AAm?$AAo?$AAr?$AAy?$AA?5?$AAf?$AAo?$AAr?$AA?5?$AAp?$AAM?$AAd?$AAd@ 1001a4f0     qmicom.obj
 0002:00003578       ??_C@_1GM@CAMBKLAF@?$AAQ?$AAM?$AAI?$AA_?$AAO?$AAp?$AAe?$AAn?$AA?3?$AA?5?$AAF?$AAa?$AAi?$AAl?$AAe?$AAd?$AA?5?$AAt?$AAo?$AA?5?$AAo?$AAp?$AAe?$AAn?$AA?5?$AAp?$AAo?$AAr?$AAt?$AA?5?$AAa?$AAs@ 1001a578     qmicom.obj
 0002:000035e8       ??_C@_1FO@KKAKCDOD@?$AAQ?$AAM?$AAI?$AA_?$AAO?$AAp?$AAe?$AAn?$AA?3?$AA?5?$AAU?$AAn?$AAr?$AAe?$AAc?$AAo?$AAg?$AAn?$AAi?$AAz?$AAe?$AAd?$AA?5?$AAQ?$AAM?$AAI?$AA?5?$AAs?$AAe?$AAr?$AAv?$AAi@ 1001a5e8     qmicom.obj
 0002:00003648       ??_C@_1HC@FNJOENON@?$AAQ?$AAM?$AAI?$AA_?$AAO?$AAp?$AAe?$AAn?$AA?0?$AA?5?$AA?$CF?$AAs?$AA?5?$AAp?$AAo?$AAr?$AAt?$AA?5?$AAw?$AAa?$AAi?$AAt?$AAi?$AAn?$AAg?$AA?5?$AAf?$AAo?$AAr?$AA?5?$AAs?$AAy@ 1001a648     qmicom.obj
 0002:000036c0       ??_C@_1HK@BPOBJNLI@?$AAE?$AAr?$AAr?$AAo?$AAr?$AA?5?$AAa?$AAl?$AAl?$AAo?$AAc?$AAa?$AAt?$AAi?$AAn?$AAg?$AA?5?$AAm?$AAe?$AAm?$AAo?$AAr?$AAy?$AA?5?$AAf?$AAo?$AAr?$AA?5?$AAQ?$AAM?$AAI?$AA_@ 1001a6c0     qmicom.obj
 0002:00003740       ??_C@_1HG@BFKPIMAG@?$AAS?$AAo?$AAr?$AAr?$AAy?$AA?$CB?$AA?5?$AAn?$AAo?$AA?5?$AAm?$AAo?$AAr?$AAe?$AA?5?$AAU?$AAN?$AAA?$AAT?$AAT?$AAE?$AAN?$AAD?$AAE?$AAD?$AA?5?$AAm?$AAo?$AAd?$AAe?$AA?5?$AAc@ 1001a740     qmicom.obj
 0002:000037b8       ??_C@_1HM@HNDHCJBC@?$AAQ?$AAM?$AAI?$AA_?$AAO?$AAp?$AAe?$AAn?$AA?3?$AA?5?$AAg?$AAo?$AAt?$AA?5?$AAc?$AAl?$AAi?$AAe?$AAn?$AAt?$AAI?$AAD?$AA?5?$AA?$CF?$AAd?$AA?5?$AAa?$AAf?$AAt?$AAe?$AAr?$AA?5@ 1001a7b8     qmicom.obj
 0002:00003834       ??_C@_1BI@PBIEBGHK@?$AAQ?$AAM?$AAI?$AA_?$AAO?$AAp?$AAe?$AAn?$AA?5?$AA?$CF?$AAs?$AA?$AA@ 1001a834     qmicom.obj
 0002:00003850       ??_C@_1IM@PEEMPOKF@?$AAQ?$AAM?$AAI?$AA_?$AAO?$AAp?$AAe?$AAn?$AA?3?$AA?5?$AAF?$AAa?$AAi?$AAl?$AAe?$AAd?$AA?5?$AAt?$AAo?$AA?5?$AAg?$AAe?$AAt?$AA?5?$AAc?$AAl?$AAi?$AAe?$AAn?$AAt?$AA?5?$AAI@ 1001a850     qmicom.obj
 0002:000038e0       ??_C@_1IE@CLMEKOCF@?$AAQ?$AAM?$AAI?$AA_?$AAO?$AAp?$AAe?$AAn?$AA?3?$AA?5?$AAD?$AAe?$AAv?$AAi?$AAc?$AAe?$AA?5?$AAr?$AAe?$AAm?$AAo?$AAv?$AAe?$AAd?$AA?5?$AAw?$AAh?$AAe?$AAn?$AA?5?$AAg?$AAe@ 1001a8e0     qmicom.obj
 0002:00003968       ??_C@_1GC@DHNEGINP@?$AAS?$AAW?$AA?5?$AAG?$AAo?$AAb?$AAi?$AA?3?$AA?5?$AAQ?$AAM?$AAI?$AA?5?$AAs?$AAe?$AAr?$AAv?$AAi?$AAc?$AAe?$AA?5?$AAt?$AAy?$AAp?$AAe?$AA?5?$AA?$CF?$AAd?$AA?5?$AAi?$AAs?$AA?5@ 1001a968     qmicom.obj
 0002:000039d0       ??_C@_1EC@BIODLAFP@?$AAQ?$AAM?$AAI?$AA_?$AAC?$AAl?$AAo?$AAs?$AAe?$AA?3?$AA?5?$AAI?$AAn?$AAv?$AAa?$AAl?$AAi?$AAd?$AA?5?$AAo?$AAp?$AAe?$AAn?$AA?5?$AAc?$AAo?$AAu?$AAn?$AAt?$AA?4?$AA?$AN?$AA?6@ 1001a9d0     qmicom.obj
 0002:00003a18       ??_C@_1EE@NKNJHOIB@?$AAQ?$AAM?$AAI?$AA_?$AAC?$AAl?$AAo?$AAs?$AAe?$AA?3?$AA?5?$AAI?$AAn?$AAv?$AAa?$AAl?$AAi?$AAd?$AA?5?$AAo?$AAp?$AAe?$AAn?$AA?5?$AAh?$AAa?$AAn?$AAd?$AAl?$AAe?$AA?4?$AA?$AN@ 1001aa18     qmicom.obj
 0002:00003a60       ??_C@_1II@PDJGBMHL@?$AAQ?$AAM?$AAI?$AA_?$AAR?$AAe?$AAa?$AAd?$AA?3?$AA?5?$AAT?$AAr?$AAy?$AAi?$AAn?$AAg?$AA?5?$AAt?$AAo?$AA?5?$AAr?$AAe?$AAa?$AAd?$AA?5?$AAw?$AAh?$AAe?$AAn?$AA?5?$AAd?$AAe@ 1001aa60     qmicom.obj
 0002:00003ae8       ??_C@_1CE@FHDPHIOB@?$AAS?$AAw?$AAi?$AAG?$AAo?$AAb?$AAi?$AA?5?$AAQ?$AAM?$AAI?$AA_?$AAR?$AAe?$AAa?$AAd?$AA?3?$AA?$AA@ 1001aae8     qmicom.obj
 0002:00003b10       ??_C@_1EE@KMIIDKMA@?$AA?$CF?$AAs?$AA?5?$AAF?$AAa?$AAi?$AAl?$AAe?$AAd?$AA?5?$AAt?$AAo?$AA?5?$AAr?$AAe?$AAa?$AAd?$AA?5?$AAt?$AAh?$AAe?$AA?5?$AAQ?$AAM?$AAI?$AA?5?$AAd?$AAa?$AAt?$AAa?$AA?4?$AA?$AN@ 1001ab10     qmicom.obj
 0002:00003b58       ??_C@_1IM@KFBGGOIA@?$AAQ?$AAM?$AAI?$AA_?$AAW?$AAr?$AAi?$AAt?$AAe?$AA?3?$AA?5?$AAT?$AAr?$AAy?$AAi?$AAn?$AAg?$AA?5?$AAt?$AAo?$AA?5?$AAw?$AAr?$AAi?$AAt?$AAe?$AA?5?$AAw?$AAh?$AAe?$AAn?$AA?5@ 1001ab58     qmicom.obj
 0002:00003be8       ??_C@_1KG@CDJJLKD@?$AAQ?$AAM?$AAI?$AA_?$AAW?$AAr?$AAi?$AAt?$AAe?$AA?5?$AA?$CF?$AAs?$AA?5?$AAn?$AAo?$AAt?$AA?5?$AAa?$AAl?$AAl?$AAo?$AAw?$AAe?$AAd?$AA?5?$AAw?$AAh?$AAi?$AAl?$AAe?$AA?5?$AAg@ 1001abe8     qmicom.obj
 0002:00003c90       ??_C@_1FE@BKHCEKGC@?$AAE?$AAv?$AAa?$AAl?$AAu?$AAa?$AAt?$AAe?$AAE?$AAv?$AAe?$AAn?$AAt?$AAF?$AAl?$AAa?$AAg?$AA?5?$AAj?$AAu?$AAs?$AAt?$AA?5?$AAa?$AAv?$AAo?$AAi?$AAd?$AAs?$AA?5?$AAa?$AA?5@ 1001ac90     qmicom.obj
 0002:00003ce8       ??_C@_1IK@CNBBLOMH@?$AAD?$AAC?$AAD?$AA?5?$AAs?$AAt?$AAa?$AAt?$AAe?$AA?5?$AAi?$AAs?$AA?5?$AA?$CF?$AAx?$AA?5?$AA?$FL?$AA0?$AA?5?$AA?$DN?$AA?5?$AAC?$AAL?$AAR?$AA?0?$AA?5?$AA1?$AA?5?$AA?$DN?$AA?5?$AAS?$AAE@ 1001ace8     qmicom.obj
 0002:00003d78       ??_C@_1GC@GFNBODFJ@?$AAF?$AAa?$AAi?$AAl?$AA?5?$AAt?$AAo?$AA?5?$AAw?$AAr?$AAi?$AAt?$AAe?$AA?5?$AA?$CF?$AAd?$AA?5?$AAb?$AAy?$AAt?$AAe?$AAs?$AA?5?$AAt?$AAo?$AA?5?$AAI?$AAn?$AAB?$AAu?$AAf?$AAf@ 1001ad78     qmicom.obj
 0002:00003ddc       ??_C@_1CK@EJMDEGNB@?$AA?5?$AAI?$AAn?$AAv?$AAa?$AAl?$AAi?$AAd?$AA?5?$AAp?$AAa?$AAr?$AAa?$AAm?$AAe?$AAt?$AAe?$AAr?$AA?$AN?$AA?6?$AA?$AA@ 1001addc     qmicom.obj
 0002:00003e08       ??_C@_1FE@DCNACOPO@?$AA?5?$AAC?$AAO?$AAM?$AA_?$AAI?$AAO?$AAC?$AAo?$AAn?$AAt?$AAr?$AAo?$AAl?$AA?5?$AA?9?$AA?5?$AAE?$AAr?$AAr?$AAo?$AAr?$AA?5?$AAi?$AAn?$AA?5?$AAW?$AAa?$AAi?$AAt?$AAC?$AAo@ 1001ae08     qmicom.obj
 0002:00003e60       ??_C@_1HK@OMNBALPN@?$AA?5?$AAI?$AAO?$AAC?$AAT?$AAL?$AA_?$AAS?$AAE?$AAR?$AAI?$AAA?$AAL?$AA_?$AAS?$AAE?$AAT?$AA_?$AAD?$AAT?$AAR?$AA?5?$AAw?$AAh?$AAi?$AAl?$AAe?$AA?5?$AAD?$AAT?$AAR?$AA_@ 1001ae60     qmicom.obj
 0002:00003ee0       ??_C@_1HI@DKOIOKPN@?$AA?5?$AAI?$AAO?$AAC?$AAT?$AAL?$AA_?$AAS?$AAE?$AAR?$AAI?$AAA?$AAL?$AA_?$AAC?$AAL?$AAR?$AA_?$AAD?$AAT?$AAR?$AA?5?$AAw?$AAi?$AAt?$AAh?$AA?5?$AAD?$AAT?$AAR?$AA_?$AAC@ 1001aee0     qmicom.obj
 0002:00003f58       ??_C@_1GK@NIHNBMCE@?$AA?$CF?$AAs?$AA?5?$AAI?$AAO?$AAC?$AAT?$AAL?$AA_?$AAS?$AAE?$AAR?$AAI?$AAA?$AAL?$AA_?$AAS?$AAE?$AAT?$AA_?$AAR?$AAT?$AAS?$AA?5?$AAw?$AAi?$AAt?$AAh?$AA?5?$AAR?$AAT?$AAS@ 1001af58     qmicom.obj
 0002:00003fc4       ??_C@_1DE@BLPJGJDB@?$AA?$CF?$AAs?$AA?5?$AAI?$AAO?$AAC?$AAT?$AAL?$AA_?$AAS?$AAE?$AAR?$AAI?$AAA?$AAL?$AA_?$AAS?$AAE?$AAT?$AA_?$AAR?$AAT?$AAS?$AA?$AN?$AA?6?$AA?$AA@ 1001afc4     qmicom.obj
 0002:00003ff8       ??_C@_1GK@KFCIHAFE@?$AA?$CF?$AAs?$AA?5?$AAI?$AAO?$AAC?$AAT?$AAL?$AA_?$AAS?$AAE?$AAR?$AAI?$AAA?$AAL?$AA_?$AAC?$AAL?$AAR?$AA_?$AAR?$AAT?$AAS?$AA?5?$AAw?$AAi?$AAt?$AAh?$AA?5?$AAR?$AAT?$AAS@ 1001aff8     qmicom.obj
 0002:00004064       ??_C@_1DE@FAKNLDBN@?$AA?$CF?$AAs?$AA?5?$AAI?$AAO?$AAC?$AAT?$AAL?$AA_?$AAS?$AAE?$AAR?$AAI?$AAA?$AAL?$AA_?$AAC?$AAL?$AAR?$AA_?$AAR?$AAT?$AAS?$AA?$AN?$AA?6?$AA?$AA@ 1001b064     qmicom.obj
 0002:00004098       ??_C@_1IM@DPHLGJPD@?$AAS?$AAW?$AA?5?$AAG?$AAo?$AAb?$AAi?$AA?5?$AA?9?$AA?5?$AAP?$AAr?$AAo?$AAc?$AAe?$AAs?$AAs?$AAC?$AAl?$AAi?$AAe?$AAn?$AAt?$AAM?$AAs?$AAg?$AA?3?$AA?5?$AAF?$AAa?$AAi?$AAl@ 1001b098     qmicom.obj
 0002:00004128       ??_C@_1GO@IOELMKHO@?$AAS?$AAw?$AAi?$AAG?$AAo?$AAb?$AAi?$AA?5?$AAr?$AAe?$AAt?$AAu?$AAr?$AAn?$AAs?$AA?5?$AAD?$AAx?$AA?$DN?$AA0?$AAx?$AA?$CF?$AAx?$AA?5?$AAf?$AAo?$AAr?$AA?5?$AAI?$AAO?$AAC?$AAT@ 1001b128     qmicom.obj
 0002:00004198       ??_C@_1EM@MMPOMNKA@?$AAI?$AAO?$AAC?$AAT?$AAL?$AA_?$AAP?$AAO?$AAW?$AAE?$AAR?$AA_?$AAS?$AAE?$AAT?$AA?5?$AAf?$AAa?$AAi?$AAl?$AAe?$AAd?$AA?5?$AAb?$AAc?$AAo?$AAs?$AA?5?$AA?$CF?$AAd?$AA?5?$AA?$DM@ 1001b198     qmicom.obj
 0002:000041e8       ??_C@_1PI@KBHPKFMG@?$AAS?$AAW?$AAI?$AAU?$AAS?$AAB?$AA?5?$AAH?$AAa?$AAn?$AAd?$AAl?$AAe?$AAd?$AA?5?$AAI?$AAO?$AAC?$AAT?$AAR?$AAL?$AA_?$AAP?$AAO?$AAW?$AAE?$AAR?$AA_?$AAS?$AAE?$AAT?$AA?5@ 1001b1e8     qmicom.obj
 0002:000042e0       ??_C@_1CM@FGAHCHKM@?$AAU?$AAn?$AAh?$AAa?$AAn?$AAd?$AAl?$AAe?$AAd?$AA?5?$AAD?$AA?$CF?$AAd?$AA?5?$AAs?$AAt?$AAa?$AAt?$AAe?$AA?$AN?$AA?6?$AA?$AA@ 1001b2e0     qmicom.obj
 0002:00004310       ??_C@_1IK@JDDBBLC@?$AAF?$AAa?$AAi?$AAl?$AA?5?$AAU?$AAs?$AAb?$AAS?$AAe?$AAt?$AAH?$AAo?$AAs?$AAt?$AAS?$AAl?$AAe?$AAe?$AAp?$AAP?$AAo?$AAw?$AAe?$AAr?$AAS?$AAt?$AAa?$AAt?$AAe?$AA?5?$AA?$CI@ 1001b310     qmicom.obj
 0002:000043a0       ??_C@_1JA@KKKNDLFK@?$AAF?$AAa?$AAi?$AAl?$AA?5?$AAU?$AAs?$AAb?$AAS?$AAe?$AAt?$AAH?$AAo?$AAs?$AAt?$AAS?$AAl?$AAe?$AAe?$AAp?$AAP?$AAo?$AAw?$AAe?$AAr?$AAS?$AAt?$AAa?$AAt?$AAe?$AA?5?$AA?$CI@ 1001b3a0     qmicom.obj
 0002:00004430       ??_7RilOutContextPool@@6B@ 1001b430     RilOutContextPool.obj
 0002:00004438       ??_C@_1EG@KMMAEDFC@?$AAR?$AAi?$AAl?$AAO?$AAu?$AAt?$AAC?$AAo?$AAn?$AAt?$AAe?$AAx?$AAt?$AAP?$AAo?$AAo?$AAl?$AA?3?$AA?3?$AAA?$AAl?$AAl?$AAo?$AAc?$AAa?$AAt?$AAe?$AA?5?$AAN?$AAU?$AAL?$AAL@ 1001b438     RilOutContextPool.obj
 0002:00004480       ??_C@_1EC@OAFALGDM@?$AAR?$AAi?$AAl?$AAO?$AAu?$AAt?$AAC?$AAo?$AAn?$AAt?$AAe?$AAx?$AAt?$AAP?$AAo?$AAo?$AAl?$AA?5?$AAs?$AAe?$AAn?$AAd?$AAi?$AAn?$AAg?$AA?5?$AAX?$AAO?$AAF?$AAF?$AA?$AN?$AA?6@ 1001b480     RilOutContextPool.obj
 0002:000044c8       ??_C@_1EI@JBOEOOGL@?$AAR?$AAi?$AAl?$AAO?$AAu?$AAt?$AAC?$AAo?$AAn?$AAt?$AAe?$AAx?$AAt?$AAP?$AAo?$AAo?$AAl?$AA?5?$AAm?$AA_?$AAI?$AAn?$AAU?$AAs?$AAe?$AAC?$AAo?$AAu?$AAn?$AAt?$AA?5?$AA?$CF@ 1001b4c8     RilOutContextPool.obj
 0002:00004510       ??_C@_1EA@OLFAODHL@?$AAR?$AAi?$AAl?$AAO?$AAu?$AAt?$AAC?$AAo?$AAn?$AAt?$AAe?$AAx?$AAt?$AAP?$AAo?$AAo?$AAl?$AA?5?$AAs?$AAe?$AAn?$AAd?$AAi?$AAn?$AAg?$AA?5?$AAX?$AAO?$AAN?$AA?$AN?$AA?6?$AA?$AA@ 1001b510     RilOutContextPool.obj
 0002:00004550       ??_7RilPacketPool@@6B@     1001b550     RilPacketPool.obj
 0002:00004554       ??_C@_1DO@HLFEGICL@?$AAR?$AAi?$AAl?$AAP?$AAa?$AAc?$AAk?$AAe?$AAt?$AAP?$AAo?$AAo?$AAl?$AA?3?$AA?3?$AAA?$AAl?$AAl?$AAo?$AAc?$AAa?$AAt?$AAe?$AA?5?$AAN?$AAU?$AAL?$AAL?$AA?$AN?$AA?6?$AA?$AA@ 1001b554     RilPacketPool.obj
 0002:000045e8       ??_C@_1HM@LCPELDFK@?$AAE?$AAr?$AAr?$AAo?$AAr?$AA?5?$AAa?$AAl?$AAl?$AAo?$AAc?$AAa?$AAt?$AAi?$AAn?$AAg?$AA?5?$AAm?$AAe?$AAm?$AAo?$AAr?$AAy?$AA?5?$AAf?$AAo?$AAr?$AA?5?$AAR?$AAi?$AAl?$AAP@ 1001b5e8     swdcom.obj
 0002:00004668       ??_C@_1IE@MEFEDKHD@?$AAE?$AAr?$AAr?$AAo?$AAr?$AA?5?$AAa?$AAl?$AAl?$AAo?$AAc?$AAa?$AAt?$AAi?$AAn?$AAg?$AA?5?$AAm?$AAe?$AAm?$AAo?$AAr?$AAy?$AA?5?$AAf?$AAo?$AAr?$AA?5?$AAR?$AAi?$AAl?$AAO@ 1001b668     swdcom.obj
 0002:000046f0       ??_C@_1GI@NPHLCOLO@?$AAE?$AAr?$AAr?$AAo?$AAr?$AA?5?$AAa?$AAl?$AAl?$AAo?$AAc?$AAa?$AAt?$AAi?$AAn?$AAg?$AA?5?$AAm?$AAe?$AAm?$AAo?$AAr?$AAy?$AA?5?$AAf?$AAo?$AAr?$AA?5?$AAp?$AAM?$AAd?$AAd@ 1001b6f0     swdcom.obj
 0002:00004758       ??_C@_1HK@MHKDNMGL@?$AAE?$AAr?$AAr?$AAo?$AAr?$AA?5?$AAa?$AAl?$AAl?$AAo?$AAc?$AAa?$AAt?$AAi?$AAn?$AAg?$AA?5?$AAm?$AAe?$AAm?$AAo?$AAr?$AAy?$AA?5?$AAf?$AAo?$AAr?$AA?5?$AAS?$AAW?$AAD?$AA_@ 1001b758     swdcom.obj
 0002:000047d4       ??_C@_1BI@KAAKHJBJ@?$AAS?$AAW?$AAD?$AA_?$AAO?$AAp?$AAe?$AAn?$AA?5?$AA?$CF?$AAs?$AA?$AA@ 1001b7d4     swdcom.obj
 0002:000047f0       ??_C@_1GM@JIDOFNFF@?$AAS?$AAW?$AAD?$AA_?$AAO?$AAp?$AAe?$AAn?$AA?3?$AA?5?$AAF?$AAa?$AAi?$AAl?$AAe?$AAd?$AA?5?$AAt?$AAo?$AA?5?$AAo?$AAp?$AAe?$AAn?$AA?5?$AAp?$AAo?$AAr?$AAt?$AA?5?$AAa?$AAs@ 1001b7f0     swdcom.obj
 0002:00004860       ??_C@_1EE@JIOOFKJK@?$AAS?$AAW?$AAD?$AA_?$AAC?$AAl?$AAo?$AAs?$AAe?$AA?3?$AA?5?$AAI?$AAn?$AAv?$AAa?$AAl?$AAi?$AAd?$AA?5?$AAo?$AAp?$AAe?$AAn?$AA?5?$AAh?$AAa?$AAn?$AAd?$AAl?$AAe?$AA?4?$AA?$AN@ 1001b860     swdcom.obj
 0002:000048a8       ??_C@_1FC@HCCKIHDM@?$AAS?$AAW?$AAD?$AA_?$AAI?$AAO?$AAC?$AAo?$AAn?$AAt?$AAr?$AAo?$AAl?$AA?5?$AAI?$AAO?$AAC?$AAT?$AAL?$AA_?$AAR?$AAI?$AAL?$AAN?$AAD?$AAI?$AAS?$AA_?$AAG?$AAE?$AAT?$AA_@ 1001b8a8     swdcom.obj
 0002:00004900       ??_C@_1GA@MKABIPNJ@?$AAS?$AAW?$AAD?$AA_?$AAI?$AAO?$AAC?$AAo?$AAn?$AAt?$AAr?$AAo?$AAl?$AA?5?$AAp?$AAf?$AAn?$AAN?$AAd?$AAi?$AAs?$AAR?$AAe?$AAc?$AAe?$AAi?$AAv?$AAe?$AAP?$AAa?$AAc?$AAk@ 1001b900     swdcom.obj
 0002:00004960       ??_C@_1FC@JHFGCBGG@?$AAS?$AAW?$AAD?$AA_?$AAI?$AAO?$AAC?$AAo?$AAn?$AAt?$AAr?$AAo?$AAl?$AA?5?$AAp?$AAf?$AAn?$AAN?$AAd?$AAi?$AAs?$AAS?$AAe?$AAn?$AAd?$AAP?$AAa?$AAc?$AAk?$AAe?$AAt?$AA?3@ 1001b960     swdcom.obj
 0002:000049b8       ??_C@_1FI@MNAOJMOH@?$AAS?$AAW?$AAD?$AA_?$AAI?$AAO?$AAC?$AAo?$AAn?$AAt?$AAr?$AAo?$AAl?$AA?5?$AAI?$AAO?$AAC?$AAT?$AAL?$AA_?$AAR?$AAI?$AAL?$AAN?$AAD?$AAI?$AAS?$AA_?$AAS?$AAE?$AAT?$AA_@ 1001b9b8     swdcom.obj
 0002:00004a10       ??_C@_1GA@NFDHHKAL@?$AAS?$AAW?$AAD?$AA_?$AAI?$AAO?$AAC?$AAo?$AAn?$AAt?$AAr?$AAo?$AAl?$AA?5?$AAp?$AAf?$AAn?$AAN?$AAd?$AAi?$AAs?$AAR?$AAe?$AAc?$AAe?$AAi?$AAv?$AAi?$AAn?$AAg?$AAP?$AAa@ 1001ba10     swdcom.obj
 0002:00004a70       ??_C@_1GC@FOMGMMOB@?$AAS?$AAW?$AAD?$AA_?$AAI?$AAO?$AAC?$AAo?$AAn?$AAt?$AAr?$AAo?$AAl?$AA?5?$AAp?$AAf?$AAn?$AAN?$AAd?$AAi?$AAs?$AAT?$AAr?$AAa?$AAn?$AAs?$AAm?$AAi?$AAt?$AAC?$AAo?$AAm@ 1001ba70     swdcom.obj
 0002:00004ad8       ??_C@_1EO@MFALGIMG@?$AAS?$AAW?$AAD?$AA_?$AAI?$AAO?$AAC?$AAo?$AAn?$AAt?$AAr?$AAo?$AAl?$AA?5?$AAp?$AAf?$AAn?$AAN?$AAd?$AAi?$AAs?$AAS?$AAt?$AAa?$AAt?$AAu?$AAs?$AAC?$AAB?$AA?3?$AA?5?$AA0@ 1001bad8     swdcom.obj
 0002:00004b28       ??_C@_1FG@FLPAGBFO@?$AAS?$AAW?$AAD?$AA_?$AAI?$AAO?$AAC?$AAo?$AAn?$AAt?$AAr?$AAo?$AAl?$AA?5?$AAp?$AAR?$AAi?$AAl?$AAC?$AAa?$AAl?$AAl?$AAb?$AAa?$AAc?$AAk?$AAC?$AAo?$AAn?$AAt?$AAe?$AAx@ 1001bb28     swdcom.obj
 0002:00004b80       ??_C@_1IO@EMKPMOGM@?$AAS?$AAW?$AAD?$AA_?$AAI?$AAO?$AAC?$AAo?$AAn?$AAt?$AAr?$AAo?$AAl?$AA?3?$AA?5?$AAT?$AAr?$AAy?$AAi?$AAn?$AAg?$AA?5?$AAt?$AAo?$AA?5?$AAI?$AAO?$AAC?$AAT?$AAL?$AA?5?$AAw@ 1001bb80     swdcom.obj
 0002:00004c10       ??_C@_1HE@PJLNBCEN@?$AA?9?$AAS?$AAi?$AAe?$AAr?$AAr?$AAa?$AAW?$AAi?$AAr?$AAe?$AAl?$AAe?$AAs?$AAs?$AA?5?$AAC?$AAE?$AA?5?$AAD?$AAr?$AAi?$AAv?$AAe?$AAr?$AA?3?$AA?5?$AAD?$AAl?$AAl?$AAE?$AAx@ 1001bc10     swicom.obj
 0002:00004c84       ??_C@_17DMBMDHNL@?$AAU?$AAS?$AAB?$AA?$AA@ 1001bc84     swicom.obj
 0002:00004c8c       ??_C@_13OHNMPHJM@?$AA?$FN?$AA?$AA@ 1001bc8c     swicom.obj
 0002:00004c90       ??_C@_1LC@JLIGKPKG@?$AAd?$AAu?$AAm?$AAp?$AAB?$AAy?$AAt?$AAe?$AAs?$AAD?$AAa?$AAt?$AAa?$AA?3?$AA?3?$AA?5?$AAi?$AA?$CL?$AAj?$AA?5?$AAi?$AAs?$AA?5?$AAn?$AAo?$AAt?$AA?5?$AAl?$AAe?$AAs?$AAs?$AA?5@ 1001bc90     swicom.obj
 0002:00004d44       ??_C@_1M@OMOAGDNC@?$AA?$CF?$AA0?$AA2?$AAx?$AA?5?$AA?$AA@ 1001bd44     swicom.obj
 0002:00004d50       ??_C@_1BE@DFBIOGAO@?$AA?$DO?$AA?$DO?$AA?$CF?$AAd?$AA?$DO?$AA?$DO?$AA?5?$AA?$FL?$AA?5?$AA?$AA@ 1001bd50     swicom.obj
 0002:00004d64       ??_C@_1M@DDJDDKAP@?$AA?$CF?$AAs?$AA?5?$AA?$AN?$AA?6?$AA?$AA@ 1001bd64     swicom.obj
 0002:00004d70       ??_C@_1DC@PDNCBGBP@?$AA?$CF?$AAs?$AA?5?$AA?4?$AA?4?$AA?4?$AA?5?$AAb?$AAu?$AAt?$AA?5?$AAl?$AAe?$AAn?$AAg?$AAt?$AAh?$AA?5?$AAi?$AAs?$AA?5?$AA0?$AA?$AN?$AA?6?$AA?$AA@ 1001bd70     swicom.obj
 0002:00004da8       ??_C@_1JI@MEAHMNJ@?$AA?$AN?$AA?6?$AA?$DO?$AA?$DO?$AA?$CF?$AAd?$AA?$DO?$AA?$DO?$AA?5?$AAN?$AAo?$AAw?$AA?5?$AAd?$AAu?$AAm?$AAp?$AAi?$AAn?$AAg?$AA?5?$AAt?$AAh?$AAe?$AA?5?$AAb?$AAu?$AAf?$AAf?$AAe?$AAr?$AA?5@ 1001bda8     swicom.obj
 0002:00004e40       ??_C@_1GO@LICGMOPA@?$AA?$AN?$AA?6?$AA?$DO?$AA?$DO?$AA?$CF?$AAd?$AA?$DO?$AA?$DO?$AA?5?$AA?$CF?$AAs?$AA?$DO?$AA?$DO?$AA?$CF?$AAd?$AA?$DO?$AA?$DO?$AA?5?$AAB?$AAy?$AAt?$AAe?$AAs?$AA?$DN?$AA?$CF?$AAd?$AA?0?$AA?5?$AAU?$AAP?$AA?$DN?$AA0@ 1001be40     swicom.obj
 0002:00004eb0       ??_C@_1DK@IMJIOKDD@?$AA?2?$AAW?$AAi?$AAn?$AAd?$AAo?$AAw?$AAs?$AA?2?$AAS?$AAt?$AAa?$AAr?$AAt?$AAU?$AAp?$AA?2?$AAW?$AAe?$AAl?$AAc?$AAo?$AAm?$AAe?$AA?4?$AAl?$AAn?$AAk?$AA?$AA@ 1001beb0     swicom.obj
 0002:00004ef0       ??_C@_1II@HDHKEPCE@?$AAF?$AAa?$AAi?$AAl?$AAe?$AAd?$AA?5?$AAt?$AAo?$AA?5?$AAc?$AAr?$AAe?$AAa?$AAt?$AAe?$AA?5?$AAe?$AAv?$AAe?$AAn?$AAt?$AAs?$AA?5?$AAf?$AAo?$AAr?$AA?5?$AAp?$AAM?$AAd?$AAd@ 1001bef0     swicom.obj
 0002:00004f78       ??_C@_1IG@DNNGCDAB@?$AAE?$AAr?$AAr?$AAo?$AAr?$AA?5?$AAa?$AAl?$AAl?$AAo?$AAc?$AAa?$AAt?$AAi?$AAn?$AAg?$AA?5?$AAm?$AAe?$AAm?$AAo?$AAr?$AAy?$AA?5?$AAf?$AAo?$AAr?$AA?5?$AAp?$AAM?$AAd?$AAd@ 1001bf78     swicom.obj
 0002:00005000       ??_C@_1KK@LKNIPEOP@?$AAM?$AAo?$AAd?$AAe?$AAm?$AA?5?$AAi?$AAs?$AAs?$AAu?$AAe?$AAs?$AA?3?$AA?5?$AAS?$AAe?$AAt?$AA?5?$AAN?$AAM?$AAE?$AAA?$AA?5?$AAs?$AAt?$AAa?$AAr?$AAt?$AAs?$AA?5?$AAr?$AAe@ 1001c000     swicom.obj
 0002:000050ac       ??_C@_1BA@DONBDPBO@?$AAG?$AAp?$AAs?$AAX?$AAt?$AAr?$AAa?$AA?$AA@ 1001c0ac     swicom.obj
 0002:000050bc       ??_C@_1BC@GEDIKHKD@?$AAN?$AAM?$AAE?$AAA?$AAM?$AAa?$AAs?$AAk?$AA?$AA@ 1001c0bc     swicom.obj
 0002:000050d0       ??_C@_1BM@CAJGGJKL@?$AAN?$AAM?$AAE?$AAA?$AAR?$AAe?$AAp?$AAo?$AAr?$AAt?$AAi?$AAn?$AAg?$AA?$AA@ 1001c0d0     swicom.obj
 0002:000050ec       ??_C@_1BC@GAMECLKF@?$AAN?$AAM?$AAE?$AAA?$AAP?$AAo?$AAr?$AAt?$AA?$AA@ 1001c0ec     swicom.obj
 0002:00005100       ??_C@_1BG@DMFMOMIL@?$AAN?$AAM?$AAE?$AAA?$AAC?$AAo?$AAn?$AAf?$AAi?$AAg?$AA?$AA@ 1001c100     swicom.obj
 0002:00005118       ??_C@_1M@BIEHMKAG@?$AAR?$AAI?$AAL?$AA1?$AA?3?$AA?$AA@ 1001c118     swicom.obj
 0002:00005124       ??_C@_1BC@OHENPEDC@?$AAA?$AAc?$AAc?$AAu?$AAr?$AAa?$AAc?$AAy?$AA?$AA@ 1001c124     swicom.obj
 0002:00005138       ??_C@_1BC@KKEAFNKD@?$AAI?$AAn?$AAt?$AAe?$AAr?$AAv?$AAa?$AAl?$AA?$AA@ 1001c138     swicom.obj
 0002:0000514c       ??_C@_1BA@BKONPLFM@?$AAT?$AAi?$AAm?$AAe?$AAo?$AAu?$AAt?$AA?$AA@ 1001c14c     swicom.obj
 0002:0000515c       ??_C@_1CI@GKIMIMCM@?$AAs?$AAw?$AAi?$AAg?$AAo?$AAb?$AAi?$AA?2?$AAG?$AAP?$AAS?$AAS?$AAe?$AAt?$AAt?$AAi?$AAn?$AAg?$AAs?$AA?$AA@ 1001c15c     swicom.obj
 0002:00005184       ??_C@_1BE@JJJGIENO@?$AAO?$AAp?$AAe?$AAr?$AAa?$AAt?$AAi?$AAo?$AAn?$AA?$AA@ 1001c184     swicom.obj
 0002:00005198       ??_C@_19FCKDNDCB@?$AAN?$AAM?$AAE?$AAA?$AA?$AA@ 1001c198     swicom.obj
 0002:000051a8       ??_C@_1HC@DPLBPDII@?$AAS?$AAW?$AAI?$AA_?$AAO?$AAp?$AAe?$AAn?$AA?0?$AA?5?$AA?$CF?$AAs?$AA?5?$AAp?$AAo?$AAr?$AAt?$AA?5?$AAw?$AAa?$AAi?$AAt?$AAi?$AAn?$AAg?$AA?5?$AAf?$AAo?$AAr?$AA?5?$AAs?$AAy@ 1001c1a8     swicom.obj
 0002:0000521c       ??_C@_1BI@BGFLHPLE@?$AAS?$AAW?$AAI?$AA_?$AAO?$AAp?$AAe?$AAn?$AA?5?$AA?$CF?$AAs?$AA?$AA@ 1001c21c     swicom.obj
 0002:00005238       ??_C@_1KC@IKEALAM@?$AAM?$AAo?$AAd?$AAe?$AAm?$AA?5?$AAi?$AAs?$AAs?$AAu?$AAe?$AAs?$AA?3?$AA?5?$AAS?$AAe?$AAt?$AA?5?$AAN?$AAM?$AAE?$AAA?$AA?5?$AAS?$AAT?$AAO?$AAP?$AA?5?$AAr?$AAe?$AAt?$AAu@ 1001c238     swicom.obj
 0002:000052e0       ??_C@_1HA@OCAIFHD@?$AAS?$AAW?$AAI?$AA_?$AAW?$AAr?$AAi?$AAt?$AAe?$AA?3?$AA?5?$AAF?$AAa?$AAi?$AAl?$AAe?$AAd?$AA?5?$AAd?$AAu?$AAe?$AA?5?$AAt?$AAo?$AA?5?$AAu?$AAn?$AAe?$AAx?$AAp?$AAe?$AAc@ 1001c2e0     swicom.obj
 0002:00005350       ??_C@_15LDIKJGMG@?$AAD?$AAM?$AA?$AA@ 1001c350     swicom.obj
 0002:00005358       ??_C@_1KG@OBGDJPAO@?$AAS?$AAW?$AAI?$AA_?$AAW?$AAr?$AAi?$AAt?$AAe?$AA?5?$AA?$CF?$AAs?$AA?5?$AAn?$AAo?$AAt?$AA?5?$AAa?$AAl?$AAl?$AAo?$AAw?$AAe?$AAd?$AA?5?$AAw?$AAh?$AAi?$AAl?$AAe?$AA?5?$AAg@ 1001c358     swicom.obj
 0002:00005400       ??_C@_1CA@HHCKMMKJ@?$AA?5?$AA?5?$AA?5?$AA?5?$AA?5?$AAE?$AAV?$AA_?$AAT?$AAX?$AAE?$AAM?$AAP?$AAT?$AAY?$AA?$AA@ 1001c400     swicom.obj
 0002:00005420       ??_C@_1BO@MANALDIG@?$AA?5?$AA?5?$AA?5?$AA?5?$AA?5?$AAE?$AAV?$AA_?$AAR?$AAX?$AAF?$AAL?$AAA?$AAG?$AA?$AA@ 1001c420     swicom.obj
 0002:00005440       ??_C@_1BO@MFHENBJF@?$AA?5?$AA?5?$AA?5?$AA?5?$AA?5?$AAE?$AAV?$AA_?$AAR?$AAX?$AAC?$AAH?$AAA?$AAR?$AA?$AA@ 1001c440     swicom.obj
 0002:00005460       ??_C@_1BK@HGILCPKA@?$AA?5?$AA?5?$AA?5?$AA?5?$AA?5?$AAE?$AAV?$AA_?$AAR?$AAL?$AAS?$AAD?$AA?$AA@ 1001c460     swicom.obj
 0002:0000547c       ??_C@_1BK@JDJGJPGP@?$AA?5?$AA?5?$AA?5?$AA?5?$AA?5?$AAE?$AAV?$AA_?$AAR?$AAI?$AAN?$AAG?$AA?$AA@ 1001c47c     swicom.obj
 0002:00005498       ??_C@_1BM@CMMIMINB@?$AA?5?$AA?5?$AA?5?$AA?5?$AA?5?$AAE?$AAV?$AA_?$AAP?$AAO?$AAW?$AAE?$AAR?$AA?$AA@ 1001c498     swicom.obj
 0002:000054b4       ??_C@_1BI@GFIONDMJ@?$AA?5?$AA?5?$AA?5?$AA?5?$AA?5?$AAE?$AAV?$AA_?$AAE?$AAR?$AAR?$AA?$AA@ 1001c4b4     swicom.obj
 0002:000054cc       ??_C@_1BI@GCHIAAPC@?$AA?5?$AA?5?$AA?5?$AA?5?$AA?5?$AAE?$AAV?$AA_?$AAD?$AAS?$AAR?$AA?$AA@ 1001c4cc     swicom.obj
 0002:000054e4       ??_C@_1BI@MNAEFODG@?$AA?5?$AA?5?$AA?5?$AA?5?$AA?5?$AAE?$AAV?$AA_?$AAC?$AAT?$AAS?$AA?$AA@ 1001c4e4     swicom.obj
 0002:000054fc       ??_C@_1BM@JGKFNNLP@?$AA?5?$AA?5?$AA?5?$AA?5?$AA?5?$AAE?$AAV?$AA_?$AAB?$AAR?$AAE?$AAA?$AAK?$AA?$AA@ 1001c4fc     swicom.obj
 0002:00005518       ??_C@_1IG@FEMKGKOP@?$AAF?$AAa?$AAi?$AAl?$AA?5?$AAo?$AAn?$AA?5?$AAV?$AAs?$AAp?$AAA?$AAd?$AAd?$AAT?$AAo?$AAR?$AAe?$AAa?$AAd?$AAQ?$AAu?$AAe?$AAu?$AAe?$AA?5?$AAb?$AAc?$AAo?$AAs?$AA?5?$AAI@ 1001c518     swicom.obj
 0002:000055a0       ??_C@_1GO@KFOFNPGK@?$AAS?$AAw?$AAi?$AAC?$AAo?$AAm?$AAp?$AA?5?$AAr?$AAe?$AAt?$AAu?$AAr?$AAn?$AAs?$AA?5?$AAD?$AAx?$AA?$DN?$AA0?$AAx?$AA?$CF?$AAx?$AA?5?$AAf?$AAo?$AAr?$AA?5?$AAI?$AAO?$AAC?$AAT@ 1001c5a0     swicom.obj
 0002:00005610       ??_C@_1EE@ILJFCBIG@?$AAS?$AAW?$AA_?$AAM?$AAO?$AAD?$AAE?$AAM?$AA_?$AAS?$AAE?$AAT?$AA_?$AAD?$AAE?$AAV?$AAI?$AAC?$AAE?$AA_?$AAR?$AAE?$AAM?$AAO?$AAT?$AAE?$AA_?$AAW?$AAA?$AAK?$AAE?$AAU@ 1001c610     swiroutines.obj
 0002:00005654       ??_C@_1DI@CEJNLMNM@?$AAS?$AAW?$AA_?$AAM?$AAO?$AAD?$AAE?$AAM?$AA_?$AAE?$AAN?$AAA?$AAB?$AAL?$AAE?$AA_?$AAD?$AAA?$AAT?$AAA?$AA_?$AAB?$AAU?$AAN?$AAD?$AAL?$AAE?$AA?$AA@ 1001c654     swiroutines.obj
 0002:00005690       ??_C@_1EI@BOAOLHGD@?$AAS?$AAW?$AA_?$AAM?$AAO?$AAD?$AAE?$AAM?$AA_?$AAC?$AAL?$AAE?$AAA?$AAR?$AA_?$AAD?$AAE?$AAV?$AAI?$AAC?$AAE?$AA_?$AAR?$AAE?$AAM?$AAO?$AAT?$AAE?$AA_?$AAW?$AAA?$AAK@ 1001c690     swiroutines.obj
 0002:000056d8       ??_C@_1DE@EGFADNCC@?$AAS?$AAW?$AA_?$AAM?$AAO?$AAD?$AAE?$AAM?$AA_?$AAC?$AAL?$AAE?$AAA?$AAR?$AA_?$AAE?$AAP?$AA_?$AAF?$AAE?$AAA?$AAT?$AAU?$AAR?$AAE?$AA?$AA@ 1001c6d8     swiroutines.obj
 0002:0000570c       ??_C@_1DC@PNJGCNOK@?$AAS?$AAW?$AA_?$AAM?$AAO?$AAD?$AAE?$AAM?$AA_?$AAG?$AAE?$AAT?$AA_?$AAL?$AAI?$AAN?$AAE?$AA_?$AAC?$AAO?$AAD?$AAI?$AAN?$AAG?$AA?$AA@ 1001c70c     swiroutines.obj
 0002:00005740       ??_C@_1EA@HKMBGILL@?$AAS?$AAW?$AA_?$AAM?$AAO?$AAD?$AAE?$AAM?$AA_?$AAE?$AAN?$AAA?$AAB?$AAL?$AAE?$AA_?$AAR?$AAI?$AAN?$AAG?$AA_?$AAI?$AAN?$AAD?$AAI?$AAC?$AAA?$AAT?$AAI?$AAO?$AAN?$AA?$AA@ 1001c740     swiroutines.obj
 0002:00005780       ??_C@_1EA@HCECDGPM@?$AAS?$AAW?$AA_?$AAM?$AAO?$AAD?$AAE?$AAM?$AA_?$AAS?$AAE?$AAT?$AA_?$AAC?$AAO?$AAN?$AAT?$AAR?$AAO?$AAL?$AA_?$AAL?$AAI?$AAN?$AAE?$AA_?$AAS?$AAT?$AAA?$AAT?$AAE?$AA?$AA@ 1001c780     swiroutines.obj
 0002:000057c0       ??_C@_1DC@JBEFFJCJ@?$AAS?$AAW?$AA_?$AAM?$AAO?$AAD?$AAE?$AAM?$AA_?$AAS?$AAE?$AAT?$AA_?$AAL?$AAI?$AAN?$AAE?$AA_?$AAC?$AAO?$AAD?$AAI?$AAN?$AAG?$AA?$AA@ 1001c7c0     swiroutines.obj
 0002:000057f4       ??_C@_1BG@LPCDMPPM@?$AAi?$AAn?$AAd?$AAe?$AAx?$AA?5?$AAz?$AAe?$AAr?$AAo?$AA?$AA@ 1001c7f4     swiroutines.obj
 0002:00005810       ??_C@_1JE@HNPENAJM@?$AAS?$AAi?$AAe?$AAr?$AAr?$AAa?$AAW?$AAi?$AAr?$AAe?$AAl?$AAe?$AAs?$AAs?$AA?5?$AAU?$AAS?$AAB?$AA?3?$AA?5?$AAE?$AAr?$AAr?$AAo?$AAr?$AA?5?$AA?9?$AA?5?$AAf?$AAa?$AAi?$AAl@ 1001c810     swiroutines.obj
 0002:000058a8       ??_C@_1GE@HMMLGCKL@?$AAS?$AAW?$AA?5?$AAU?$AAS?$AAB?$AA?3?$AA?5?$AAF?$AAa?$AAi?$AAl?$AA?5?$AAT?$AAo?$AA?5?$AAO?$AAp?$AAe?$AAn?$AA?5?$AAI?$AAn?$AAt?$AAe?$AAr?$AAr?$AAu?$AAp?$AAt?$AA?5?$AAE@ 1001c8a8     swiroutines.obj
 0002:00005910       ??_C@_1JE@GLKBIMAB@?$AAS?$AAW?$AAI?$AAU?$AAS?$AAB?$AAP?$AAo?$AAw?$AAe?$AAr?$AAC?$AAo?$AAn?$AAt?$AAr?$AAo?$AAl?$AA?5?$AAf?$AAa?$AAi?$AAl?$AAe?$AAd?$AA?5?$AAt?$AAo?$AA?5?$AAS?$AAe?$AAt@ 1001c910     swiroutines.obj
 0002:000059a8       ??_C@_1FM@KPLPAIPA@?$AAg?$AAM?$AAo?$AAd?$AAe?$AAm?$AA?4?$AAl?$AAp?$AAU?$AAS?$AAB?$AAD?$AAI?$AAF?$AAu?$AAn?$AAc?$AAs?$AA?9?$AA?$DO?$AAl?$AAp?$AAR?$AAe?$AAs?$AAu?$AAm?$AAe?$AAD?$AAe?$AAv@ 1001c9a8     swiroutines.obj
 0002:00005a08       ??_C@_1FO@EFBCMNGA@?$AAg?$AAM?$AAo?$AAd?$AAe?$AAm?$AA?4?$AAl?$AAp?$AAU?$AAS?$AAB?$AAD?$AAI?$AAF?$AAu?$AAn?$AAc?$AAs?$AA?9?$AA?$DO?$AAl?$AAp?$AAS?$AAu?$AAs?$AAp?$AAe?$AAn?$AAd?$AAD?$AAe@ 1001ca08     swiroutines.obj
 0002:00005a68       ??_C@_1EO@LAGGILJL@?$AAS?$AAW?$AAI?$AAC?$AAr?$AAe?$AAa?$AAt?$AAe?$AAM?$AAe?$AAm?$AAo?$AAr?$AAy?$AA?5?$AAf?$AAa?$AAi?$AAl?$AAs?$AA?5?$AAl?$AAa?$AAs?$AAt?$AAE?$AAr?$AAr?$AAo?$AAr?$AA?5@ 1001ca68     swiroutines.obj
 0002:00005ab8       ??_C@_1GA@MFKNPGFC@?$AAS?$AAW?$AAI?$AAF?$AAr?$AAe?$AAe?$AAM?$AAe?$AAm?$AAo?$AAr?$AAy?$AA?5?$AAf?$AAa?$AAi?$AAl?$AAs?$AA?5?$AA?$EA?$AA?5?$AA0?$AAx?$AA?$CF?$AAx?$AA?4?$AA?5?$AAB?$AAa?$AAd?$AA?5@ 1001cab8     swiroutines.obj
 0002:00005b18       ??_C@_1FK@EINJEGME@?$AAS?$AAW?$AAI?$AAF?$AAr?$AAe?$AAe?$AAM?$AAe?$AAm?$AAo?$AAr?$AAy?$AA?5?$AAf?$AAa?$AAi?$AAl?$AAs?$AA?5?$AA?$EA?$AA?5?$AA0?$AAx?$AA?$CF?$AAx?$AA?0?$AA?5?$AAl?$AAa?$AAs?$AAt@ 1001cb18     swiroutines.obj
 0002:00005b78       ??_C@_1FC@HBHNINNG@?$AAS?$AAW?$AAI?$AAF?$AAr?$AAe?$AAe?$AAM?$AAe?$AAm?$AAo?$AAr?$AAy?$AA?5?$AAf?$AAa?$AAi?$AAl?$AAs?$AA?5?$AAt?$AAo?$AA?5?$AAD?$AAE?$AAC?$AAO?$AAM?$AAM?$AAI?$AAT?$AA?5@ 1001cb78     swiroutines.obj
 0002:00005bd0       ??_C@_1FE@CJBJKLLB@?$AAE?$AAr?$AAr?$AAo?$AAr?$AA?5?$AAg?$AAe?$AAt?$AAt?$AAi?$AAn?$AAg?$AA?5?$AAd?$AAe?$AAs?$AAc?$AAr?$AAi?$AAp?$AAt?$AAo?$AAr?$AA?5?$AA?$CF?$AAu?$AA?0?$AA?5?$AA?$CF?$AAu?$AA?4@ 1001cbd0     swiroutines.obj
 0002:00005c28       ??_C@_1IC@BEBCBJNC@?$AA?$AN?$AA?6?$AA?5?$AAN?$AAo?$AAn?$AA?9?$AAs?$AAu?$AAp?$AAp?$AAo?$AAr?$AAt?$AAe?$AAd?$AA?5?$AAG?$AAo?$AAb?$AAi?$AA?5?$AAm?$AAo?$AAd?$AAe?$AAm?$AA?5?$AAd?$AAe?$AAt?$AAe@ 1001cc28     swiroutines.obj
 0002:00005cb0       ??_C@_1GA@DKIBCCHC@?$AA?$CF?$AAs?$AA?5?$AAF?$AAa?$AAi?$AAl?$AAe?$AAd?$AA?5?$AAt?$AAo?$AA?5?$AAw?$AAa?$AAi?$AAt?$AA?5?$AAo?$AAb?$AAj?$AAe?$AAc?$AAt?$AA?5?$AAo?$AAn?$AA?5?$AAr?$AAe?$AAs?$AAp@ 1001ccb0     swiroutines.obj
 0002:00005d10       ??_C@_1DI@EBJHNGA@?$AAS?$AAw?$AAi?$AAG?$AAo?$AAb?$AAi?$AA?5?$AAS?$AAe?$AAn?$AAd?$AAS?$AAy?$AAn?$AAc?$AAG?$AAP?$AAS?$AAC?$AAo?$AAm?$AAm?$AAa?$AAn?$AAd?$AA?3?$AA?$AA@ 1001cd10     swiroutines.obj
 0002:00005d48       ??_C@_1FM@PMCELGOM@?$AA?$CF?$AAs?$AA?5?$AAF?$AAa?$AAi?$AAl?$AAe?$AAd?$AA?5?$AAt?$AAo?$AA?5?$AAw?$AAr?$AAi?$AAt?$AAe?$AA?5?$AAc?$AAo?$AAm?$AAm?$AAa?$AAn?$AAd?$AA?5?$AA?$CF?$AAd?$AA?5?$AAt?$AAo@ 1001cd48     swiroutines.obj
 0002:00005da4       ??_C@_0L@HHPDMMBG@$GPS_START?$AA@ 1001cda4     swiroutines.obj
 0002:00005db0       ??_C@_09KAFCFKGE@$GPS_STOP?$AA@ 1001cdb0     swiroutines.obj
 0002:00005dc0       ??_C@_1MK@FBOFAFOB@?$AAS?$AAW?$AA?5?$AAU?$AAS?$AAB?$AA?3?$AA?5?$AAS?$AAe?$AAn?$AAd?$AAI?$AAn?$AAi?$AAt?$AAC?$AAo?$AAn?$AAt?$AAr?$AAo?$AAl?$AAR?$AAe?$AAq?$AAu?$AAe?$AAs?$AAt?$AAs?$AA?5@ 1001cdc0     swiroutines.obj
 0002:00005e90       ??_C@_1NI@OFNKBANI@?$AAS?$AAW?$AA?5?$AAU?$AAS?$AAB?$AA?3?$AA?5?$AAS?$AAe?$AAn?$AAd?$AAI?$AAn?$AAi?$AAt?$AAC?$AAo?$AAn?$AAt?$AAr?$AAo?$AAl?$AAR?$AAe?$AAq?$AAu?$AAe?$AAs?$AAt?$AAs?$AA?5@ 1001ce90     swiroutines.obj
 0002:00005f68       ??_C@_1NC@KMPHAELI@?$AAS?$AAW?$AA?5?$AAU?$AAS?$AAB?$AA?3?$AA?5?$AAS?$AAe?$AAn?$AAd?$AAI?$AAn?$AAi?$AAt?$AAC?$AAo?$AAn?$AAt?$AAr?$AAo?$AAl?$AAR?$AAe?$AAq?$AAu?$AAe?$AAs?$AAt?$AAs?$AA?5@ 1001cf68     swiroutines.obj
 0002:00006040       ??_C@_1NE@KPFJNNMF@?$AAS?$AAW?$AA?5?$AAU?$AAS?$AAB?$AA?3?$AA?5?$AAS?$AAe?$AAn?$AAd?$AAI?$AAn?$AAi?$AAt?$AAC?$AAo?$AAn?$AAt?$AAr?$AAo?$AAl?$AAR?$AAe?$AAq?$AAu?$AAe?$AAs?$AAt?$AAs?$AA?5@ 1001d040     swiroutines.obj
 0002:00006118       ??_C@_1GM@PHEJCCPP@?$AAS?$AAe?$AAn?$AAd?$AAI?$AAn?$AAi?$AAt?$AAC?$AAo?$AAn?$AAt?$AAr?$AAo?$AAl?$AAR?$AAe?$AAq?$AAu?$AAe?$AAs?$AAt?$AAs?$AA?3?$AA?5?$AAd?$AAw?$AAC?$AAh?$AAa?$AAn?$AAn@ 1001d118     swiroutines.obj
 0002:00006188       ??_C@_1JO@LOJMLNKF@?$AAS?$AAW?$AA?5?$AAU?$AAS?$AAB?$AA?3?$AA?5?$AAS?$AAe?$AAn?$AAd?$AAI?$AAn?$AAi?$AAt?$AAC?$AAo?$AAn?$AAt?$AAr?$AAo?$AAl?$AAR?$AAe?$AAq?$AAu?$AAe?$AAs?$AAt?$AAs?$AA?5@ 1001d188     swiroutines.obj
 0002:00006228       ??_C@_1KK@HCNGBHNP@?$AAS?$AAW?$AA?5?$AAU?$AAS?$AAB?$AA?3?$AA?5?$AAS?$AAe?$AAn?$AAd?$AAI?$AAn?$AAi?$AAt?$AAC?$AAo?$AAn?$AAt?$AAr?$AAo?$AAl?$AAR?$AAe?$AAq?$AAu?$AAe?$AAs?$AAt?$AAs?$AA?5@ 1001d228     swiroutines.obj
 0002:000062d8       ??_C@_1LO@DONKJMOO@?$AAU?$AAs?$AAb?$AAS?$AAe?$AAt?$AAH?$AAo?$AAs?$AAt?$AAS?$AAl?$AAe?$AAe?$AAp?$AAP?$AAo?$AAw?$AAe?$AAr?$AAS?$AAt?$AAa?$AAt?$AAe?$AA?5?$AAS?$AAL?$AAE?$AAE?$AAP?$AA?5@ 1001d2d8     swiroutines.obj
 0002:00006398       ??_C@_1IA@BBOGIBAL@?$AAS?$AAe?$AAn?$AAd?$AAH?$AAo?$AAs?$AAt?$AAT?$AAo?$AAI?$AAn?$AAt?$AAe?$AAr?$AAf?$AAa?$AAc?$AAe?$AAC?$AAo?$AAm?$AAm?$AAa?$AAn?$AAd?$AAS?$AAy?$AAn?$AAc?$AA?3?$AA?3@ 1001d398     swiroutines.obj
 0002:00006418       ??_C@_1JI@ILBLMDBE@?$AAS?$AAe?$AAn?$AAd?$AAH?$AAo?$AAs?$AAt?$AAT?$AAo?$AAI?$AAn?$AAt?$AAe?$AAr?$AAf?$AAa?$AAc?$AAe?$AAC?$AAo?$AAm?$AAm?$AAa?$AAn?$AAd?$AAS?$AAy?$AAn?$AAc?$AA?3?$AA?3@ 1001d418     swiroutines.obj
 0002:000064b0       ??_C@_1JK@JPFLBJII@?$AAS?$AAe?$AAn?$AAd?$AAH?$AAo?$AAs?$AAt?$AAT?$AAo?$AAI?$AAn?$AAt?$AAe?$AAr?$AAf?$AAa?$AAc?$AAe?$AAC?$AAo?$AAm?$AAm?$AAa?$AAn?$AAd?$AAS?$AAy?$AAn?$AAc?$AA?3?$AA?3@ 1001d4b0     swiroutines.obj
 0002:00006550       ??_C@_1EG@LIGIGBGK@?$AAS?$AAw?$AAi?$AAG?$AAo?$AAb?$AAi?$AA?5?$AAU?$AAs?$AAb?$AAS?$AAe?$AAt?$AAH?$AAo?$AAs?$AAt?$AAS?$AAl?$AAe?$AAe?$AAp?$AAP?$AAo?$AAw?$AAe?$AAr?$AAS?$AAt?$AAa?$AAt@ 1001d550     swiroutines.obj
 0002:00006598       ??_C@_1DO@NNHPGFID@?$AA?$CF?$AAs?$AA?5?$AAE?$AAn?$AAs?$AAu?$AAr?$AAe?$AAP?$AAo?$AAr?$AAt?$AAR?$AAe?$AAs?$AAu?$AAm?$AAe?$AAd?$AA?5?$AAf?$AAa?$AAi?$AAl?$AAe?$AAd?$AA?4?$AA?$AN?$AA?6?$AA?$AA@ 1001d598     swiroutines.obj
 0002:000065d8       ??_C@_1JA@JCKLAOOP@?$AA?$CF?$AAs?$AA?5?$AAR?$AAe?$AAc?$AAe?$AAi?$AAv?$AAe?$AAd?$AA?5?$AAC?$AAt?$AAl?$AAF?$AAl?$AAa?$AAg?$AAs?$AA?5?$AAd?$AAa?$AAt?$AAa?$AA?5?$AA?$DN?$AA?5?$AA?$CF?$AAd?$AA?0?$AA?5@ 1001d5d8     swiusb.obj
 0002:00006668       ??_C@_1DA@POPHJCCC@?$AAS?$AAw?$AAi?$AAG?$AAo?$AAb?$AAi?$AA?5?$AAD?$AAi?$AAs?$AAp?$AAa?$AAt?$AAc?$AAh?$AAQ?$AAM?$AAI?$AAM?$AAs?$AAg?$AA?3?$AA?$AA@ 1001d668     swiusb.obj
 0002:00006698       ??_C@_1IC@PMBECDPP@?$AA?$CF?$AAs?$AA?5?$AAR?$AAe?$AAc?$AAe?$AAi?$AAv?$AAe?$AAd?$AA?5?$AAI?$AAf?$AAT?$AAy?$AAp?$AAe?$AA?5?$AA?$DN?$AA?5?$AA?$CF?$AAd?$AA?0?$AA?5?$AAd?$AAa?$AAt?$AAa?$AA?5?$AAd?$AAu@ 1001d698     swiusb.obj
 0002:00006720       ??_C@_1GA@FBJMBCLO@?$AAD?$AAi?$AAs?$AAp?$AAa?$AAt?$AAc?$AAh?$AAQ?$AAM?$AAI?$AAM?$AAs?$AAg?$AA?3?$AA?5?$AAT?$AAh?$AAr?$AAe?$AAa?$AAd?$AAI?$AAd?$AA?$DN?$AA0?$AAx?$AA?$CF?$AAx?$AA?5?$AAd?$AAa@ 1001d720     swiusb.obj
 0002:00006780       ??_C@_1HK@LOPCLHEG@?$AAQ?$AAM?$AAI?$AA?5?$AAd?$AAa?$AAt?$AAa?$AA?5?$AAr?$AAe?$AAc?$AAe?$AAi?$AAv?$AAe?$AAd?$AA?5?$AAa?$AAn?$AAd?$AA?5?$AAd?$AAi?$AAs?$AAc?$AAa?$AAr?$AAd?$AAe?$AAd?$AA?5@ 1001d780     swiusb.obj
 0002:00006800       ??_C@_1IO@KAOIMFED@?$AAS?$AAw?$AAi?$AAG?$AAo?$AAb?$AAi?$AA?5?$AAQ?$AAM?$AAI?$AAT?$AAh?$AAr?$AAe?$AAa?$AAd?$AA?3?$AA?5?$AAD?$AAe?$AAv?$AAi?$AAc?$AAe?$AA?5?$AAr?$AAe?$AAm?$AAo?$AAv?$AAa@ 1001d800     swiusb.obj
 0002:00006890       ??_C@_1CC@PNCGBGJI@?$AAQ?$AAM?$AAI?$AAT?$AAh?$AAr?$AAe?$AAa?$AAd?$AA?3?$AA?5?$AAO?$AAu?$AAt?$AA?$AN?$AA?6?$AA?$AA@ 1001d890     swiusb.obj
 0002:000068b4       ??_C@_1CA@IMBFLIGM@?$AAQ?$AAM?$AAI?$AAT?$AAh?$AAr?$AAe?$AAa?$AAd?$AA?3?$AA?5?$AAI?$AAn?$AA?$AN?$AA?6?$AA?$AA@ 1001d8b4     swiusb.obj
 0002:000068d8       ??_C@_1GK@OHIKAIFA@?$AAS?$AAw?$AAi?$AAG?$AAo?$AAb?$AAi?$AA?5?$AAQ?$AAM?$AAI?$AAT?$AAh?$AAr?$AAe?$AAa?$AAd?$AA?3?$AA?5?$AAF?$AAa?$AAi?$AAl?$AAe?$AAd?$AA?5?$AAt?$AAo?$AA?5?$AAw?$AAa?$AAi@ 1001d8d8     swiusb.obj
 0002:00006948       ??_C@_1KO@GMGEHLEK@?$AAS?$AAw?$AAi?$AAG?$AAo?$AAb?$AAi?$AA?5?$AAQ?$AAM?$AAI?$AAT?$AAh?$AAr?$AAe?$AAa?$AAd?$AA?3?$AA?5?$AAT?$AAh?$AAr?$AAe?$AAa?$AAd?$AA?5?$AAw?$AAa?$AAi?$AAt?$AA?5?$AAf@ 1001d948     swiusb.obj
 0002:000069f8       ??_C@_1FE@KBLGFMAM@?$AAS?$AAw?$AAi?$AAG?$AAo?$AAb?$AAi?$AA?5?$AAQ?$AAM?$AAI?$AAT?$AAh?$AAr?$AAe?$AAa?$AAd?$AA?5?$AAe?$AAx?$AAi?$AAt?$AAs?$AA?0?$AA?5?$AAt?$AAi?$AAc?$AAk?$AAC?$AAo?$AAu@ 1001d9f8     swiusb.obj
 0002:00006a88       ??_C@_1EA@MGOHAFJA@?$AAS?$AAw?$AAi?$AAG?$AAo?$AAb?$AAi?$AA?5?$AA?9?$AAI?$AAn?$AAi?$AAt?$AAi?$AAa?$AAl?$AAi?$AAz?$AAe?$AAQ?$AAM?$AAI?$AAC?$AAh?$AAa?$AAn?$AAn?$AAe?$AAl?$AA?$AN?$AA?6?$AA?$AA@ 1001da88     swiusb.obj
 0002:00006ac8       ??_C@_1DM@EJNLPOPH@?$AAS?$AAw?$AAi?$AAG?$AAo?$AAb?$AAi?$AA?5?$AAI?$AAn?$AAi?$AAt?$AAi?$AAa?$AAl?$AAi?$AAz?$AAe?$AAQ?$AAM?$AAI?$AAC?$AAh?$AAa?$AAn?$AAn?$AAe?$AAl?$AA?3?$AA?$AA@ 1001dac8     swiusb.obj
 0002:00006b08       ??_C@_1FK@BCGILHPH@?$AA?$CF?$AAs?$AA?5?$AAF?$AAa?$AAi?$AAl?$AAe?$AAd?$AA?5?$AAt?$AAo?$AA?5?$AAc?$AAr?$AAe?$AAa?$AAt?$AAe?$AA?5?$AAo?$AAb?$AAj?$AAe?$AAc?$AAt?$AA?5?$AAf?$AAo?$AAr?$AA?5?$AAC@ 1001db08     swiusb.obj
 0002:00006b64       ??_C@_1BA@LGMFDPNK@?$AAQ?$AAM?$AAI?$AAD?$AAa?$AAt?$AAa?$AA?$AA@ 1001db64     swiusb.obj
 0002:00006b78       ??_C@_1JK@KNGKGAG@?$AAS?$AAw?$AAi?$AAG?$AAo?$AAb?$AAi?$AA?5?$AAI?$AAn?$AAi?$AAt?$AAi?$AAa?$AAl?$AAi?$AAz?$AAe?$AAQ?$AAM?$AAI?$AAC?$AAh?$AAa?$AAn?$AAn?$AAe?$AAl?$AA?3?$AA?5?$AAF?$AAa@ 1001db78     swiusb.obj
 0002:00006c18       ??_C@_1EA@ELEDGPFI@?$AAS?$AAw?$AAi?$AAG?$AAo?$AAb?$AAi?$AA?5?$AA?$CL?$AAI?$AAn?$AAi?$AAt?$AAi?$AAa?$AAl?$AAi?$AAz?$AAe?$AAQ?$AAM?$AAI?$AAC?$AAh?$AAa?$AAn?$AAn?$AAe?$AAl?$AA?$AN?$AA?6?$AA?$AA@ 1001dc18     swiusb.obj
 0002:00006c58       ??_C@_1DK@BFELPNAG@?$AAS?$AAw?$AAi?$AAG?$AAo?$AAb?$AAi?$AA?5?$AA?9?$AAC?$AAl?$AAe?$AAa?$AAn?$AAu?$AAp?$AAQ?$AAM?$AAI?$AAC?$AAh?$AAa?$AAn?$AAn?$AAe?$AAl?$AA?$AN?$AA?6?$AA?$AA@ 1001dc58     swiusb.obj
 0002:00006c98       ??_C@_1EC@IBLPMPCC@?$AAS?$AAw?$AAi?$AAG?$AAo?$AAb?$AAi?$AA?5?$AAQ?$AAm?$AAi?$AAT?$AAh?$AAr?$AAe?$AAa?$AAd?$AA?5?$AAe?$AAx?$AAi?$AAt?$AA?5?$AAt?$AAi?$AAm?$AAe?$AAo?$AAu?$AAt?$AA?$AN?$AA?6@ 1001dc98     swiusb.obj
 0002:00006cdc       ??_C@_1DK@GFDMOLOA@?$AAS?$AAw?$AAi?$AAG?$AAo?$AAb?$AAi?$AA?5?$AA?$CL?$AAC?$AAl?$AAe?$AAa?$AAn?$AAu?$AAp?$AAQ?$AAM?$AAI?$AAC?$AAh?$AAa?$AAn?$AAn?$AAe?$AAl?$AA?$AN?$AA?6?$AA?$AA@ 1001dcdc     swiusb.obj
 0002:00006d18       ??_C@_1EE@CCEGBEIH@?$AAS?$AAw?$AAi?$AAG?$AAo?$AAb?$AAi?$AA?5?$AA?9?$AAC?$AAl?$AAe?$AAa?$AAn?$AAu?$AAp?$AAD?$AAi?$AAr?$AAe?$AAc?$AAt?$AAI?$AAp?$AAC?$AAh?$AAa?$AAn?$AAn?$AAe?$AAl?$AA?$AN@ 1001dd18     swiusb.obj
 0002:00006d60       ??_C@_1GG@HDILOFMI@?$AAS?$AAw?$AAi?$AAG?$AAo?$AAb?$AAi?$AA?5?$AAI?$AAn?$AAt?$AAe?$AAr?$AAr?$AAu?$AAp?$AAt?$AAT?$AAh?$AAr?$AAe?$AAa?$AAd?$AA?0?$AA?5?$AAc?$AAh?$AAa?$AAn?$AAn?$AAe?$AAl@ 1001dd60     swiusb.obj
 0002:00006dc8       ??_C@_1HC@MIMLBHAN@?$AAS?$AAw?$AAi?$AAG?$AAo?$AAb?$AAi?$AA?5?$AAB?$AAu?$AAl?$AAk?$AAO?$AAu?$AAt?$AAD?$AAi?$AAr?$AAe?$AAc?$AAt?$AAI?$AAp?$AAT?$AAh?$AAr?$AAe?$AAa?$AAd?$AA?0?$AA?5?$AAc@ 1001ddc8     swiusb.obj
 0002:00006e40       ??_C@_1HA@CFFNBOLC@?$AAS?$AAw?$AAi?$AAG?$AAo?$AAb?$AAi?$AA?5?$AAB?$AAu?$AAl?$AAk?$AAI?$AAn?$AAD?$AAi?$AAr?$AAe?$AAc?$AAt?$AAI?$AAp?$AAT?$AAh?$AAr?$AAe?$AAa?$AAd?$AA?0?$AA?5?$AAc?$AAh@ 1001de40     swiusb.obj
 0002:00006eb0       ??_C@_1EE@INJNBKOI@?$AAS?$AAw?$AAi?$AAG?$AAo?$AAb?$AAi?$AA?5?$AA?$CL?$AAC?$AAl?$AAe?$AAa?$AAn?$AAu?$AAp?$AAD?$AAi?$AAr?$AAe?$AAc?$AAt?$AAI?$AAp?$AAC?$AAh?$AAa?$AAn?$AAn?$AAe?$AAl?$AA?$AN@ 1001deb0     swiusb.obj
 0002:00006f50       ??_C@_1FI@GDCFFDCI@?$AAS?$AAw?$AAi?$AAG?$AAo?$AAb?$AAi?$AA?5?$AAF?$AAa?$AAi?$AAl?$AAe?$AAd?$AA?5?$AAt?$AAo?$AA?5?$AAi?$AAn?$AAi?$AAt?$AAi?$AAa?$AAl?$AAi?$AAz?$AAe?$AA?5?$AAD?$AAM?$AAS@ 1001df50     swiusb.obj
 0002:00006fa8       ??_C@_1FE@OJDANFEM@?$AAS?$AAw?$AAi?$AAG?$AAo?$AAb?$AAi?$AA?5?$AAF?$AAa?$AAi?$AAl?$AAe?$AAd?$AA?5?$AAt?$AAo?$AA?5?$AAa?$AAl?$AAl?$AAo?$AAc?$AAa?$AAt?$AAe?$AA?5?$AAD?$AAM?$AAS?$AA?5?$AAs@ 1001dfa8     swiusb.obj
 0002:00007000       ??_C@_1FK@JGNECOPF@?$AAS?$AAw?$AAi?$AAG?$AAo?$AAb?$AAi?$AA?5?$AAG?$AAe?$AAt?$AAC?$AAl?$AAi?$AAe?$AAn?$AAt?$AAI?$AAD?$AA?$CI?$AAD?$AAM?$AAS?$AA?$CJ?$AA?5?$AAa?$AAf?$AAt?$AAe?$AAr?$AA?5?$AA?$CF@ 1001e000     swiusb.obj
 0002:00007060       ??_C@_1GK@HDNOKEBM@?$AAS?$AAw?$AAi?$AAG?$AAo?$AAb?$AAi?$AA?5?$AAG?$AAe?$AAt?$AAC?$AAl?$AAi?$AAe?$AAn?$AAt?$AAI?$AAD?$AA?$CI?$AAD?$AAM?$AAS?$AA?$CJ?$AA?5?$AAf?$AAa?$AAi?$AAl?$AAe?$AAd?$AA?0@ 1001e060     swiusb.obj
 0002:000070d0       ??_C@_1HE@FCLFGHIL@?$AAS?$AAt?$AAa?$AAr?$AAt?$AAD?$AAm?$AAs?$AAS?$AAe?$AAr?$AAv?$AAi?$AAc?$AAe?$AA?3?$AA?5?$AAD?$AAe?$AAv?$AAi?$AAc?$AAe?$AA?5?$AAr?$AAe?$AAm?$AAo?$AAv?$AAe?$AAd?$AA?5@ 1001e0d0     swiusb.obj
 0002:000071a0       ??_C@_1FI@FLHCFPMH@?$AAS?$AAw?$AAi?$AAG?$AAo?$AAb?$AAi?$AA?5?$AAF?$AAa?$AAi?$AAl?$AAe?$AAd?$AA?5?$AAt?$AAo?$AA?5?$AAi?$AAn?$AAi?$AAt?$AAi?$AAa?$AAl?$AAi?$AAz?$AAe?$AA?5?$AAW?$AAD?$AAS@ 1001e1a0     swiusb.obj
 0002:000071f8       ??_C@_1FE@NBGHNJKD@?$AAS?$AAw?$AAi?$AAG?$AAo?$AAb?$AAi?$AA?5?$AAF?$AAa?$AAi?$AAl?$AAe?$AAd?$AA?5?$AAt?$AAo?$AA?5?$AAa?$AAl?$AAl?$AAo?$AAc?$AAa?$AAt?$AAe?$AA?5?$AAW?$AAD?$AAS?$AA?5?$AAs@ 1001e1f8     swiusb.obj
 0002:00007250       ??_C@_1FK@OEJFDMIH@?$AAS?$AAw?$AAi?$AAG?$AAo?$AAb?$AAi?$AA?5?$AAG?$AAe?$AAt?$AAC?$AAl?$AAi?$AAe?$AAn?$AAt?$AAI?$AAD?$AA?$CI?$AAW?$AAD?$AAS?$AA?$CJ?$AA?5?$AAa?$AAf?$AAt?$AAe?$AAr?$AA?5?$AA?$CF@ 1001e250     swiusb.obj
 0002:000072b0       ??_C@_1GK@MBOCMDPA@?$AAS?$AAw?$AAi?$AAG?$AAo?$AAb?$AAi?$AA?5?$AAG?$AAe?$AAt?$AAC?$AAl?$AAi?$AAe?$AAn?$AAt?$AAI?$AAD?$AA?$CI?$AAW?$AAD?$AAS?$AA?$CJ?$AA?5?$AAf?$AAa?$AAi?$AAl?$AAe?$AAd?$AA?0@ 1001e2b0     swiusb.obj
 0002:00007320       ??_C@_1HE@MMKBEHAL@?$AAS?$AAt?$AAa?$AAr?$AAt?$AAW?$AAd?$AAs?$AAS?$AAe?$AAr?$AAv?$AAi?$AAc?$AAe?$AA?3?$AA?5?$AAD?$AAe?$AAv?$AAi?$AAc?$AAe?$AA?5?$AAr?$AAe?$AAm?$AAo?$AAv?$AAe?$AAd?$AA?5@ 1001e320     swiusb.obj
 0002:00007398       ??_C@_1EK@GJNAAJOA@?$AA?$CK?$AA?$CK?$AA?$CK?$AA?5?$AAS?$AAw?$AAi?$AAG?$AAo?$AAb?$AAi?$AA?5?$AAR?$AAe?$AAs?$AAe?$AAt?$AAP?$AAi?$AAp?$AAe?$AA?5?$AAE?$AAR?$AAR?$AAO?$AAR?$AA?3?$AA?$CF?$AAd?$AA?5?$AA?$CK@ 1001e398     swiusb.obj
 0002:000073e4       ??_C@_1BE@OEMMCIEP@?$AA?2?$AA?$CF?$AAd?$AA_?$AA?$CF?$AAd?$AA_?$AA?$CF?$AAd?$AA?$AA@ 1001e3e4     swiusb.obj
 0002:000073f8       ??_C@_1BC@GEJDPPEB@?$AA?2?$AAD?$AAe?$AAf?$AAa?$AAu?$AAl?$AAt?$AA?$AA@ 1001e3f8     swiusb.obj
 0002:0000740c       ??_C@_1BI@OLMMMJNF@?$AA?$CF?$AAs?$AA?2?$AA?$CF?$AAs?$AA?2?$AA?$CF?$AAd?$AA_?$AA?$CF?$AAd?$AA?$AA@ 1001e40c     swiusb.obj
 0002:00007428       ??_C@_1OG@JNJDPHFH@?$AAS?$AAw?$AAi?$AAG?$AAo?$AAb?$AAi?$AA?5?$AAT?$AAr?$AAa?$AAn?$AAs?$AAm?$AAi?$AAt?$AAB?$AAy?$AAt?$AAe?$AAs?$AA?3?$AA?5?$AAC?$AAh?$AAa?$AAn?$AAn?$AAe?$AAl?$AAN?$AAu@ 1001e428     swiusb.obj
 0002:00007510       ??_C@_1PG@IMHMOFDH@?$AAS?$AAw?$AAi?$AAG?$AAo?$AAb?$AAi?$AA?5?$AAT?$AAr?$AAa?$AAn?$AAs?$AAm?$AAi?$AAt?$AAB?$AAy?$AAt?$AAe?$AAs?$AAD?$AAi?$AAr?$AAe?$AAc?$AAt?$AAI?$AAp?$AA?3?$AA?5?$AAC@ 1001e510     swiusb.obj
 0002:00007608       ??_C@_1FM@KJOGJHAH@?$AAS?$AAw?$AAi?$AAG?$AAo?$AAb?$AAi?$AA?5?$AAR?$AAi?$AAl?$AAN?$AAd?$AAi?$AAs?$AAS?$AAe?$AAn?$AAd?$AAP?$AAa?$AAc?$AAk?$AAe?$AAt?$AA?3?$AA?5?$AAp?$AAa?$AAc?$AAk?$AAe@ 1001e608     swiusb.obj
 0002:00007668       ??_C@_1HC@MNCABPAM@?$AAS?$AAw?$AAi?$AAG?$AAo?$AAb?$AAi?$AA?5?$AAR?$AAi?$AAl?$AAN?$AAd?$AAi?$AAs?$AAS?$AAe?$AAn?$AAd?$AAP?$AAa?$AAc?$AAk?$AAe?$AAt?$AA?3?$AA?5?$AAa?$AAl?$AAl?$AAo?$AAc@ 1001e668     swiusb.obj
 0002:000076e0       ??_C@_1JE@PLPABAK@?$AAR?$AAi?$AAl?$AAN?$AAd?$AAi?$AAs?$AAS?$AAe?$AAn?$AAd?$AAP?$AAa?$AAc?$AAk?$AAe?$AAt?$AA?5?$AAt?$AAr?$AAy?$AAi?$AAn?$AAg?$AA?5?$AAt?$AAo?$AA?5?$AAs?$AAe?$AAn?$AAd@ 1001e6e0     swiusb.obj
 0002:00007778       ??_C@_1GC@ONJCIFEA@?$AAS?$AAw?$AAi?$AAG?$AAo?$AAb?$AAi?$AA?3?$AA?5?$AAI?$AAn?$AAt?$AAe?$AAr?$AAr?$AAu?$AAp?$AAt?$AA?5?$AAT?$AAh?$AAr?$AAe?$AAa?$AAd?$AA?5?$AAE?$AAx?$AAi?$AAt?$AA?0?$AA?5@ 1001e778     swiusb.obj
 0002:000077e0       ??_C@_1GI@FAIBCAH@?$AAS?$AAw?$AAi?$AAG?$AAo?$AAb?$AAi?$AA?5?$AAI?$AAn?$AAt?$AAe?$AAr?$AAr?$AAu?$AAp?$AAt?$AAT?$AAh?$AAr?$AAe?$AAa?$AAd?$AA?5?$AAe?$AAx?$AAi?$AAt?$AAs?$AA?5?$AAb?$AAc@ 1001e7e0     swiusb.obj
 0002:00007848       ??_C@_1LC@ILIIDMKJ@?$AA?$AN?$AA?6?$AAS?$AAw?$AAi?$AAG?$AAo?$AAb?$AAi?$AA?5?$AAI?$AAn?$AAt?$AAe?$AAr?$AAr?$AAu?$AAp?$AAt?$AAT?$AAh?$AAr?$AAe?$AAa?$AAd?$AA?3?$AA?5?$AAA?$AAb?$AAo?$AAu?$AAt@ 1001e848     swiusb.obj
 0002:00007900       ??_C@_1NK@CJFIENBD@?$AAS?$AAw?$AAi?$AAG?$AAo?$AAb?$AAi?$AA?5?$AAG?$AAe?$AAt?$AA?5?$AAI?$AAn?$AAt?$AAe?$AAr?$AAr?$AAu?$AAp?$AAt?$AA?5?$AAT?$AAr?$AAa?$AAn?$AAs?$AAf?$AAe?$AAr?$AA?5?$AAe@ 1001e900     swiusb.obj
 0002:000079e0       ??_C@_1GA@JLGJKCEN@?$AAF?$AAa?$AAi?$AAl?$AAe?$AAd?$AA?5?$AAt?$AAo?$AA?5?$AAr?$AAe?$AAs?$AAe?$AAt?$AA?5?$AAi?$AAn?$AAt?$AAe?$AAr?$AAr?$AAu?$AAp?$AAt?$AA?5?$AAp?$AAi?$AAp?$AAe?$AA?5?$AAo@ 1001e9e0     swiusb.obj
 0002:00007a40       ??_C@_1JM@MCBOLKAL@?$AAI?$AAn?$AAt?$AAe?$AAr?$AAu?$AAp?$AAt?$AAT?$AAh?$AAr?$AAe?$AAa?$AAd?$AA?3?$AA?5?$AAA?$AAb?$AAo?$AAu?$AAt?$AA?5?$AAt?$AAo?$AA?5?$AAr?$AAe?$AAs?$AAu?$AAm?$AAe?$AA?5@ 1001ea40     swiusb.obj
 0002:00007ae0       ??_C@_1KA@EGEGGEIK@?$AAI?$AAn?$AAt?$AAe?$AAr?$AAr?$AAu?$AAp?$AAt?$AAT?$AAh?$AAr?$AAe?$AAa?$AAd?$AA?5?$AAf?$AAo?$AAr?$AAc?$AAe?$AAs?$AA?5?$AAi?$AAs?$AAP?$AAo?$AAr?$AAt?$AAS?$AAu?$AAs@ 1001eae0     swiusb.obj
 0002:00007b80       ??_C@_1HM@CMJENPOC@?$AAI?$AAn?$AAt?$AAe?$AAr?$AAr?$AAu?$AAp?$AAt?$AAT?$AAh?$AAr?$AAe?$AAa?$AAd?$AA?5?$AA?3?$AAW?$AAa?$AAi?$AAt?$AAi?$AAn?$AAg?$AA?5?$AAf?$AAo?$AAr?$AA?5?$AAd?$AAe?$AAv@ 1001eb80     swiusb.obj
 0002:00007c00       ??_C@_1IO@JLHKKCBO@?$AAS?$AAw?$AAi?$AAG?$AAo?$AAb?$AAi?$AA?5?$AAp?$AAC?$AAo?$AAm?$AAm?$AAp?$AAo?$AAr?$AAt?$AAM?$AAd?$AAd?$AA?5?$AAi?$AAs?$AA?5?$AAN?$AAU?$AAL?$AAL?$AA?5?$AAf?$AAo?$AAr@ 1001ec00     swiusb.obj
 0002:00007c90       ??_C@_1HC@IDINAHBG@?$AAS?$AAw?$AAi?$AAG?$AAo?$AAb?$AAi?$AA?3?$AA?5?$AAI?$AAn?$AAt?$AAe?$AAr?$AAr?$AAu?$AAp?$AAt?$AAD?$AAi?$AAr?$AAe?$AAc?$AAt?$AAI?$AAp?$AA?5?$AAT?$AAh?$AAr?$AAe?$AAa@ 1001ec90     swiusb.obj
 0002:00007d08       ??_C@_1HI@JGCICBKN@?$AAS?$AAw?$AAi?$AAG?$AAo?$AAb?$AAi?$AA?5?$AAI?$AAn?$AAt?$AAe?$AAr?$AAr?$AAu?$AAp?$AAt?$AAD?$AAi?$AAr?$AAe?$AAc?$AAt?$AAI?$AAp?$AAT?$AAh?$AAr?$AAe?$AAa?$AAd?$AA?5@ 1001ed08     swiusb.obj
 0002:00007d80       ??_C@_1MC@NEMDKOII@?$AA?$AN?$AA?6?$AAS?$AAw?$AAi?$AAG?$AAo?$AAb?$AAi?$AA?5?$AAI?$AAn?$AAt?$AAe?$AAr?$AAr?$AAu?$AAp?$AAt?$AAD?$AAi?$AAr?$AAe?$AAc?$AAt?$AAI?$AAp?$AAT?$AAh?$AAr?$AAe?$AAa@ 1001ed80     swiusb.obj
 0002:00007e48       ??_C@_1LE@DKLJBDID@?$AAI?$AAn?$AAt?$AAe?$AAr?$AAr?$AAu?$AAp?$AAt?$AAD?$AAi?$AAr?$AAe?$AAc?$AAt?$AAI?$AAp?$AAT?$AAh?$AAr?$AAe?$AAa?$AAd?$AA?3?$AA?5?$AAi?$AAs?$AAC?$AAl?$AAe?$AAa?$AAr@ 1001ee48     swiusb.obj
 0002:00007f00       ??_C@_1LA@MKABLLKE@?$AAI?$AAn?$AAt?$AAe?$AAr?$AAr?$AAu?$AAp?$AAt?$AAD?$AAi?$AAr?$AAe?$AAc?$AAt?$AAI?$AAp?$AAT?$AAh?$AAr?$AAe?$AAa?$AAd?$AA?5?$AAf?$AAo?$AAr?$AAc?$AAe?$AAs?$AA?5?$AAi@ 1001ef00     swiusb.obj
 0002:00007fb0       ??_C@_1IM@OLBCKIBA@?$AAI?$AAn?$AAt?$AAe?$AAr?$AAr?$AAu?$AAp?$AAt?$AAD?$AAi?$AAr?$AAe?$AAc?$AAt?$AAI?$AAp?$AAT?$AAh?$AAr?$AAe?$AAa?$AAd?$AA?3?$AA?5?$AAW?$AAa?$AAi?$AAt?$AAi?$AAn?$AAg@ 1001efb0     swiusb.obj
 0002:00008040       ??_C@_1GC@JBEPAGCJ@?$AAS?$AAw?$AAi?$AAG?$AAo?$AAb?$AAi?$AA?5?$AAp?$AAM?$AAd?$AAd?$AA?5?$AAi?$AAs?$AA?5?$AAN?$AAU?$AAL?$AAL?$AA?5?$AAf?$AAo?$AAr?$AA?5?$AA?$CF?$AAs?$AA?5?$AAi?$AAn?$AAt?$AAe@ 1001f040     swiusb.obj
 0002:000080a4       ??_C@_1DK@DBAGBDEO@?$AAS?$AAw?$AAi?$AAG?$AAo?$AAb?$AAi?$AA?5?$AAD?$AAi?$AAs?$AAp?$AAl?$AAa?$AAy?$AAM?$AAe?$AAm?$AAo?$AAr?$AAy?$AAS?$AAt?$AAa?$AAt?$AAu?$AAs?$AA?3?$AA?$AA@ 1001f0a4     swiusb.obj
 0002:000080e0       ??_C@_1KE@LBNPNIMH@?$AA?$CF?$AAs?$AA?5?$AAM?$AAe?$AAm?$AA?5?$AAs?$AAt?$AAa?$AAt?$AAu?$AAs?$AA?3?$AA?5?$AAT?$AAo?$AAt?$AAa?$AAl?$AAP?$AAh?$AAy?$AAs?$AA?3?$AA?5?$AA?$CF?$AAd?$AA?0?$AA?5?$AAA?$AAv@ 1001f0e0     swiusb.obj
 0002:00008188       ??_C@_1HO@EKHNIINC@?$AAS?$AAw?$AAi?$AAG?$AAo?$AAb?$AAi?$AA?3?$AA?5?$AAD?$AAe?$AAv?$AAi?$AAc?$AAe?$AA?5?$AAR?$AAe?$AAm?$AAo?$AAv?$AAe?$AAd?$AA?5?$AA?$EA?$AA?5?$AAt?$AAc?$AA?5?$AA?$DN?$AA?5?$AA?$CF@ 1001f188     swiusb.obj
 0002:00008208       ??_C@_1IC@LOEEAHEO@?$AAS?$AAw?$AAi?$AAG?$AAo?$AAb?$AAi?$AA?5?$AAU?$AAS?$AAB?$AAD?$AAe?$AAv?$AAi?$AAc?$AAe?$AAN?$AAo?$AAt?$AAi?$AAf?$AAi?$AAc?$AAa?$AAt?$AAi?$AAo?$AAn?$AAs?$AA?3?$AA?5@ 1001f208     swiusb.obj
 0002:00008290       ??_C@_1EE@NJKPCDFH@?$AAS?$AAw?$AAi?$AAG?$AAo?$AAb?$AAi?$AA?5?$AAD?$AAe?$AAa?$AAc?$AAt?$AAi?$AAv?$AAa?$AAt?$AAe?$AA?5?$AAQ?$AAM?$AAI?$AA1?$AA?3?$AA?5?$AAf?$AAa?$AAi?$AAl?$AAe?$AAd?$AA?$AN@ 1001f290     swiusb.obj
 0002:000082d8       ??_C@_1GC@BPAJEJEK@?$AAS?$AAw?$AAi?$AAG?$AAo?$AAb?$AAi?$AA?5?$AAB?$AAu?$AAl?$AAk?$AAO?$AAu?$AAt?$AAT?$AAh?$AAr?$AAe?$AAa?$AAd?$AA?0?$AA?5?$AAc?$AAh?$AAa?$AAn?$AAn?$AAe?$AAl?$AA?5?$AA?$CF@ 1001f2d8     swiusb.obj
 0002:00008340       ??_C@_1GA@FFLPJKOE@?$AAS?$AAw?$AAi?$AAG?$AAo?$AAb?$AAi?$AA?5?$AAB?$AAu?$AAl?$AAk?$AAI?$AAn?$AAT?$AAh?$AAr?$AAe?$AAa?$AAd?$AA?0?$AA?5?$AAc?$AAh?$AAa?$AAn?$AAn?$AAe?$AAl?$AA?5?$AA?$CF?$AAd@ 1001f340     swiusb.obj
 0002:000083a0       ??_C@_1EO@KJFLEPPC@?$AAS?$AAw?$AAi?$AAG?$AAo?$AAb?$AAi?$AA?5?$AAh?$AAA?$AAc?$AAt?$AAi?$AAv?$AAi?$AAt?$AAy?$AAT?$AAh?$AAr?$AAe?$AAa?$AAd?$AA?5?$AAe?$AAx?$AAi?$AAt?$AA?5?$AAt?$AAi?$AAm@ 1001f3a0     swiusb.obj
 0002:000083f0       ??_C@_1GI@JPHJHAJL@?$AAS?$AAw?$AAi?$AAG?$AAo?$AAb?$AAi?$AA?5?$AAN?$AAd?$AAi?$AAs?$AAD?$AAe?$AAr?$AAe?$AAg?$AAi?$AAs?$AAt?$AAe?$AAr?$AAA?$AAd?$AAa?$AAp?$AAt?$AAe?$AAr?$AA?5?$AAf?$AAa@ 1001f3f0     swiusb.obj
 0002:00008458       ??_C@_1EG@NKDFBPEM@?$AAS?$AAw?$AAi?$AAG?$AAo?$AAb?$AAi?$AA?5?$AAN?$AAd?$AAi?$AAs?$AAD?$AAe?$AAr?$AAe?$AAg?$AAi?$AAs?$AAt?$AAe?$AAr?$AAA?$AAd?$AAa?$AAp?$AAt?$AAe?$AAr?$AA?5?$AAO?$AAK@ 1001f458     swiusb.obj
 0002:000084a0       ??_C@_1FA@EHCJFIKE@?$AAS?$AAw?$AAi?$AAG?$AAo?$AAb?$AAi?$AA?5?$AAC?$AAa?$AAl?$AAl?$AAi?$AAn?$AAg?$AA?5?$AAN?$AAd?$AAi?$AAs?$AAD?$AAe?$AAr?$AAe?$AAg?$AAi?$AAs?$AAt?$AAe?$AAr?$AAA?$AAd@ 1001f4a0     swiusb.obj
 0002:000084f0       ??_C@_1BO@LGKPMAIO@?$AAS?$AAW?$AAG?$AAo?$AAb?$AAi?$AAU?$AAS?$AAB?$AAN?$AAD?$AAI?$AAS?$AA1?$AA?$AA@ 1001f4f0     swiusb.obj
 0002:00008510       ??_C@_1BK@KPLOIJDF@?$AAM?$AAi?$AAn?$AAi?$AAp?$AAo?$AAr?$AAt?$AAN?$AAa?$AAm?$AAe?$AA?$AA@ 1001f510     swiusb.obj
 0002:0000852c       ??_C@_1BC@FDHFOMEN@?$AAD?$AAe?$AAv?$AAi?$AAc?$AAe?$AAI?$AAD?$AA?$AA@ 1001f52c     swiusb.obj
 0002:00008540       ??_C@_1FG@FMKGKDFP@?$AAS?$AAi?$AAg?$AAn?$AAa?$AAl?$AA?5?$AAA?$AAP?$AAI?$AA?5?$AAt?$AAh?$AAa?$AAt?$AA?5?$AAd?$AAe?$AAv?$AAi?$AAc?$AAe?$AA?5?$AAh?$AAa?$AAs?$AA?5?$AAb?$AAe?$AAe?$AAn?$AA?5@ 1001f540     swiusb.obj
 0002:00008598       ??_C@_1EG@ENBGGGFB@?$AAS?$AAw?$AAi?$AAG?$AAo?$AAb?$AAi?$AA?3?$AA?5?$AA?$CB?$AA?$CB?$AA?$CB?$AA?5?$AAD?$AAe?$AAv?$AAi?$AAc?$AAe?$AA?5?$AAr?$AAe?$AAm?$AAo?$AAv?$AAe?$AAd?$AA?5?$AA?$CB?$AA?$CB?$AA?$CB?$AA?5@ 1001f598     swiusb.obj
 0002:000085e0       ??_C@_1FM@GPNAOFCO@?$AAS?$AAi?$AAg?$AAn?$AAa?$AAl?$AA?5?$AAd?$AAr?$AAi?$AAv?$AAe?$AAr?$AA?5?$AAt?$AAh?$AAa?$AAt?$AA?5?$AAd?$AAe?$AAv?$AAi?$AAc?$AAe?$AA?5?$AAh?$AAa?$AAs?$AA?5?$AAb?$AAe@ 1001f5e0     swiusb.obj
 0002:00008640       ??_C@_1GC@LMOGAKGL@?$AAS?$AAw?$AAi?$AAG?$AAo?$AAb?$AAi?$AA?5?$AAU?$AAn?$AAh?$AAa?$AAn?$AAd?$AAl?$AAe?$AAd?$AA?5?$AAU?$AAS?$AAB?$AA?5?$AAn?$AAo?$AAt?$AAi?$AAf?$AAi?$AAc?$AAa?$AAt?$AAi@ 1001f640     swiusb.obj
 0002:000086a8       ??_C@_1FG@DCMDDMKJ@?$AAU?$AAS?$AAB?$AAI?$AAn?$AAs?$AAt?$AAa?$AAl?$AAl?$AAD?$AAr?$AAi?$AAv?$AAe?$AAr?$AA?5?$AAi?$AAs?$AA?5?$AAc?$AAa?$AAl?$AAl?$AAe?$AAd?$AA?5?$AAf?$AAo?$AAr?$AA?5?$AAd@ 1001f6a8     swiusb.obj
 0002:00008700       ??_C@_17JADPJEII@?$AAP?$AAD?$AAP?$AA?$AA@ 1001f700     swiusb.obj
 0002:00008708       ??_C@_1LE@BONBHEGL@?$AAS?$AAw?$AAi?$AAG?$AAo?$AAb?$AAi?$AA?5?$AAW?$AAa?$AAi?$AAt?$AA?5?$AAf?$AAo?$AAr?$AA?5?$AAp?$AAo?$AAr?$AAt?$AA?5?$AAs?$AAu?$AAs?$AAp?$AAe?$AAn?$AAd?$AAe?$AAd?$AA?5@ 1001f708     swiusb.obj
 0002:000087c0       ??_C@_1HK@OPGCLGFJ@?$AAS?$AAw?$AAi?$AAG?$AAo?$AAb?$AAi?$AA?5?$AAR?$AAe?$AAs?$AAu?$AAm?$AAe?$AAd?$AA?5?$AAw?$AAa?$AAi?$AAt?$AA?5?$AAf?$AAo?$AAr?$AA?5?$AAs?$AAu?$AAs?$AAp?$AAe?$AAn?$AAd@ 1001f7c0     swiusb.obj
 0002:00008840       ??_C@_1GA@MIFFOIFD@?$AAS?$AAw?$AAi?$AAG?$AAo?$AAb?$AAi?$AA?5?$AAW?$AAa?$AAi?$AAt?$AAi?$AAn?$AAg?$AA?5?$AAf?$AAo?$AAr?$AA?5?$AAs?$AAu?$AAs?$AAp?$AAe?$AAn?$AAd?$AA?5?$AAb?$AAu?$AAt?$AA?5@ 1001f840     swiusb.obj
 0002:000088a0       ??_C@_1BCK@LDPGOCGP@?$AAM?$AAo?$AAd?$AAe?$AAm?$AA?5?$AAi?$AAn?$AAt?$AAe?$AAr?$AAr?$AAu?$AAp?$AAt?$AAs?$AA?5?$AAd?$AAu?$AAr?$AAi?$AAn?$AAg?$AA?5?$AAg?$AAD?$AAe?$AAv?$AAi?$AAc?$AAe?$AAP@ 1001f8a0     swiusb.obj
 0002:000089cc       ??_C@_1BG@PGILDLLG@?$AAu?$AAn?$AAa?$AAt?$AAt?$AAe?$AAn?$AAd?$AAe?$AAd?$AA?$AA@ 1001f9cc     swiusb.obj
 0002:000089e8       ??_C@_1HM@NMBENKNL@?$AAS?$AAw?$AAi?$AAG?$AAo?$AAb?$AAi?$AA?5?$AAS?$AAu?$AAs?$AAp?$AAe?$AAn?$AAd?$AAe?$AAd?$AA?5?$AAw?$AAa?$AAi?$AAt?$AA?5?$AAf?$AAo?$AAr?$AA?5?$AAr?$AAe?$AAs?$AAu?$AAm@ 1001f9e8     swiusb.obj
 0002:00008a68       ??_C@_1GE@HKDHMCKD@?$AAA?$AAc?$AAt?$AAi?$AAv?$AAi?$AAt?$AAy?$AAT?$AAh?$AAr?$AAe?$AAa?$AAd?$AA?5?$AAU?$AAn?$AAb?$AAl?$AAo?$AAc?$AAk?$AA?5?$AAb?$AAe?$AAc?$AAa?$AAu?$AAs?$AAe?$AA?0?$AA?5@ 1001fa68     swiusb.obj
 0002:00008ad0       ??_C@_1FO@IBCIFKNM@?$AAS?$AAw?$AAi?$AAG?$AAo?$AAb?$AAi?$AA?5?$AAW?$AAa?$AAi?$AAt?$AAi?$AAn?$AAg?$AA?5?$AAf?$AAo?$AAr?$AA?5?$AAr?$AAe?$AAs?$AAu?$AAm?$AAe?$AA?5?$AAb?$AAu?$AAt?$AA?5?$AAw@ 1001fad0     swiusb.obj
 0002:00008b30       ??_C@_1GM@DCIMNFOC@?$AAS?$AAw?$AAi?$AAG?$AAo?$AAb?$AAi?$AA?5?$AAP?$AAa?$AAr?$AAs?$AAe?$AAT?$AAl?$AAp?$AAT?$AAr?$AAa?$AAn?$AAs?$AAf?$AAe?$AAr?$AA?3?$AA?5?$AAE?$AAt?$AAh?$AAe?$AAr?$AAn@ 1001fb30     swiusb.obj
 0002:00008ba0       ??_C@_1GM@NKCGGICJ@?$AAS?$AAw?$AAi?$AAG?$AAo?$AAb?$AAi?$AA?5?$AAP?$AAa?$AAr?$AAs?$AAe?$AAT?$AAl?$AAp?$AAT?$AAr?$AAa?$AAn?$AAs?$AAf?$AAe?$AAr?$AA?3?$AA?5?$AAE?$AAt?$AAh?$AAe?$AAr?$AAn@ 1001fba0     swiusb.obj
 0002:00008c10       ??_C@_1FO@FDIKDKEN@?$AAS?$AAw?$AAi?$AAG?$AAo?$AAb?$AAi?$AA?5?$AAP?$AAa?$AAr?$AAs?$AAe?$AAT?$AAl?$AAp?$AAT?$AAr?$AAa?$AAn?$AAs?$AAf?$AAe?$AAr?$AA?3?$AA?5?$AAB?$AAa?$AAd?$AA?5?$AAT?$AAL@ 1001fc10     swiusb.obj
 0002:00008c70       ??_C@_1HM@ONMCFGBO@?$AAS?$AAw?$AAi?$AAG?$AAo?$AAb?$AAi?$AA?5?$AAP?$AAa?$AAr?$AAs?$AAe?$AAT?$AAl?$AAp?$AAT?$AAr?$AAa?$AAn?$AAs?$AAf?$AAe?$AAr?$AA?3?$AA?5?$AAe?$AAt?$AAh?$AAe?$AAr?$AAn@ 1001fc70     swiusb.obj
 0002:00008cf0       ??_C@_1GO@POBLCIJG@?$AAS?$AAw?$AAi?$AAG?$AAo?$AAb?$AAi?$AA?3?$AA?5?$AAE?$AAt?$AAh?$AAe?$AAr?$AAn?$AAe?$AAt?$AAF?$AAr?$AAa?$AAm?$AAe?$AAH?$AAa?$AAn?$AAd?$AAl?$AAe?$AAr?$AAR?$AAi?$AAl@ 1001fcf0     swiusb.obj
 0002:00008d60       ??_C@_1GK@LDKFHKKJ@?$AAS?$AAw?$AAi?$AAG?$AAo?$AAb?$AAi?$AA?3?$AA?5?$AAE?$AAt?$AAh?$AAe?$AAr?$AAn?$AAe?$AAt?$AAF?$AAr?$AAa?$AAm?$AAe?$AAH?$AAa?$AAn?$AAd?$AAl?$AAe?$AAr?$AAR?$AAi?$AAl@ 1001fd60     swiusb.obj
 0002:00008dd0       ??_C@_1EC@CCMPGMLD@?$AAS?$AAw?$AAi?$AAG?$AAo?$AAb?$AAi?$AA?3?$AA?5?$AAR?$AAe?$AAc?$AAe?$AAi?$AAv?$AAe?$AAd?$AA?5?$AAA?$AAR?$AAP?$AA?5?$AAr?$AAe?$AAq?$AAu?$AAe?$AAs?$AAt?$AA?4?$AA?$AN?$AA?6@ 1001fdd0     swiusb.obj
 0002:00008e18       ??_C@_1JG@KGGBMIGL@?$AAS?$AAw?$AAi?$AAG?$AAo?$AAb?$AAi?$AA?3?$AA?5?$AAE?$AAt?$AAh?$AAe?$AAr?$AAn?$AAe?$AAt?$AAF?$AAr?$AAa?$AAm?$AAe?$AAH?$AAa?$AAn?$AAd?$AAl?$AAe?$AAr?$AAR?$AAi?$AAl@ 1001fe18     swiusb.obj
 0002:00008eb0       ??_C@_1HK@IOHHCPNA@?$AAE?$AAt?$AAh?$AAe?$AAr?$AAn?$AAe?$AAt?$AAF?$AAr?$AAa?$AAm?$AAe?$AAH?$AAa?$AAn?$AAd?$AAl?$AAe?$AAr?$AAR?$AAi?$AAl?$AAP?$AAa?$AAc?$AAk?$AAe?$AAt?$AA?5?$AAu?$AAn@ 1001feb0     swiusb.obj
 0002:00008f30       ??_C@_1EA@LCPHBMND@?$AAP?$AAe?$AAn?$AAd?$AAi?$AAn?$AAg?$AA?5?$AAo?$AAu?$AAt?$AA?5?$AAp?$AAa?$AAc?$AAk?$AAe?$AAt?$AAs?$AA?5?$AAr?$AAe?$AAl?$AAe?$AAa?$AAs?$AAe?$AAd?$AA?4?$AA?$AN?$AA?6?$AA?$AA@ 1001ff30     swiusb.obj
 0002:00008f70       ??_C@_1IO@KHHLFEHL@?$AA?6?$AAS?$AAw?$AAi?$AAG?$AAo?$AAb?$AAi?$AA?5?$AAB?$AAu?$AAl?$AAk?$AAI?$AAn?$AAD?$AAi?$AAr?$AAe?$AAc?$AAt?$AAI?$AAp?$AAN?$AAo?$AAT?$AAl?$AAp?$AAT?$AAh?$AAr?$AAe@ 1001ff70     swiusb.obj
 0002:00009000       ??_C@_1JI@GHOECOPD@?$AA?6?$AAS?$AAw?$AAi?$AAG?$AAo?$AAb?$AAi?$AA?5?$AAB?$AAu?$AAl?$AAk?$AAI?$AAn?$AAD?$AAi?$AAr?$AAe?$AAc?$AAt?$AAI?$AAp?$AAN?$AAo?$AAT?$AAl?$AAp?$AAT?$AAh?$AAr?$AAe@ 10020000     swiusb.obj
 0002:00009098       ??_C@_1II@IBBJGHJD@?$AA?$AN?$AA?6?$AA?$CF?$AAs?$AA?3?$AA?5?$AAA?$AAb?$AAo?$AAu?$AAt?$AA?5?$AAt?$AAo?$AA?5?$AAr?$AAe?$AAs?$AAu?$AAm?$AAe?$AA?5?$AAo?$AAp?$AAe?$AAr?$AAa?$AAt?$AAi?$AAo?$AAn?$AA?0@ 10020098     swiusb.obj
 0002:00009120       ??_C@_1IO@GMFAAMPK@?$AAS?$AAw?$AAi?$AAG?$AAo?$AAb?$AAi?$AA?3?$AA?5?$AAB?$AAu?$AAl?$AAk?$AAI?$AAn?$AAD?$AAi?$AAr?$AAe?$AAc?$AAt?$AAI?$AAp?$AAN?$AAo?$AAT?$AAl?$AAp?$AAT?$AAh?$AAr?$AAe@ 10020120     swiusb.obj
 0002:000091b0       ??_C@_1LE@DICKDNO@?$AAB?$AAu?$AAl?$AAk?$AAI?$AAn?$AAD?$AAi?$AAr?$AAe?$AAc?$AAt?$AAI?$AAp?$AAN?$AAo?$AAT?$AAl?$AAp?$AAT?$AAh?$AAr?$AAe?$AAa?$AAd?$AA?5?$AAf?$AAo?$AAr?$AAc?$AAe?$AAs@ 100201b0     swiusb.obj
 0002:00009268       ??_C@_1HE@OHPCMFMO@?$AAS?$AAw?$AAi?$AAG?$AAo?$AAb?$AAi?$AA?5?$AAB?$AAu?$AAl?$AAk?$AAi?$AAn?$AAD?$AAi?$AAr?$AAe?$AAc?$AAt?$AAI?$AAp?$AAN?$AAo?$AAT?$AAl?$AAp?$AAT?$AAh?$AAr?$AAe?$AAa@ 10020268     swiusb.obj
 0002:000092e0       ??_C@_1EO@LDEDCGHM@?$AAS?$AAw?$AAi?$AAG?$AAo?$AAb?$AAi?$AA?5?$AAB?$AAu?$AAl?$AAk?$AAI?$AAn?$AAD?$AAi?$AAr?$AAe?$AAc?$AAt?$AAI?$AAp?$AAN?$AAo?$AAT?$AAl?$AAp?$AAT?$AAh?$AAr?$AAe?$AAa@ 100202e0     swiusb.obj
 0002:00009330       ??_C@_1KO@KPHBGHNI@?$AA?$AN?$AA?6?$AAS?$AAw?$AAi?$AAG?$AAo?$AAb?$AAi?$AA?5?$AAB?$AAu?$AAl?$AAk?$AAI?$AAn?$AAD?$AAi?$AAr?$AAe?$AAc?$AAt?$AAI?$AAp?$AAN?$AAo?$AAT?$AAl?$AAp?$AAT?$AAh?$AAr@ 10020330     swiusb.obj
 0002:000093e0       ??_C@_1HO@HCKEPAKI@?$AAS?$AAw?$AAi?$AAG?$AAo?$AAb?$AAi?$AA?3?$AA?5?$AAB?$AAu?$AAl?$AAk?$AAO?$AAu?$AAt?$AAT?$AAh?$AAr?$AAe?$AAa?$AAd?$AA?5?$AAC?$AAh?$AAa?$AAn?$AAn?$AAe?$AAl?$AA?5?$AA?$CD@ 100203e0     swiusb.obj
 0002:00009460       ??_C@_1HE@IOALGNPD@?$AAS?$AAw?$AAi?$AAG?$AAo?$AAb?$AAi?$AA?3?$AA?5?$AAB?$AAu?$AAl?$AAk?$AAO?$AAu?$AAt?$AAT?$AAh?$AAr?$AAe?$AAa?$AAd?$AA?5?$AAC?$AAh?$AAa?$AAn?$AAn?$AAe?$AAl?$AA?5?$AA?$CD@ 10020460     swiusb.obj
 0002:000094d8       ??_C@_1HO@KEFHOHGH@?$AAS?$AAw?$AAi?$AAG?$AAo?$AAb?$AAi?$AA?5?$AAB?$AAu?$AAl?$AAk?$AAO?$AAu?$AAt?$AAT?$AAh?$AAr?$AAe?$AAa?$AAd?$AA?5?$AAe?$AAx?$AAi?$AAt?$AAs?$AA?5?$AAb?$AAe?$AAc?$AAa@ 100204d8     swiusb.obj
 0002:00009558       ??_C@_1NI@NOGOFFAF@?$AAS?$AAw?$AAi?$AAG?$AAo?$AAb?$AAi?$AA?5?$AAB?$AAu?$AAl?$AAk?$AAO?$AAu?$AAt?$AAT?$AAh?$AAr?$AAe?$AAa?$AAd?$AA?5?$AAw?$AAa?$AAi?$AAt?$AAs?$AA?5?$AAf?$AAo?$AAr?$AA?5@ 10020558     swiusb.obj
 0002:00009630       ??_C@_1IE@HEKDPAKD@?$AAS?$AAw?$AAi?$AAG?$AAo?$AAb?$AAi?$AA?3?$AA?5?$AAB?$AAu?$AAl?$AAk?$AAO?$AAu?$AAt?$AAD?$AAi?$AAr?$AAe?$AAc?$AAt?$AAI?$AAp?$AAT?$AAh?$AAr?$AAe?$AAa?$AAd?$AA?5?$AAC@ 10020630     swiusb.obj
 0002:000096b8       ??_C@_1IO@EMDIENLO@?$AAS?$AAw?$AAi?$AAG?$AAo?$AAb?$AAi?$AA?5?$AAB?$AAu?$AAl?$AAk?$AAO?$AAu?$AAt?$AAD?$AAi?$AAr?$AAe?$AAc?$AAt?$AAI?$AAp?$AAT?$AAh?$AAr?$AAe?$AAa?$AAd?$AA?5?$AAe?$AAx@ 100206b8     swiusb.obj
 0002:00009748       ??_C@_1OI@NAFKMDGO@?$AAS?$AAw?$AAi?$AAG?$AAo?$AAb?$AAi?$AA?5?$AAB?$AAu?$AAl?$AAk?$AAO?$AAu?$AAt?$AAD?$AAi?$AAr?$AAe?$AAc?$AAt?$AAI?$AAp?$AAT?$AAh?$AAr?$AAe?$AAa?$AAd?$AA?5?$AAw?$AAa@ 10020748     swiusb.obj
 0002:00009830       ??_C@_1GO@LHJOPKNM@?$AAS?$AAw?$AAi?$AAG?$AAo?$AAb?$AAi?$AA?3?$AA?5?$AAB?$AAu?$AAl?$AAk?$AAO?$AAu?$AAt?$AAD?$AAi?$AAr?$AAe?$AAc?$AAt?$AAI?$AAp?$AAT?$AAh?$AAr?$AAe?$AAa?$AAd?$AA?5?$AAs@ 10020830     swiusb.obj
 0002:000098a0       ??_C@_1HC@PBIJMCDO@?$AAS?$AAw?$AAi?$AAG?$AAo?$AAb?$AAi?$AA?3?$AA?5?$AAB?$AAu?$AAl?$AAk?$AAO?$AAu?$AAt?$AAD?$AAi?$AAr?$AAe?$AAc?$AAt?$AAI?$AAp?$AAT?$AAh?$AAr?$AAe?$AAa?$AAd?$AA?5?$AAs@ 100208a0     swiusb.obj
 0002:00009918       ??_C@_1GO@KNJMLDEM@?$AAS?$AAw?$AAi?$AAG?$AAo?$AAb?$AAi?$AA?3?$AA?5?$AAB?$AAu?$AAl?$AAk?$AAO?$AAu?$AAt?$AAD?$AAi?$AAr?$AAe?$AAc?$AAt?$AAI?$AAp?$AAT?$AAh?$AAr?$AAe?$AAa?$AAd?$AA?5?$AAs@ 10020918     swiusb.obj
 0002:00009988       ??_C@_1DO@PCGKFANH@?$AAS?$AAw?$AAi?$AAG?$AAo?$AAb?$AAi?$AA?5?$AAB?$AAu?$AAl?$AAk?$AAO?$AAu?$AAt?$AAD?$AAi?$AAr?$AAe?$AAc?$AAt?$AAI?$AAp?$AAT?$AAh?$AAr?$AAe?$AAa?$AAd?$AA?3?$AA?$AA@ 10020988     swiusb.obj
 0002:000099c8       ??_C@_1KO@BJMBOGEJ@?$AA?$CF?$AAs?$AA?5?$AAD?$AAa?$AAt?$AAa?$AA?5?$AAt?$AAr?$AAa?$AAn?$AAs?$AAf?$AAe?$AAr?$AA?5?$AAn?$AAo?$AAt?$AA?5?$AAa?$AAl?$AAl?$AAo?$AAw?$AAe?$AAd?$AA?5?$AAw?$AAh?$AAi@ 100209c8     swiusb.obj
 0002:00009a78       ??_C@_1GM@EHDLPKDI@?$AAS?$AAw?$AAi?$AAG?$AAo?$AAb?$AAi?$AA?5?$AAB?$AAu?$AAl?$AAk?$AAO?$AAu?$AAt?$AAD?$AAi?$AAr?$AAe?$AAc?$AAt?$AAI?$AAp?$AAT?$AAh?$AAr?$AAe?$AAa?$AAd?$AA?5?$AAe?$AAx@ 10020a78     swiusb.obj
 0002:00009ae8       ??_C@_1IE@BHFHBPPO@?$AAS?$AAw?$AAi?$AAG?$AAo?$AAb?$AAi?$AA?5?$AAP?$AAa?$AAr?$AAs?$AAe?$AAA?$AAn?$AAd?$AAA?$AAd?$AAd?$AAT?$AAo?$AAR?$AAe?$AAa?$AAd?$AAQ?$AAu?$AAe?$AAu?$AAe?$AA?5?$AAe@ 10020ae8     swiusb.obj
 0002:00009b70       ??_C@_1HE@BNGJKBAE@?$AA?6?$AAS?$AAw?$AAi?$AAG?$AAo?$AAb?$AAi?$AA?5?$AAB?$AAu?$AAl?$AAk?$AAI?$AAn?$AAT?$AAh?$AAr?$AAe?$AAa?$AAd?$AA?0?$AA?5?$AAC?$AAh?$AAa?$AAn?$AAn?$AAe?$AAl?$AA?5?$AA?$CD@ 10020b70     swiusb.obj
 0002:00009be8       ??_C@_1HO@GFMFAIL@?$AA?6?$AAS?$AAw?$AAi?$AAG?$AAo?$AAb?$AAi?$AA?5?$AAB?$AAu?$AAl?$AAk?$AAI?$AAn?$AAT?$AAh?$AAr?$AAe?$AAa?$AAd?$AA?0?$AA?5?$AAC?$AAh?$AAa?$AAn?$AAn?$AAe?$AAl?$AA?5?$AA?$CD@ 10020be8     swiusb.obj
 0002:00009c68       ??_C@_1IK@CBIGLABM@?$AA?$CF?$AAs?$AA?3?$AA?5?$AAi?$AAs?$AAC?$AAl?$AAe?$AAa?$AAr?$AAP?$AAo?$AAr?$AAt?$AAS?$AAu?$AAs?$AAp?$AAe?$AAn?$AAd?$AAe?$AAd?$AA?5?$AA?$DN?$AA?5?$AAT?$AAR?$AAU?$AAE?$AA?0@ 10020c68     swiusb.obj
 0002:00009cf8       ??_C@_1IG@PDJNDNEG@?$AA?$CF?$AAs?$AA?5?$AAf?$AAo?$AAr?$AAc?$AAe?$AAs?$AA?5?$AAi?$AAs?$AAP?$AAo?$AAr?$AAt?$AAS?$AAu?$AAs?$AAp?$AAe?$AAn?$AAd?$AAe?$AAd?$AA?5?$AA?$DN?$AA?5?$AAF?$AAA?$AAL?$AAS@ 10020cf8     swiusb.obj
 0002:00009d80       ??_C@_1GA@DFFBMFFK@?$AA?$CF?$AAs?$AA?3?$AAW?$AAa?$AAi?$AAt?$AAi?$AAn?$AAg?$AA?5?$AAf?$AAo?$AAr?$AA?5?$AAd?$AAe?$AAv?$AAi?$AAc?$AAe?$AAr?$AAe?$AAs?$AAu?$AAm?$AAe?$AAd?$AA?9?$AA?$DO?$AA?5?$AAU@ 10020d80     swiusb.obj
 0002:00009de0       ??_C@_1HK@PNFPFNEB@?$AAS?$AAw?$AAi?$AAG?$AAo?$AAb?$AAi?$AA?5?$AAp?$AAC?$AAo?$AAm?$AAm?$AAp?$AAo?$AAr?$AAt?$AAM?$AAd?$AAd?$AA?5?$AAi?$AAs?$AA?5?$AAN?$AAU?$AAL?$AAL?$AA?5?$AAf?$AAo?$AAr@ 10020de0     swiusb.obj
 0002:00009e60       ??_C@_1JE@JDCHBNDD@?$AA?$AN?$AA?6?$AAS?$AAw?$AAi?$AAG?$AAo?$AAb?$AAi?$AA?5?$AAB?$AAu?$AAl?$AAk?$AAI?$AAn?$AAT?$AAh?$AAr?$AAe?$AAa?$AAd?$AA?0?$AA?5?$AAC?$AAh?$AAa?$AAn?$AAn?$AAe?$AAl?$AA?5@ 10020e60     swiusb.obj
 0002:00009ef8       ??_C@_1IE@EINCOBJP@?$AA?6?$AAS?$AAw?$AAi?$AAG?$AAo?$AAb?$AAi?$AA?5?$AAB?$AAu?$AAl?$AAk?$AAI?$AAn?$AAD?$AAi?$AAr?$AAe?$AAc?$AAt?$AAI?$AAp?$AAT?$AAh?$AAr?$AAe?$AAa?$AAd?$AA?0?$AA?5?$AAC@ 10020ef8     swiusb.obj
 0002:00009f80       ??_C@_1IO@BLPECMHD@?$AA?6?$AAS?$AAw?$AAi?$AAG?$AAo?$AAb?$AAi?$AA?5?$AAB?$AAu?$AAl?$AAk?$AAI?$AAn?$AAD?$AAi?$AAr?$AAe?$AAc?$AAt?$AAI?$AAp?$AAT?$AAh?$AAr?$AAe?$AAa?$AAd?$AA?0?$AA?5?$AAC@ 10020f80     swiusb.obj
 0002:0000a010       ??_C@_1KK@EHGMBIJE@?$AAB?$AAu?$AAl?$AAk?$AAI?$AAn?$AAD?$AAi?$AAr?$AAe?$AAc?$AAt?$AAI?$AAp?$AAT?$AAh?$AAr?$AAe?$AAa?$AAd?$AA?5?$AAf?$AAo?$AAr?$AAc?$AAe?$AAs?$AA?5?$AAi?$AAs?$AAP?$AAo@ 10021010     swiusb.obj
 0002:0000a0c0       ??_C@_1GK@GNMIBBIH@?$AAS?$AAw?$AAi?$AAG?$AAo?$AAb?$AAi?$AA?5?$AAB?$AAu?$AAl?$AAk?$AAi?$AAn?$AAD?$AAi?$AAr?$AAe?$AAc?$AAt?$AAI?$AAp?$AAT?$AAh?$AAr?$AAe?$AAa?$AAd?$AA?5?$AAe?$AAx?$AAi@ 100210c0     swiusb.obj
 0002:0000a130       ??_C@_1KE@FGBLFEFC@?$AA?$AN?$AA?6?$AAS?$AAw?$AAi?$AAG?$AAo?$AAb?$AAi?$AA?5?$AAB?$AAu?$AAl?$AAk?$AAI?$AAn?$AAD?$AAi?$AAr?$AAe?$AAc?$AAt?$AAI?$AAp?$AAT?$AAh?$AAr?$AAe?$AAa?$AAd?$AA?0?$AA?5@ 10021130     swiusb.obj
 0002:0000a1d8       ??_C@_1IE@PMMAAOCO@?$AAS?$AAw?$AAi?$AAG?$AAo?$AAb?$AAi?$AA?3?$AA?5?$AAB?$AAu?$AAl?$AAk?$AAO?$AAu?$AAt?$AAM?$AAi?$AAn?$AAi?$AAp?$AAo?$AAr?$AAt?$AAT?$AAh?$AAr?$AAe?$AAa?$AAd?$AA?5?$AAC@ 100211d8     swiusb.obj
 0002:0000a260       ??_C@_1BAO@OIDHLMJK@?$AAS?$AAw?$AAi?$AAG?$AAo?$AAb?$AAi?$AA?5?$AAB?$AAu?$AAl?$AAk?$AAO?$AAu?$AAt?$AAM?$AAi?$AAn?$AAi?$AAp?$AAo?$AAr?$AAt?$AAT?$AAh?$AAr?$AAe?$AAa?$AAd?$AA?5?$AAw?$AAa@ 10021260     swiusb.obj
 0002:0000a370       ??_C@_1IO@IOLIHCPO@?$AAS?$AAw?$AAi?$AAG?$AAo?$AAb?$AAi?$AA?5?$AAB?$AAu?$AAl?$AAk?$AAO?$AAu?$AAt?$AAM?$AAi?$AAn?$AAi?$AAp?$AAo?$AAr?$AAt?$AAT?$AAh?$AAr?$AAe?$AAa?$AAd?$AA?5?$AAe?$AAx@ 10021370     swiusb.obj
 0002:0000a400       ??_C@_1FO@CMLNHBDG@?$AAS?$AAw?$AAi?$AAG?$AAo?$AAb?$AAi?$AA?3?$AA?5?$AAR?$AAe?$AAc?$AAe?$AAi?$AAv?$AAe?$AAd?$AA?5?$AAA?$AAR?$AAP?$AA?5?$AAs?$AAe?$AAn?$AAd?$AAe?$AAr?$AA?5?$AAI?$AAP?$AA?3@ 10021400     swiusb.obj
 0002:0000a460       ??_C@_1FO@CGKKLCIG@?$AAS?$AAw?$AAi?$AAG?$AAo?$AAb?$AAi?$AA?3?$AA?5?$AAR?$AAe?$AAc?$AAe?$AAi?$AAv?$AAe?$AAd?$AA?5?$AAA?$AAR?$AAP?$AA?5?$AAt?$AAa?$AAr?$AAg?$AAe?$AAt?$AA?5?$AAI?$AAP?$AA?3@ 10021460     swiusb.obj
 0002:0000a4c0       ??_C@_1FA@BLDDPAA@?$AAS?$AAw?$AAi?$AAG?$AAo?$AAb?$AAi?$AA?3?$AA?5?$AAa?$AAf?$AAt?$AAe?$AAr?$AA?5?$AAP?$AAa?$AAr?$AAs?$AAe?$AAA?$AAn?$AAd?$AAA?$AAd?$AAd?$AAT?$AAo?$AAR?$AAe?$AAa?$AAd@ 100214c0     swiusb.obj
 0002:0000a510       ??_C@_1GA@GMKJJGN@?$AAS?$AAw?$AAi?$AAG?$AAo?$AAb?$AAi?$AA?5?$AAB?$AAu?$AAl?$AAk?$AAO?$AAu?$AAt?$AAM?$AAi?$AAn?$AAi?$AAp?$AAo?$AAr?$AAt?$AAT?$AAh?$AAr?$AAe?$AAa?$AAd?$AA?3?$AA?5?$AAU@ 10021510     swiusb.obj
 0002:0000a570       ??_C@_1EK@KEBEGGLA@?$AAS?$AAw?$AAi?$AAG?$AAo?$AAb?$AAi?$AA?5?$AA?9?$AAI?$AAn?$AAi?$AAt?$AAi?$AAa?$AAl?$AAi?$AAz?$AAe?$AAD?$AAi?$AAr?$AAe?$AAc?$AAt?$AAI?$AAp?$AAC?$AAh?$AAa?$AAn?$AAn@ 10021570     swiusb.obj
 0002:0000a5c0       ??_C@_1GM@BLHCGCCK@?$AA?$CF?$AAs?$AA?5?$AAC?$AAh?$AAa?$AAn?$AAn?$AAe?$AAl?$AA?5?$AA?$CF?$AAd?$AA?5?$AAb?$AAu?$AAl?$AAk?$AAo?$AAu?$AAt?$AA?5?$AAt?$AAh?$AAr?$AAe?$AAa?$AAd?$AA?5?$AAp?$AAr?$AAi@ 100215c0     swiusb.obj
 0002:0000a630       ??_C@_1HK@LPAAAIIA@?$AA?$CF?$AAs?$AA?5?$AAF?$AAa?$AAi?$AAl?$AAe?$AAd?$AA?5?$AAt?$AAo?$AA?5?$AAs?$AAe?$AAt?$AA?5?$AAc?$AAh?$AAa?$AAn?$AAn?$AAe?$AAl?$AA?5?$AA?$CF?$AAd?$AA?5?$AAb?$AAu?$AAl?$AAk@ 10021630     swiusb.obj
 0002:0000a6ac       ??_C@_1CE@NHOFNKJK@?$AAO?$AAu?$AAt?$AAT?$AAh?$AAr?$AAe?$AAa?$AAd?$AAP?$AAr?$AAi?$AAo?$AAr?$AAi?$AAt?$AAy?$AA?$AA@ 100216ac     swiusb.obj
 0002:0000a6d0       ??_C@_1GK@JCANNBJJ@?$AA?$CF?$AAs?$AA?5?$AAC?$AAh?$AAa?$AAn?$AAn?$AAe?$AAl?$AA?5?$AA?$CF?$AAd?$AA?5?$AAb?$AAu?$AAl?$AAk?$AAi?$AAn?$AA?5?$AAt?$AAh?$AAr?$AAe?$AAa?$AAd?$AA?5?$AAp?$AAr?$AAi?$AAo@ 100216d0     swiusb.obj
 0002:0000a740       ??_C@_1EG@JNDFIOCA@?$AAS?$AAw?$AAi?$AAG?$AAo?$AAb?$AAi?$AA?5?$AAI?$AAn?$AAi?$AAt?$AAi?$AAa?$AAl?$AAi?$AAz?$AAe?$AAD?$AAi?$AAr?$AAe?$AAc?$AAt?$AAI?$AAp?$AAC?$AAh?$AAa?$AAn?$AAn?$AAe@ 10021740     swiusb.obj
 0002:0000a788       ??_C@_1HI@IBJIPFDF@?$AA?$CF?$AAs?$AA?5?$AAF?$AAa?$AAi?$AAl?$AAe?$AAd?$AA?5?$AAt?$AAo?$AA?5?$AAs?$AAe?$AAt?$AA?5?$AAc?$AAh?$AAa?$AAn?$AAn?$AAe?$AAl?$AA?5?$AA?$CF?$AAd?$AA?5?$AAb?$AAu?$AAl?$AAk@ 10021788     swiusb.obj
 0002:0000a800       ??_C@_1CC@CGONKFLE@?$AAI?$AAn?$AAT?$AAh?$AAr?$AAe?$AAa?$AAd?$AAP?$AAr?$AAi?$AAo?$AAr?$AAi?$AAt?$AAy?$AA?$AA@ 10021800     swiusb.obj
 0002:0000a824       ??_C@_1DA@BDKGJBLB@?$AAC?$AAl?$AAe?$AAa?$AAr?$AAi?$AAn?$AAg?$AA?5?$AAN?$AAD?$AAI?$AAS?$AA?5?$AAI?$AAN?$AAT?$AA?5?$AAE?$AAP?$AA?5?$AA?$CF?$AAx?$AA?$AA@ 10021824     swiusb.obj
 0002:0000a854       ??_C@_1DA@EEPBCDBC@?$AAC?$AAl?$AAe?$AAa?$AAr?$AAi?$AAn?$AAg?$AA?5?$AAN?$AAD?$AAI?$AAS?$AA?5?$AAO?$AAU?$AAT?$AA?5?$AAE?$AAP?$AA?5?$AA?$CF?$AAx?$AA?$AA@ 10021854     swiusb.obj
 0002:0000a884       ??_C@_1CO@BDIMNLLJ@?$AAC?$AAl?$AAe?$AAa?$AAr?$AAi?$AAn?$AAg?$AA?5?$AAN?$AAD?$AAI?$AAS?$AA?5?$AAI?$AAN?$AA?5?$AAE?$AAP?$AA?5?$AA?$CF?$AAx?$AA?$AA@ 10021884     swiusb.obj
 0002:0000a8b4       ??_C@_1CE@FNPDALLB@?$AAC?$AAl?$AAe?$AAa?$AAr?$AAI?$AAn?$AAt?$AAE?$AAP?$AAF?$AAe?$AAa?$AAt?$AAu?$AAr?$AAe?$AA?$AA@ 100218b4     swiusb.obj
 0002:0000a8d8       ??_C@_1CE@JHFFDMKL@?$AAC?$AAl?$AAe?$AAa?$AAr?$AAO?$AAu?$AAt?$AAE?$AAP?$AAF?$AAe?$AAa?$AAt?$AAu?$AAr?$AAe?$AA?$AA@ 100218d8     swiusb.obj
 0002:0000a8fc       ??_C@_1M@PIGKLJLL@?$AA?$CF?$AAs?$AA?2?$AA?$CF?$AAd?$AA?$AA@ 100218fc     swiusb.obj
 0002:0000a908       ??_C@_1BC@IDPNFFME@?$AAF?$AAu?$AAn?$AAc?$AAt?$AAi?$AAo?$AAn?$AA?$AA@ 10021908     swiusb.obj
 0002:0000a91c       ??_C@_1CC@ODKMAMBP@?$AAC?$AAl?$AAe?$AAa?$AAr?$AAI?$AAn?$AAE?$AAP?$AAF?$AAe?$AAa?$AAt?$AAu?$AAr?$AAe?$AA?$AA@ 1002191c     swiusb.obj
 0002:0000a940       ??_C@_1EK@MBPHEBJL@?$AAS?$AAw?$AAi?$AAG?$AAo?$AAb?$AAi?$AA?5?$AA?$CL?$AAI?$AAn?$AAi?$AAt?$AAi?$AAa?$AAl?$AAi?$AAz?$AAe?$AAD?$AAi?$AAr?$AAe?$AAc?$AAt?$AAI?$AAp?$AAC?$AAh?$AAa?$AAn?$AAn@ 10021940     swiusb.obj
 0002:0000a990       ??_C@_1IO@OPKCELBJ@?$AAS?$AAw?$AAi?$AAG?$AAo?$AAb?$AAi?$AA?5?$AAU?$AAS?$AAB?$AAD?$AAe?$AAv?$AAi?$AAc?$AAe?$AAA?$AAt?$AAt?$AAa?$AAc?$AAh?$AA?3?$AA?5?$AAF?$AAa?$AAi?$AAl?$AAe?$AAd?$AA?5@ 10021990     swiusb.obj
 0002:0000aa20       ??_C@_1EI@PAEMMKEO@?$AAS?$AAw?$AAi?$AAG?$AAo?$AAb?$AAi?$AA?5?$AAU?$AAS?$AAB?$AAD?$AAe?$AAv?$AAi?$AAc?$AAe?$AAA?$AAt?$AAt?$AAa?$AAc?$AAh?$AA?3?$AA?5?$AAD?$AAo?$AAn?$AAe?$AA?0?$AA?5?$AA?$CF@ 10021a20     swiusb.obj
 0002:0000aa68       ??_C@_1KG@IEGLHPEA@?$AAS?$AAw?$AAi?$AAG?$AAo?$AAb?$AAi?$AA?5?$AAU?$AAS?$AAB?$AAD?$AAe?$AAv?$AAi?$AAc?$AAe?$AAA?$AAt?$AAt?$AAa?$AAc?$AAh?$AA?3?$AA?5?$AAF?$AAa?$AAi?$AAl?$AAe?$AAd?$AA?5@ 10021a68     swiusb.obj
 0002:0000ab10       ??_C@_1IO@JOHFGI@?$AAS?$AAw?$AAi?$AAG?$AAo?$AAb?$AAi?$AA?5?$AAU?$AAS?$AAB?$AAD?$AAe?$AAv?$AAi?$AAc?$AAe?$AAA?$AAt?$AAt?$AAa?$AAc?$AAh?$AA?3?$AA?5?$AAS?$AAe?$AAt?$AA?5?$AAd?$AAe?$AAv@ 10021b10     swiusb.obj
 0002:0000aba0       ??_C@_1JA@CAIGNFJA@?$AAS?$AAw?$AAi?$AAG?$AAo?$AAb?$AAi?$AA?5?$AAU?$AAS?$AAB?$AAD?$AAe?$AAv?$AAi?$AAc?$AAe?$AAA?$AAt?$AAt?$AAa?$AAc?$AAh?$AA?3?$AA?5?$AAF?$AAa?$AAi?$AAl?$AAe?$AAd?$AA?5@ 10021ba0     swiusb.obj
 0002:0000ac30       ??_C@_1CM@BKFKHOOJ@?$AAS?$AAw?$AAi?$AAU?$AAs?$AAb?$AAH?$AAa?$AAr?$AAd?$AAw?$AAa?$AAr?$AAe?$AAP?$AAr?$AAe?$AAs?$AAe?$AAn?$AAt?$AA?$AA@ 10021c30     swiusb.obj
 0002:0000ac5c       ??_C@_1CK@LGACNNLK@?$AAS?$AAw?$AAi?$AAU?$AAs?$AAb?$AAH?$AAa?$AAr?$AAd?$AAw?$AAa?$AAr?$AAe?$AAA?$AAb?$AAs?$AAe?$AAn?$AAt?$AA?$AA@ 10021c5c     swiusb.obj
 0002:0000ac88       ??_C@_1CI@PBANIAGA@?$AAV?$AAI?$AAD?$AA_?$AA?$CF?$AA4?$AA?4?$AA4?$AAX?$AA?$CG?$AAP?$AAI?$AAD?$AA_?$AA?$CF?$AA4?$AA?4?$AA4?$AAX?$AA?$AA@ 10021c88     swiusb.obj
 0002:0000acb0       ??_C@_1IE@OBOFFEGH@?$AAS?$AAw?$AAi?$AAG?$AAo?$AAb?$AAi?$AA?5?$AAU?$AAS?$AAB?$AAD?$AAe?$AAv?$AAi?$AAc?$AAe?$AAA?$AAt?$AAt?$AAa?$AAc?$AAh?$AA?3?$AA?5?$AAN?$AAd?$AAi?$AAs?$AAR?$AAe?$AAg@ 10021cb0     swiusb.obj
 0002:0000ad38       ??_C@_1HE@NAABIMPE@?$AAS?$AAw?$AAi?$AAG?$AAo?$AAb?$AAi?$AA?5?$AAU?$AAS?$AAB?$AAD?$AAe?$AAv?$AAi?$AAc?$AAe?$AAA?$AAt?$AAt?$AAa?$AAc?$AAh?$AA?3?$AA?5?$AAN?$AAD?$AAI?$AAS?$AA?5?$AAc?$AAo@ 10021d38     swiusb.obj
 0002:0000adac       ??_C@_1BM@CHMOLOMB@?$AAS?$AAW?$AAG?$AAo?$AAb?$AAi?$AAU?$AAS?$AAB?$AAN?$AAD?$AAI?$AAS?$AA?$AA@ 10021dac     swiusb.obj
 0002:0000adc8       ??_C@_1KK@DINCFEAI@?$AAS?$AAw?$AAi?$AAG?$AAo?$AAb?$AAi?$AA?5?$AAU?$AAS?$AAB?$AAD?$AAe?$AAv?$AAi?$AAc?$AAe?$AAA?$AAt?$AAt?$AAa?$AAc?$AAh?$AA?3?$AA?5?$AAG?$AAo?$AAt?$AA?5?$AAQ?$AAM?$AAI@ 10021dc8     swiusb.obj
 0002:0000ae78       ??_C@_1JI@DIIFAAIM@?$AAS?$AAw?$AAi?$AAG?$AAo?$AAb?$AAi?$AA?5?$AAU?$AAS?$AAB?$AAD?$AAe?$AAv?$AAi?$AAc?$AAe?$AAA?$AAt?$AAt?$AAa?$AAc?$AAh?$AA?3?$AA?5?$AAF?$AAa?$AAi?$AAl?$AAe?$AAd?$AA?5@ 10021e78     swiusb.obj
 0002:0000af10       ??_C@_17FGILNNML@?$AAQ?$AAM?$AAI?$AA?$AA@ 10021f10     swiusb.obj
 0002:0000af18       ??_C@_1DC@DNGEGCKJ@?$AAE?$AAn?$AAa?$AAb?$AAl?$AAi?$AAn?$AAg?$AA?5?$AAd?$AAa?$AAt?$AAa?$AA?5?$AAb?$AAu?$AAn?$AAd?$AAl?$AAe?$AA?5?$AA1?$AA?$AN?$AA?6?$AA?$AA@ 10021f18     swiusb.obj
 0002:0000af50       ??_C@_1EE@DBLEDIGP@?$AAE?$AAn?$AAa?$AAb?$AAl?$AAi?$AAn?$AAg?$AA?5?$AAd?$AAe?$AAv?$AAi?$AAc?$AAe?$AA?5?$AAr?$AAe?$AAm?$AAo?$AAt?$AAe?$AA?5?$AAw?$AAa?$AAk?$AAe?$AAu?$AAp?$AA?5?$AA0?$AA?$AN@ 10021f50     swiusb.obj
 0002:0000af98       ??_C@_1KG@FEDDAAAA@?$AAS?$AAw?$AAi?$AAG?$AAo?$AAb?$AAi?$AA?5?$AAU?$AAS?$AAB?$AAD?$AAe?$AAv?$AAi?$AAc?$AAe?$AAA?$AAt?$AAt?$AAa?$AAc?$AAh?$AA?3?$AA?5?$AAg?$AAU?$AAs?$AAe?$AAN?$AAd?$AAi@ 10021f98     swiusb.obj
 0002:0000b040       ??_C@_1DC@KHBCLBPJ@?$AAS?$AAw?$AAi?$AAG?$AAo?$AAb?$AAi?$AA?5?$AAU?$AAS?$AAB?$AAD?$AAe?$AAv?$AAi?$AAc?$AAe?$AAA?$AAt?$AAt?$AAa?$AAc?$AAh?$AA?3?$AA?$AA@ 10022040     swiusb.obj
 0002:0000b078       ??_C@_1GK@EECPFCLJ@?$AAS?$AAw?$AAi?$AAG?$AAo?$AAb?$AAi?$AA?3?$AA?5?$AAE?$AAr?$AAr?$AAo?$AAr?$AA?5?$AA?$CF?$AA0?$AA8?$AAx?$AA?5?$AAI?$AAn?$AA?5?$AAA?$AAc?$AAt?$AAi?$AAv?$AAi?$AAt?$AAy?$AAT@ 10022078     swiusb.obj
 0002:0000b0e8       ??_C@_1JK@ILMHAPK@?$AAS?$AAw?$AAi?$AAG?$AAo?$AAb?$AAi?$AA?5?$AAU?$AAS?$AAB?$AAD?$AAe?$AAv?$AAi?$AAc?$AAe?$AAA?$AAt?$AAt?$AAa?$AAc?$AAh?$AA?3?$AA?5?$AAg?$AAd?$AAw?$AAI?$AAd?$AAl?$AAe@ 100220e8     swiusb.obj
 0002:0000b188       ??_C@_1GA@JOEBFIJB@?$AAS?$AAw?$AAi?$AAG?$AAo?$AAb?$AAi?$AA?5?$AAU?$AAs?$AAi?$AAn?$AAg?$AA?5?$AAD?$AAe?$AAf?$AAa?$AAu?$AAl?$AAt?$AA?5?$AAg?$AAd?$AAw?$AAR?$AAe?$AAs?$AAu?$AAm?$AAe?$AAD@ 10022188     swiusb.obj
 0002:0000b1e8       ??_C@_1CK@LNODLPNH@?$AAR?$AAe?$AAs?$AAu?$AAm?$AAe?$AAD?$AAe?$AAt?$AAe?$AAc?$AAt?$AAI?$AAn?$AAt?$AAe?$AAr?$AAv?$AAa?$AAl?$AA?$AA@ 100221e8     swiusb.obj
 0002:0000b214       ??_C@_1CI@CLLEFEHP@?$AAD?$AAe?$AAf?$AAa?$AAu?$AAl?$AAt?$AAT?$AAr?$AAa?$AAn?$AAs?$AAf?$AAe?$AAr?$AAS?$AAi?$AAz?$AAe?$AA?$AA@ 10022214     swiusb.obj
 0002:0000b23c       ??_C@_1BM@PGFIDDDJ@?$AAS?$AAa?$AAv?$AAe?$AAP?$AAo?$AAw?$AAe?$AAr?$AAI?$AAn?$AAD?$AA2?$AA?$AA@ 1002223c     swiusb.obj
 0002:0000b258       ??_C@_1BI@MBBAJPEA@?$AAI?$AAd?$AAl?$AAe?$AAT?$AAi?$AAm?$AAe?$AAo?$AAu?$AAt?$AA?$AA@ 10022258     swiusb.obj
 0002:0000b270       ??_C@_1HO@FOFGLGND@?$AAS?$AAw?$AAi?$AAG?$AAo?$AAb?$AAi?$AA?5?$AAU?$AAS?$AAB?$AAD?$AAe?$AAv?$AAi?$AAc?$AAe?$AAA?$AAt?$AAt?$AAa?$AAc?$AAh?$AA?3?$AA?5?$AAD?$AAo?$AAn?$AAe?$AA?5?$AAs?$AAc@ 10022270     swiusb.obj
 0002:0000b2f0       ??_C@_1IO@MKLFMMKN@?$AAS?$AAw?$AAi?$AAG?$AAo?$AAb?$AAi?$AA?5?$AAU?$AAS?$AAB?$AAD?$AAe?$AAv?$AAi?$AAc?$AAe?$AAA?$AAt?$AAt?$AAa?$AAc?$AAh?$AA?3?$AA?5?$AAF?$AAa?$AAi?$AAl?$AAe?$AAd?$AA?5@ 100222f0     swiusb.obj
 0002:0000b380       ??_C@_1HI@LNPLICGP@?$AAS?$AAw?$AAi?$AAG?$AAo?$AAb?$AAi?$AA?5?$AAU?$AAS?$AAB?$AAD?$AAe?$AAv?$AAi?$AAc?$AAe?$AAA?$AAt?$AAt?$AAa?$AAc?$AAh?$AA?3?$AA?5?$AAD?$AAo?$AAn?$AAe?$AA?5?$AAs?$AAe@ 10022380     swiusb.obj
 0002:0000b3f8       ??_C@_1MI@CIBDKBDN@?$AAS?$AAw?$AAi?$AAG?$AAo?$AAb?$AAi?$AA?5?$AAU?$AAS?$AAB?$AAD?$AAe?$AAv?$AAi?$AAc?$AAe?$AAA?$AAt?$AAt?$AAa?$AAc?$AAh?$AA?3?$AA?5?$AAA?$AAc?$AAt?$AAi?$AAv?$AAa?$AAt@ 100223f8     swiusb.obj
 0002:0000b4c0       ??_C@_1BK@BFIEKNFP@?$AAF?$AAr?$AAi?$AAe?$AAn?$AAd?$AAl?$AAy?$AAN?$AAa?$AAm?$AAe?$AA?$AA@ 100224c0     swiusb.obj
 0002:0000b4e0       ??_C@_1GC@CPANMJOO@?$AAS?$AAw?$AAi?$AAG?$AAo?$AAb?$AAi?$AA?5?$AAU?$AAS?$AAB?$AAD?$AAe?$AAv?$AAi?$AAc?$AAe?$AAA?$AAt?$AAt?$AAa?$AAc?$AAh?$AA?3?$AA?5?$AA?$CF?$AAs?$AA?5?$AAc?$AAh?$AAa?$AAn@ 100224e0     swiusb.obj
 0002:0000b544       ??_C@_1BC@IALNFLAF@?$AAU?$AAn?$AAi?$AAm?$AAo?$AAd?$AAe?$AAm?$AA?$AA@ 10022544     swiusb.obj
 0002:0000b558       ??_C@_1BK@BIHJIGMO@?$AAR?$AAI?$AAL?$AA?2?$AAC?$AAD?$AAM?$AAA?$AAD?$AAa?$AAt?$AAa?$AA?$AA@ 10022558     swiusb.obj
 0002:0000b578       ??_C@_1IE@KLBBDPOH@?$AAS?$AAw?$AAi?$AAG?$AAo?$AAb?$AAi?$AA?5?$AAU?$AAS?$AAB?$AAD?$AAe?$AAv?$AAi?$AAc?$AAe?$AAA?$AAt?$AAt?$AAa?$AAc?$AAh?$AA?3?$AA?5?$AAA?$AAc?$AAt?$AAi?$AAv?$AAa?$AAt@ 10022578     swiusb.obj
 0002:0000b5fc       ??_C@_1M@NLGBAKO@?$AAA?$AAT?$AAP?$AAP?$AAP?$AA?$AA@ 100225fc     swiusb.obj
 0002:0000b608       ??_C@_1GC@MPMCDCAH@?$AAS?$AAw?$AAi?$AAG?$AAo?$AAb?$AAi?$AA?5?$AAU?$AAS?$AAB?$AAD?$AAe?$AAv?$AAi?$AAc?$AAe?$AAA?$AAt?$AAt?$AAa?$AAc?$AAh?$AA?3?$AA?5?$AAs?$AAk?$AAi?$AAp?$AAp?$AAi?$AAn@ 10022608     swiusb.obj
 0002:0000b66c       ??_C@_1O@ELHCGDOL@?$AAS?$AAW?$AAG?$AAo?$AAb?$AAi?$AA?$AA@ 1002266c     swiusb.obj
 0002:0000b67c       ??_C@_1BA@HEBNFGMC@?$AA?$CF?$AAs?$AA?2?$AA?$CF?$AAs?$AA?$CF?$AAs?$AA?$AA@ 1002267c     swiusb.obj
 0002:0000b690       ??_C@_1IK@ENDPALKN@?$AAS?$AAw?$AAi?$AAG?$AAo?$AAb?$AAi?$AA?5?$AAU?$AAS?$AAB?$AAD?$AAe?$AAv?$AAi?$AAc?$AAe?$AAA?$AAt?$AAt?$AAa?$AAc?$AAh?$AA?3?$AA?5?$AAF?$AAa?$AAi?$AAl?$AAe?$AAd?$AA?5@ 10022690     swiusb.obj
 0002:0000b71c       ??_C@_1BM@OCMDIFOI@?$AAS?$AAe?$AAt?$AAL?$AAi?$AAn?$AAe?$AAC?$AAo?$AAd?$AAi?$AAn?$AAg?$AA?$AA@ 1002271c     swiusb.obj
 0002:0000b738       ??_C@_1JG@DDINGIBN@?$AAS?$AAw?$AAi?$AAG?$AAo?$AAb?$AAi?$AA?5?$AAU?$AAS?$AAB?$AAD?$AAe?$AAv?$AAi?$AAc?$AAe?$AAA?$AAt?$AAt?$AAa?$AAc?$AAh?$AA?3?$AA?5?$AAF?$AAa?$AAi?$AAl?$AAe?$AAd?$AA?5@ 10022738     swiusb.obj
 0002:0000b7d0       ??_C@_1CI@NGOHLIOM@?$AAS?$AAe?$AAt?$AAC?$AAo?$AAn?$AAt?$AAr?$AAo?$AAl?$AAL?$AAi?$AAn?$AAe?$AAS?$AAt?$AAa?$AAt?$AAe?$AA?$AA@ 100227d0     swiusb.obj
 0002:0000b7f8       ??_C@_1CG@GOFLMGIA@?$AAC?$AAl?$AAe?$AAa?$AAr?$AAi?$AAn?$AAg?$AA?5?$AAI?$AAN?$AAT?$AA?5?$AAE?$AAP?$AA?5?$AA?$CF?$AAx?$AA?$AA@ 100227f8     swiusb.obj
 0002:0000b820       ??_C@_1CG@DJAMHECD@?$AAC?$AAl?$AAe?$AAa?$AAr?$AAi?$AAn?$AAg?$AA?5?$AAO?$AAU?$AAT?$AA?5?$AAE?$AAP?$AA?5?$AA?$CF?$AAx?$AA?$AA@ 10022820     swiusb.obj
 0002:0000b848       ??_C@_1CE@NFDBDHKH@?$AAC?$AAl?$AAe?$AAa?$AAr?$AAi?$AAn?$AAg?$AA?5?$AAI?$AAN?$AA?5?$AAE?$AAP?$AA?5?$AA?$CF?$AAx?$AA?$AA@ 10022848     swiusb.obj
 0002:0000b870       ??_C@_1KC@CPIGEKIA@?$AAS?$AAw?$AAi?$AAG?$AAo?$AAb?$AAi?$AA?5?$AAU?$AAS?$AAB?$AAD?$AAe?$AAv?$AAi?$AAc?$AAe?$AAA?$AAt?$AAt?$AAa?$AAc?$AAh?$AA?3?$AA?5?$AAF?$AAa?$AAi?$AAl?$AAe?$AAd?$AA?5@ 10022870     swiusb.obj
 0002:0000b914       ??_C@_1BI@GMNOMLIK@?$AAU?$AAN?$AAS?$AAU?$AAP?$AAP?$AAO?$AAR?$AAT?$AAE?$AAD?$AA?$AA@ 10022914     swiusb.obj
 0002:0000b92c       ??_C@_1DA@FPCNAFLN@?$AAE?$AAn?$AAd?$AAp?$AAo?$AAi?$AAn?$AAt?$AA?5?$AA?$CF?$AAx?$AA?5?$AAi?$AAn?$AAt?$AAe?$AAr?$AAr?$AAu?$AAp?$AAt?$AA?$AN?$AA?6?$AA?$AA@ 1002292c     swiusb.obj
 0002:0000b95c       ??_C@_1CO@FPHPHJHI@?$AAE?$AAn?$AAd?$AAp?$AAo?$AAi?$AAn?$AAt?$AA?5?$AA?$CF?$AAx?$AA?5?$AAb?$AAu?$AAl?$AAk?$AA?5?$AAo?$AAu?$AAt?$AA?$AN?$AA?6?$AA?$AA@ 1002295c     swiusb.obj
 0002:0000b98c       ??_C@_1CM@PMPAEAIL@?$AAE?$AAn?$AAd?$AAp?$AAo?$AAi?$AAn?$AAt?$AA?5?$AA?$CF?$AAx?$AA?5?$AAb?$AAu?$AAl?$AAk?$AA?5?$AAi?$AAn?$AA?$AN?$AA?6?$AA?$AA@ 1002298c     swiusb.obj
 0002:0000b9b8       ??_C@_1IE@FDPNDEHI@?$AAS?$AAw?$AAi?$AAG?$AAo?$AAb?$AAi?$AA?5?$AAU?$AAS?$AAB?$AAD?$AAe?$AAv?$AAi?$AAc?$AAe?$AAA?$AAt?$AAt?$AAa?$AAc?$AAh?$AA?3?$AA?5?$AAF?$AAa?$AAi?$AAl?$AAe?$AAd?$AA?5@ 100229b8     swiusb.obj
 0002:0000ba40       ??_C@_1HE@MOFOHOLE@?$AAS?$AAw?$AAi?$AAG?$AAo?$AAb?$AAi?$AA?5?$AAU?$AAS?$AAB?$AAD?$AAe?$AAv?$AAi?$AAc?$AAe?$AAA?$AAt?$AAt?$AAa?$AAc?$AAh?$AA?3?$AA?5?$AAi?$AAn?$AAi?$AAt?$AAi?$AAa?$AAl@ 10022a40     swiusb.obj
 0002:0000bab8       ??_C@_1BCI@IIJDHPGC@?$AAS?$AAw?$AAi?$AAG?$AAo?$AAb?$AAi?$AA?5?$AAU?$AAS?$AAB?$AAD?$AAe?$AAv?$AAi?$AAc?$AAe?$AAA?$AAt?$AAt?$AAa?$AAc?$AAh?$AA?3?$AA?5?$AAi?$AAt?$AAe?$AAr?$AAa?$AAt?$AAi@ 10022ab8     swiusb.obj
 0002:0000bbe0       ??_C@_1GO@MPGCNPFC@?$AAS?$AAw?$AAi?$AAG?$AAo?$AAb?$AAi?$AA?5?$AAU?$AAS?$AAB?$AAD?$AAe?$AAv?$AAi?$AAc?$AAe?$AAA?$AAt?$AAt?$AAa?$AAc?$AAh?$AA?3?$AA?5?$AAg?$AAM?$AAo?$AAd?$AAe?$AAm?$AA?4@ 10022be0     swiusb.obj
 0002:0000bc50       ??_C@_1HK@JEKLACDH@?$AAS?$AAw?$AAi?$AAG?$AAo?$AAb?$AAi?$AA?5?$AAU?$AAS?$AAB?$AAD?$AAe?$AAv?$AAi?$AAc?$AAe?$AAA?$AAt?$AAt?$AAa?$AAc?$AAh?$AA?3?$AA?5?$AAF?$AAa?$AAi?$AAl?$AAe?$AAd?$AA?5@ 10022c50     swiusb.obj
 0002:0000bccc       ??_C@_1CI@IDPHKGBP@?$AAQ?$AAm?$AAi?$AAF?$AAi?$AAl?$AAt?$AAe?$AAr?$AA?$CF?$AAd?$AA?5?$AA?$DN?$AA?5?$AA?$CF?$AAx?$AA?4?$AA?$AN?$AA?6?$AA?$AA@ 10022ccc     swiusb.obj
 0002:0000bcf4       ??_C@_1DI@JGBFKNCP@?$AAF?$AAa?$AAi?$AAl?$AA?5?$AAt?$AAo?$AA?5?$AAr?$AAe?$AAa?$AAd?$AA?5?$AAQ?$AAm?$AAi?$AAF?$AAi?$AAl?$AAt?$AAe?$AAr?$AA?$CF?$AAd?$AA?4?$AA?$AN?$AA?6?$AA?$AA@ 10022cf4     swiusb.obj
 0002:0000bd2c       ??_C@_1BI@IDOOOGG@?$AAQ?$AAm?$AAi?$AAF?$AAi?$AAl?$AAt?$AAe?$AAr?$AA?$CF?$AAd?$AA?$AA@ 10022d2c     swiusb.obj
 0002:0000bd44       ??_C@_1DK@IPCEPODL@?$AAF?$AAa?$AAi?$AAl?$AA?5?$AAt?$AAo?$AA?5?$AAr?$AAe?$AAa?$AAd?$AA?5?$AAQ?$AAm?$AAi?$AAF?$AAi?$AAl?$AAt?$AAe?$AAr?$AAC?$AAn?$AAt?$AA?4?$AA?$AN?$AA?6?$AA?$AA@ 10022d44     swiusb.obj
 0002:0000bd80       ??_C@_1BK@CHFHLGPB@?$AAQ?$AAm?$AAi?$AAF?$AAi?$AAl?$AAt?$AAe?$AAr?$AAC?$AAn?$AAt?$AA?$AA@ 10022d80     swiusb.obj
 0002:0000bda0       ??_C@_1HI@NIAOAIBJ@?$AAF?$AAa?$AAi?$AAl?$AA?5?$AAt?$AAo?$AA?5?$AAr?$AAe?$AAa?$AAd?$AA?5?$AAQ?$AAm?$AAi?$AAF?$AAi?$AAl?$AAt?$AAe?$AAr?$AAi?$AAn?$AAg?$AAS?$AAu?$AAp?$AAp?$AAo?$AAr?$AAt@ 10022da0     swiusb.obj
 0002:0000be18       ??_C@_1CI@DJCKPDBO@?$AAQ?$AAm?$AAi?$AAF?$AAi?$AAl?$AAt?$AAe?$AAr?$AAi?$AAn?$AAg?$AAS?$AAu?$AAp?$AAp?$AAo?$AAr?$AAt?$AA?$AA@ 10022e18     swiusb.obj
 0002:0000be40       ??_C@_1GG@HBMCAIMK@?$AAS?$AAw?$AAi?$AAG?$AAo?$AAb?$AAi?$AA?5?$AAU?$AAs?$AAi?$AAn?$AAg?$AA?5?$AAD?$AAe?$AAf?$AAa?$AAu?$AAl?$AAt?$AA?5?$AAg?$AAd?$AAw?$AAM?$AAa?$AAx?$AAA?$AAl?$AAl?$AAo@ 10022e40     swiusb.obj
 0002:0000bea8       ??_C@_1DA@GPDPFPLB@?$AAM?$AAa?$AAx?$AAA?$AAl?$AAl?$AAo?$AAc?$AAa?$AAt?$AAe?$AAS?$AAi?$AAz?$AAe?$AAP?$AAe?$AAr?$AAC?$AAh?$AAu?$AAn?$AAk?$AA?$AA@ 10022ea8     swiusb.obj
 0002:0000bed8       ??_C@_1GG@EGDODIDA@?$AAS?$AAw?$AAi?$AAG?$AAo?$AAb?$AAi?$AA?5?$AAU?$AAS?$AAB?$AAD?$AAe?$AAv?$AAi?$AAc?$AAe?$AAA?$AAt?$AAt?$AAa?$AAc?$AAh?$AA?3?$AA?5?$AAU?$AAs?$AAe?$AAN?$AAd?$AAi?$AAs@ 10022ed8     swiusb.obj
 0002:0000bf40       ??_C@_1MM@MFIHENPM@?$AAS?$AAw?$AAi?$AAG?$AAo?$AAb?$AAi?$AA?5?$AAU?$AAS?$AAB?$AAD?$AAe?$AAv?$AAi?$AAc?$AAe?$AAA?$AAt?$AAt?$AAa?$AAc?$AAh?$AA?3?$AA?5?$AAU?$AAs?$AAe?$AAN?$AAd?$AAi?$AAs@ 10022f40     swiusb.obj
 0002:0000c010       ??_C@_1NE@CPEGCCIA@?$AAS?$AAw?$AAi?$AAG?$AAo?$AAb?$AAi?$AA?5?$AAU?$AAS?$AAB?$AAD?$AAe?$AAv?$AAi?$AAc?$AAe?$AAA?$AAt?$AAt?$AAa?$AAc?$AAh?$AA?3?$AA?5?$AAU?$AAs?$AAe?$AAN?$AAd?$AAi?$AAs@ 10023010     swiusb.obj
 0002:0000c0e4       ??_C@_1BC@IIOGDLPJ@?$AAP?$AAo?$AAc?$AAk?$AAe?$AAt?$AAP?$AAC?$AA?$AA@ 100230e4     swiusb.obj
 0002:0000c0f8       ??_C@_1CC@JPACPGJM@?$AAE?$AAn?$AAa?$AAb?$AAl?$AAe?$AAD?$AAa?$AAt?$AAa?$AAB?$AAu?$AAn?$AAd?$AAl?$AAe?$AA?$AA@ 100230f8     swiusb.obj
 0002:0000c11c       ??_C@_1CG@MGIIHJNI@?$AAD?$AAe?$AAv?$AAi?$AAc?$AAe?$AAR?$AAe?$AAm?$AAo?$AAt?$AAe?$AAW?$AAa?$AAk?$AAe?$AAu?$AAp?$AA?$AA@ 1002311c     swiusb.obj
 0002:0000c148       ??_C@_1JG@CEBLNALF@?$AAS?$AAw?$AAi?$AAG?$AAo?$AAb?$AAi?$AA?5?$AAU?$AAS?$AAB?$AAD?$AAe?$AAv?$AAi?$AAc?$AAe?$AAA?$AAt?$AAt?$AAa?$AAc?$AAh?$AA?3?$AA?5?$AAE?$AAn?$AAa?$AAb?$AAl?$AAe?$AAD@ 10023148     swiusb.obj
 0002:0000c1e0       ??_C@_1CK@PADNAHAE@?$AAU?$AAs?$AAe?$AAN?$AAd?$AAi?$AAs?$AAC?$AAo?$AAn?$AAf?$AAi?$AAg?$AAu?$AAr?$AAa?$AAt?$AAi?$AAo?$AAn?$AA?$AA@ 100231e0     swiusb.obj
 0002:0000c210       ??_C@_1LC@FLODCLEI@?$AAS?$AAw?$AAi?$AAG?$AAo?$AAb?$AAi?$AA?5?$AAU?$AAS?$AAB?$AAD?$AAe?$AAv?$AAi?$AAc?$AAe?$AAA?$AAt?$AAt?$AAa?$AAc?$AAh?$AA?3?$AA?5?$AAQ?$AAm?$AAi?$AA?5?$AAc?$AAh?$AAa@ 10023210     swiusb.obj
 0002:0000c2c4       ??_C@_1BG@MKCDCOAH@?$AAQ?$AAM?$AAI?$AAC?$AAh?$AAa?$AAn?$AAn?$AAe?$AAl?$AA?$AA@ 100232c4     swiusb.obj
 0002:0000c2e0       ??_C@_1FK@JLBLJDH@?$AAS?$AAw?$AAi?$AAG?$AAo?$AAb?$AAi?$AA?5?$AAU?$AAS?$AAB?$AAD?$AAe?$AAv?$AAi?$AAc?$AAe?$AAA?$AAt?$AAt?$AAa?$AAc?$AAh?$AA?3?$AA?5?$AAQ?$AAm?$AAi?$AA?5?$AAc?$AAh?$AAa@ 100232e0     swiusb.obj
 0002:0000c340       ??_C@_1GA@FIJIABPP@?$AAS?$AAw?$AAi?$AAG?$AAo?$AAb?$AAi?$AA?5?$AAU?$AAS?$AAB?$AAD?$AAe?$AAv?$AAi?$AAc?$AAe?$AAA?$AAt?$AAt?$AAa?$AAc?$AAh?$AA?3?$AA?5?$AAM?$AAo?$AAd?$AAu?$AAl?$AAe?$AAS@ 10023340     swiusb.obj
 0002:0000c3a0       ??_C@_1CE@HIGJLKC@?$AAD?$AAi?$AAs?$AAa?$AAb?$AAl?$AAe?$AAQ?$AAM?$AAI?$AAC?$AAh?$AAa?$AAn?$AAn?$AAe?$AAl?$AA?$AA@ 100233a0     swiusb.obj
 0002:0000c3c8       ??_C@_1LK@KKJLEBJ@?$AAS?$AAw?$AAi?$AAG?$AAo?$AAb?$AAi?$AA?5?$AAU?$AAS?$AAB?$AAD?$AAe?$AAv?$AAi?$AAc?$AAe?$AAA?$AAt?$AAt?$AAa?$AAc?$AAh?$AA?3?$AA?5?$AAD?$AAi?$AAs?$AAc?$AAr?$AAi?$AAm@ 100233c8     swiusb.obj
 0002:0000c488       ??_C@_1GE@FAKGLPDI@?$AAS?$AAw?$AAi?$AAG?$AAo?$AAb?$AAi?$AA?5?$AAU?$AAS?$AAB?$AAD?$AAe?$AAv?$AAi?$AAc?$AAe?$AAA?$AAt?$AAt?$AAa?$AAc?$AAh?$AA?3?$AA?5?$AAg?$AAM?$AAo?$AAd?$AAe?$AAm?$AA?4@ 10023488     swiusb.obj
 0002:0000c4f0       ??_C@_1FC@DCKKILJE@?$AAS?$AAw?$AAi?$AAG?$AAo?$AAb?$AAi?$AA?5?$AAU?$AAS?$AAB?$AAD?$AAe?$AAv?$AAi?$AAc?$AAe?$AAA?$AAt?$AAt?$AAa?$AAc?$AAh?$AA?$CI?$AA?$CJ?$AA?5?$AA?$CF?$AAx?$AA?3?$AA?$CF?$AAx?$AA?0@ 100234f0     swiusb.obj
 0002:0000c548       ??_C@_1KE@DOLIKAJO@?$AAS?$AAw?$AAi?$AAG?$AAo?$AAb?$AAi?$AA?5?$AAU?$AAS?$AAB?$AAD?$AAe?$AAv?$AAi?$AAc?$AAe?$AAA?$AAt?$AAt?$AAa?$AAc?$AAh?$AA?5?$AAf?$AAa?$AAi?$AAl?$AAe?$AAd?$AA?5?$AAb@ 10023548     swiusb.obj
 0002:0000c5ec       ??_C@_0L@FFLPPCPC@2?43?40?4248?$AA?$AA@ 100235ec     swiusb.obj
 0002:0000c5f8       ??_C@_1GM@MCHONOHB@?$AAS?$AAw?$AAi?$AAG?$AAo?$AAb?$AAi?$AA?5?$AA?$CF?$AAs?$AA?5?$AAU?$AAS?$AAB?$AAD?$AAe?$AAv?$AAi?$AAc?$AAe?$AAA?$AAt?$AAt?$AAa?$AAc?$AAh?$AA?$CI?$AA?$CJ?$AA?5?$AAc?$AAa?$AAl@ 100235f8     swiusb.obj
 0002:0000c664       ??_7WdsService@@6B@        10023664     WdsService.obj
 0002:0000c668       ??_C@_1BG@MPHODBAD@?$AAM?$AAA?$AAC?$AAA?$AAd?$AAd?$AAr?$AAe?$AAs?$AAs?$AA?$AA@ 10023668     wrp.obj
 0002:0000c680       ??_C@_0BK@LBOGNABE@Allocate?5Mem?5for?5Adapter?$CB?$AA@ 10023680     wrp.obj
 0002:0000c69c       ??_C@_0BC@MDBJCCMB@OID_PNP_SET_POWER?$AA@ 1002369c     wrpoid.obj
 0002:0000c6b0       ??_C@_0BE@JKEJBMBE@OID_PNP_QUERY_POWER?$AA@ 100236b0     wrpoid.obj
 0002:0000c6c4       ??_C@_0BM@OJJIMKNI@OID_PNP_ADD_WAKE_UP_PATTERN?$AA@ 100236c4     wrpoid.obj
 0002:0000c6e0       ??_C@_0BP@BIOEBNGF@OID_PNP_REMOVE_WAKE_UP_PATTERN?$AA@ 100236e0     wrpoid.obj
 0002:0000c700       ??_C@_0BH@OJMBGEJC@OID_PNP_ENABLE_WAKE_UP?$AA@ 10023700     wrpoid.obj
 0002:0000c718       ??_C@_0BF@LFNCIFLM@OID_PNP_CAPABILITIES?$AA@ 10023718     wrpoid.obj
 0002:0000c730       ??_C@_0BG@CPNFBMBB@OID_802_3_RCV_OVERRUN?$AA@ 10023730     wrpoid.obj
 0002:0000c748       ??_C@_0BI@MHFCPDCD@OID_802_3_XMIT_UNDERRUN?$AA@ 10023748     wrpoid.obj
 0002:0000c760       ??_C@_0CB@NHIJAIHB@OID_802_3_XMIT_HEARTBEAT_FAILURE@ 10023760     wrpoid.obj
 0002:0000c784       ??_C@_0BO@OBOJJGEE@OID_802_3_XMIT_TIMES_CRS_LOST?$AA@ 10023784     wrpoid.obj
 0002:0000c7a4       ??_C@_0BP@HKGMKPAO@OID_802_3_XMIT_LATE_COLLISIONS?$AA@ 100237a4     wrpoid.obj
 0002:0000c7c4       ??_C@_0BF@DBJDFIIP@OID_TCP_TASK_OFFLOAD?$AA@ 100237c4     wrpoid.obj
 0002:0000c7dc       ??_C@_0BO@LHEEJDIC@OID_802_3_XMIT_MAX_COLLISIONS?$AA@ 100237dc     wrpoid.obj
 0002:0000c7fc       ??_C@_0BG@DJLEHAKJ@OID_802_3_MAC_OPTIONS?$AA@ 100237fc     wrpoid.obj
 0002:0000c814       ??_C@_0BO@JOMCHLFL@OID_802_3_RCV_ERROR_ALIGNMENT?$AA@ 10023814     wrpoid.obj
 0002:0000c834       ??_C@_0BN@FPAEEELK@OID_802_3_XMIT_ONE_COLLISION?$AA@ 10023834     wrpoid.obj
 0002:0000c854       ??_C@_0BP@MBLFGNFM@OID_802_3_XMIT_MORE_COLLISIONS?$AA@ 10023854     wrpoid.obj
 0002:0000c874       ??_C@_0BI@FANFODJE@OID_802_3_XMIT_DEFERRED?$AA@ 10023874     wrpoid.obj
 0002:0000c88c       ??_C@_0BM@FPCCEEDI@OID_802_3_MAXIMUM_LIST_SIZE?$AA@ 1002388c     wrpoid.obj
 0002:0000c8a8       ??_C@_0BF@HIFFIOBM@OID_GEN_INIT_TIME_MS?$AA@ 100238a8     wrpoid.obj
 0002:0000c8c0       ??_C@_0BF@HDAJAGLL@OID_GEN_RESET_COUNTS?$AA@ 100238c0     wrpoid.obj
 0002:0000c8d8       ??_C@_0BL@HEHOEBGJ@OID_GEN_MEDIA_SENSE_COUNTS?$AA@ 100238d8     wrpoid.obj
 0002:0000c8f4       ??_C@_0BM@CAKPHAJN@OID_802_3_PERMANENT_ADDRESS?$AA@ 100238f4     wrpoid.obj
 0002:0000c910       ??_C@_0BK@JOACIFFK@OID_802_3_CURRENT_ADDRESS?$AA@ 10023910     wrpoid.obj
 0002:0000c92c       ??_C@_0BJ@CKLEHGNL@OID_802_3_MULTICAST_LIST?$AA@ 1002392c     wrpoid.obj
 0002:0000c948       ??_C@_0BH@BHDABHDN@OID_GEN_DEVICE_PROFILE?$AA@ 10023948     wrpoid.obj
 0002:0000c960       ??_C@_0BF@IJACFDP@OID_GEN_NETCARD_LOAD?$AA@ 10023960     wrpoid.obj
 0002:0000c978       ??_C@_0BJ@PLCKPGJO@OID_GEN_GET_NETCARD_TIME?$AA@ 10023978     wrpoid.obj
 0002:0000c994       ??_C@_0BG@EFCMMCPA@OID_GEN_GET_TIME_CAPS?$AA@ 10023994     wrpoid.obj
 0002:0000c9ac       ??_C@_0BO@DNKICFCL@OID_GEN_TRANSMIT_QUEUE_LENGTH?$AA@ 100239ac     wrpoid.obj
 0002:0000c9cc       ??_C@_0BG@GFCAPEIO@OID_GEN_RCV_CRC_ERROR?$AA@ 100239cc     wrpoid.obj
 0002:0000c9e4       ??_C@_0BN@IALAGHHD@OID_GEN_BROADCAST_FRAMES_RCV?$AA@ 100239e4     wrpoid.obj
 0002:0000ca04       ??_C@_0BM@BDEGPINC@OID_GEN_BROADCAST_BYTES_RCV?$AA@ 10023a04     wrpoid.obj
 0002:0000ca20       ??_C@_0BN@FGFAFGIK@OID_GEN_MULTICAST_FRAMES_RCV?$AA@ 10023a20     wrpoid.obj
 0002:0000ca40       ??_C@_0BM@CFNEOJHC@OID_GEN_MULTICAST_BYTES_RCV?$AA@ 10023a40     wrpoid.obj
 0002:0000ca5c       ??_C@_0BM@IFPJCDGF@OID_GEN_DIRECTED_FRAMES_RCV?$AA@ 10023a5c     wrpoid.obj
 0002:0000ca78       ??_C@_0BL@FKFFPNBF@OID_GEN_DIRECTED_BYTES_RCV?$AA@ 10023a78     wrpoid.obj
 0002:0000ca94       ??_C@_0BO@KKEOIDGO@OID_GEN_BROADCAST_FRAMES_XMIT?$AA@ 10023a94     wrpoid.obj
 0002:0000cab4       ??_C@_0BN@LAMOGIP@OID_GEN_BROADCAST_BYTES_XMIT?$AA@ 10023ab4     wrpoid.obj
 0002:0000cad4       ??_C@_0BG@KEBGHFLF@OID_GEN_RCV_NO_BUFFER?$AA@ 10023ad4     wrpoid.obj
 0002:0000caec       ??_C@_0BM@OEFKCJJ@OID_GEN_DIRECTED_BYTES_XMIT?$AA@ 10023aec     wrpoid.obj
 0002:0000cb08       ??_C@_0BN@FOJPHPHL@OID_GEN_DIRECTED_FRAMES_XMIT?$AA@ 10023b08     wrpoid.obj
 0002:0000cb28       ??_C@_0BN@NNOMNHHG@OID_GEN_MULTICAST_BYTES_XMIT?$AA@ 10023b28     wrpoid.obj
 0002:0000cb48       ??_C@_0BO@GOPJCJOH@OID_GEN_MULTICAST_FRAMES_XMIT?$AA@ 10023b48     wrpoid.obj
 0002:0000cb68       ??_C@_0BC@ONFJJFBK@OID_GEN_RCV_ERROR?$AA@ 10023b68     wrpoid.obj
 0002:0000cb7c       ??_C@_0BI@CDALPKOI@OID_GEN_PHYSICAL_MEDIUM?$AA@ 10023b7c     wrpoid.obj
 0002:0000cb94       ??_C@_0BF@HFNEDJIP@OID_GEN_MACHINE_NAME?$AA@ 10023b94     wrpoid.obj
 0002:0000cbac       ??_C@_0BA@PMNPHIKH@OID_GEN_VLAN_ID?$AA@ 10023bac     wrpoid.obj
 0002:0000cbbc       ??_C@_0BA@KDEAMBC@OID_GEN_XMIT_OK?$AA@ 10023bbc     wrpoid.obj
 0002:0000cbcc       ??_C@_0P@GCNHCIO@OID_GEN_RCV_OK?$AA@ 10023bcc     wrpoid.obj
 0002:0000cbdc       ??_C@_0BD@MMIHCIDK@OID_GEN_XMIT_ERROR?$AA@ 10023bdc     wrpoid.obj
 0002:0000cbf0       ??_C@_0BL@FPFDHMAL@OID_GEN_MEDIA_CAPABILITIES?$AA@ 10023bf0     wrpoid.obj
 0002:0000cc0c       ??_C@_0CA@PJEFHMLF@OID_GEN_TRANSPORT_HEADER_OFFSET?$AA@ 10023c0c     wrpoid.obj
 0002:0000cc2c       ??_C@_0CA@BGMGBMGO@OID_GEN_NETWORK_LAYER_ADDRESSES?$AA@ 10023c2c     wrpoid.obj
 0002:0000cc4c       ??_C@_0BI@EECPDLPA@OID_GEN_SUPPORTED_GUIDS?$AA@ 10023c4c     wrpoid.obj
 0002:0000cc64       ??_C@_0BO@HNPMPDID@OID_GEN_VENDOR_DRIVER_VERSION?$AA@ 10023c64     wrpoid.obj
 0002:0000cc84       ??_C@_0BN@DFFNGMPL@OID_GEN_MAXIMUM_SEND_PACKETS?$AA@ 10023c84     wrpoid.obj
 0002:0000cca4       ??_C@_0BN@DHCFNFOF@OID_GEN_MEDIA_CONNECT_STATUS?$AA@ 10023ca4     wrpoid.obj
 0002:0000ccc4       ??_C@_0BE@MBIIMLOK@OID_GEN_MAC_OPTIONS?$AA@ 10023cc4     wrpoid.obj
 0002:0000ccd8       ??_C@_0BJ@JFMBEBBO@OID_GEN_PROTOCOL_OPTIONS?$AA@ 10023cd8     wrpoid.obj
 0002:0000ccf4       ??_C@_0BL@JANNBEHP@OID_GEN_MAXIMUM_TOTAL_SIZE?$AA@ 10023cf4     wrpoid.obj
 0002:0000cd10       ??_C@_0BH@EGJPBFMD@OID_GEN_DRIVER_VERSION?$AA@ 10023d10     wrpoid.obj
 0002:0000cd28       ??_C@_0BK@PGGOCJND@OID_GEN_CURRENT_LOOKAHEAD?$AA@ 10023d28     wrpoid.obj
 0002:0000cd44       ??_C@_0BO@OPJLNKIE@OID_GEN_CURRENT_PACKET_FILTER?$AA@ 10023d44     wrpoid.obj
 0002:0000cd64       ??_C@_0BL@HPFNNEGO@OID_GEN_VENDOR_DESCRIPTION?$AA@ 10023d64     wrpoid.obj
 0002:0000cd80       ??_C@_0BC@BGMLJMJO@OID_GEN_VENDOR_ID?$AA@ 10023d80     wrpoid.obj
 0002:0000cd94       ??_C@_0BL@GGCMPDBD@OID_GEN_RECEIVE_BLOCK_SIZE?$AA@ 10023d94     wrpoid.obj
 0002:0000cdb0       ??_C@_0BM@KEBLGIOC@OID_GEN_TRANSMIT_BLOCK_SIZE?$AA@ 10023db0     wrpoid.obj
 0002:0000cdcc       ??_C@_0BN@EFKECEFB@OID_GEN_RECEIVE_BUFFER_SPACE?$AA@ 10023dcc     wrpoid.obj
 0002:0000cdec       ??_C@_0BO@CPNOHMFG@OID_GEN_TRANSMIT_BUFFER_SPACE?$AA@ 10023dec     wrpoid.obj
 0002:0000ce0c       ??_C@_0BD@GJDHJMIG@OID_GEN_LINK_SPEED?$AA@ 10023e0c     wrpoid.obj
 0002:0000ce20       ??_C@_0BL@JAHHDEIP@OID_GEN_MAXIMUM_FRAME_SIZE?$AA@ 10023e20     wrpoid.obj
 0002:0000ce3c       ??_C@_0BK@BEBJNGFH@OID_GEN_MAXIMUM_LOOKAHEAD?$AA@ 10023e3c     wrpoid.obj
 0002:0000ce58       ??_C@_0BF@CAILKECK@OID_GEN_MEDIA_IN_USE?$AA@ 10023e58     wrpoid.obj
 0002:0000ce70       ??_C@_0BI@BACFMEHI@OID_GEN_MEDIA_SUPPORTED?$AA@ 10023e70     wrpoid.obj
 0002:0000ce88       ??_C@_0BI@NKMHNFOK@OID_GEN_HARDWARE_STATUS?$AA@ 10023e88     wrpoid.obj
 0002:0000cea0       ??_C@_0BH@OPBIGOOD@OID_GEN_SUPPORTED_LIST?$AA@ 10023ea0     wrpoid.obj
 0002:0000ceb8       ??_C@_0BB@FGHCFFEN@Sierra?5Wireless?5?$AA@ 10023eb8     wrpoid.obj
 0002:0000cecc       ??_C@_08IMPLNKDD@?5Adapter?$AA@ 10023ecc     wrpoid.obj
 0002:0000ced8       ??_C@_04OPBHEPOC@0x?$CFx?$AA@ 10023ed8     wrpoid.obj
 0002:0000d020       __IMPORT_DESCRIPTOR_NDIS   10024020     ndis:NDIS.dll
 0002:0000d034       __IMPORT_DESCRIPTOR_WS2    10024034     ws2:WS2.dll
 0002:0000d048       __IMPORT_DESCRIPTOR_COREDLL 10024048     coredll:COREDLL.dll
 0002:0000d05c       __NULL_IMPORT_DESCRIPTOR   1002405c     ndis:NDIS.dll
 0003:00000000       __imp_ReadFile             10025000     coredll:COREDLL.dll
 0003:00000004       __imp_TlsGetValue          10025004     coredll:COREDLL.dll
 0003:00000008       __imp_TlsSetValue          10025008     coredll:COREDLL.dll
 0003:0000000c       __imp_TlsCall              1002500c     coredll:COREDLL.dll
 0003:00000010       __imp_memmove              10025010     coredll:COREDLL.dll
 0003:00000014       __imp_?terminate@std@@YAXXZ 10025014     coredll:COREDLL.dll
 0003:00000018       __imp_strcmp               10025018     coredll:COREDLL.dll
 0003:0000001c       __imp___security_gen_cookie 1002501c     coredll:COREDLL.dll
 0003:00000020       __imp_LocalSize            10025020     coredll:COREDLL.dll
 0003:00000024       __imp_LocalReAlloc         10025024     coredll:COREDLL.dll
 0003:00000028       __imp___report_gsfailure   10025028     coredll:COREDLL.dll
 0003:0000002c       __imp_sprintf              1002502c     coredll:COREDLL.dll
 0003:00000030       __imp_strlen               10025030     coredll:COREDLL.dll
 0003:00000034       __imp_memcmp               10025034     coredll:COREDLL.dll
 0003:00000038       __imp_wcscmp               10025038     coredll:COREDLL.dll
 0003:0000003c       __imp_wcscpy               1002503c     coredll:COREDLL.dll
 0003:00000040       __imp_MultiByteToWideChar  10025040     coredll:COREDLL.dll
 0003:00000044       __imp_SystemParametersInfoW 10025044     coredll:COREDLL.dll
 0003:00000048       __imp_ActivateDeviceEx     10025048     coredll:COREDLL.dll
 0003:0000004c       __imp_GetSystemPowerState  1002504c     coredll:COREDLL.dll
 0003:00000050       __imp__wcslwr              10025050     coredll:COREDLL.dll
 0003:00000054       __imp_wcsstr               10025054     coredll:COREDLL.dll
 0003:00000058       __imp_SetSystemPowerState  10025058     coredll:COREDLL.dll
 0003:0000005c       __imp_DeactivateDevice     1002505c     coredll:COREDLL.dll
 0003:00000060       __imp_StringCchPrintfW     10025060     coredll:COREDLL.dll
 0003:00000064       __imp_StringCchCatW        10025064     coredll:COREDLL.dll
 0003:00000068       __imp_TerminateThread      10025068     coredll:COREDLL.dll
 0003:0000006c       __imp_IsBadReadPtr         1002506c     coredll:COREDLL.dll
 0003:00000070       __imp_VirtualFree          10025070     coredll:COREDLL.dll
 0003:00000074       __imp_HeapFree             10025074     coredll:COREDLL.dll
 0003:00000078       __imp_VirtualAlloc         10025078     coredll:COREDLL.dll
 0003:0000007c       __imp_GetProcessHeap       1002507c     coredll:COREDLL.dll
 0003:00000080       __imp_EventModify          10025080     coredll:COREDLL.dll
 0003:00000084       __imp_CloseMsgQueue        10025084     coredll:COREDLL.dll
 0003:00000088       __imp_DeleteCriticalSection 10025088     coredll:COREDLL.dll
 0003:0000008c       __imp_LeaveCriticalSection 1002508c     coredll:COREDLL.dll
 0003:00000090       __imp_CloseHandle          10025090     coredll:COREDLL.dll
 0003:00000094       __imp_NKDbgPrintfW         10025094     coredll:COREDLL.dll
 0003:00000098       __imp_WaitForSingleObject  10025098     coredll:COREDLL.dll
 0003:0000009c       __imp_EnterCriticalSection 1002509c     coredll:COREDLL.dll
 0003:000000a0       __imp_Sleep                100250a0     coredll:COREDLL.dll
 0003:000000a4       __imp_GetTickCount         100250a4     coredll:COREDLL.dll
 0003:000000a8       __imp_GetLastError         100250a8     coredll:COREDLL.dll
 0003:000000ac       __imp_ReadMsgQueue         100250ac     coredll:COREDLL.dll
 0003:000000b0       __imp_memset               100250b0     coredll:COREDLL.dll
 0003:000000b4       __imp_WaitForMultipleObjects 100250b4     coredll:COREDLL.dll
 0003:000000b8       __imp_CeSetThreadPriority  100250b8     coredll:COREDLL.dll
 0003:000000bc       __imp_RequestPowerNotifications 100250bc     coredll:COREDLL.dll
 0003:000000c0       __imp_CreateMsgQueue       100250c0     coredll:COREDLL.dll
 0003:000000c4       __imp_InitializeCriticalSection 100250c4     coredll:COREDLL.dll
 0003:000000c8       __imp_CreateThread         100250c8     coredll:COREDLL.dll
 0003:000000cc       __imp_CreateEventW         100250cc     coredll:COREDLL.dll
 0003:000000d0       __imp_memcpy               100250d0     coredll:COREDLL.dll
 0003:000000d4       __imp___rt_udiv            100250d4     coredll:COREDLL.dll
 0003:000000d8       __imp_vswprintf            100250d8     coredll:COREDLL.dll
 0003:000000dc       __imp_SetCommMask          100250dc     coredll:COREDLL.dll
 0003:000000e0       __imp_??3@YAXPAX@Z         100250e0     coredll:COREDLL.dll
 0003:000000e4       __imp_SetCommState         100250e4     coredll:COREDLL.dll
 0003:000000e8       __imp_CreateFileW          100250e8     coredll:COREDLL.dll
 0003:000000ec       __imp_swprintf             100250ec     coredll:COREDLL.dll
 0003:000000f0       __imp_??2@YAPAXI@Z         100250f0     coredll:COREDLL.dll
 0003:000000f4       __imp_GetCommModemStatus   100250f4     coredll:COREDLL.dll
 0003:000000f8       __imp_EscapeCommFunction   100250f8     coredll:COREDLL.dll
 0003:000000fc       __imp_SetLastError         100250fc     coredll:COREDLL.dll
 0003:00000100       __imp_InterlockedCompareExchange 10025100     coredll:COREDLL.dll
 0003:00000104       __imp_WriteFile            10025104     coredll:COREDLL.dll
 0003:00000108       __imp_DeviceIoControl      10025108     coredll:COREDLL.dll
 0003:0000010c       __imp_??_L@YAXPAXIHP6AX0@Z1@Z 1002510c     coredll:COREDLL.dll
 0003:00000110       __imp_??_M@YAXPAXIHP6AX0@Z@Z 10025110     coredll:COREDLL.dll
 0003:00000114       __imp_SystemTimeToFileTime 10025114     coredll:COREDLL.dll
 0003:00000118       __imp_GetSystemTime        10025118     coredll:COREDLL.dll
 0003:0000011c       __imp___rt_udiv64by64      1002511c     coredll:COREDLL.dll
 0003:00000120       __imp_FlushFileBuffers     10025120     coredll:COREDLL.dll
 0003:00000124       __imp_SetFilePointer       10025124     coredll:COREDLL.dll
 0003:00000128       __imp_RegCloseKey          10025128     coredll:COREDLL.dll
 0003:0000012c       __imp_RegDeleteValueW      1002512c     coredll:COREDLL.dll
 0003:00000130       __imp_RegOpenKeyExW        10025130     coredll:COREDLL.dll
 0003:00000134       __imp_wsprintfW            10025134     coredll:COREDLL.dll
 0003:00000138       __imp_wcslen               10025138     coredll:COREDLL.dll
 0003:0000013c       __imp_strncpy              1002513c     coredll:COREDLL.dll
 0003:00000140       __imp___C_specific_handler 10025140     coredll:COREDLL.dll
 0003:00000144       __imp_InterlockedExchange  10025144     coredll:COREDLL.dll
 0003:00000148       __imp_LocalAlloc           10025148     coredll:COREDLL.dll
 0003:0000014c       __imp_LocalFree            1002514c     coredll:COREDLL.dll
 0003:00000150       __imp_RegQueryValueExW     10025150     coredll:COREDLL.dll
 0003:00000154       __imp_RegSetValueExW       10025154     coredll:COREDLL.dll
 0003:00000158       __imp_RegCreateKeyExW      10025158     coredll:COREDLL.dll
 0003:0000015c       __imp_wcsncat              1002515c     coredll:COREDLL.dll
 0003:00000160       __imp__snwprintf           10025160     coredll:COREDLL.dll
 0003:00000164       __imp_rand                 10025164     coredll:COREDLL.dll
 0003:00000168       __imp_wcscat               10025168     coredll:COREDLL.dll
 0003:0000016c       __imp_FindClose            1002516c     coredll:COREDLL.dll
 0003:00000170       __imp_FindFirstFileW       10025170     coredll:COREDLL.dll
 0003:00000174       __imp__wcsicmp             10025174     coredll:COREDLL.dll
 0003:00000178       __imp_GetStoreInformation  10025178     coredll:COREDLL.dll
 0003:0000017c       __imp_GlobalMemoryStatus   1002517c     coredll:COREDLL.dll
 0003:00000180       __imp_HeapAlloc            10025180     coredll:COREDLL.dll
 0003:00000184       \177COREDLL_NULL_THUNK_DATA 10025184     coredll:COREDLL.dll
 0003:00000188       __imp_NdisInitializeEvent  10025188     ndis:NDIS.dll
 0003:0000018c       __imp_NdisAcquireSpinLock  1002518c     ndis:NDIS.dll
 0003:00000190       __imp_NdisResetEvent       10025190     ndis:NDIS.dll
 0003:00000194       __imp_NdisUnicodeStringToAnsiString 10025194     ndis:NDIS.dll
 0003:00000198       __imp_NdisReadConfiguration 10025198     ndis:NDIS.dll
 0003:0000019c       __imp_NdisCloseConfiguration 1002519c     ndis:NDIS.dll
 0003:000001a0       __imp_NdisOpenConfiguration 100251a0     ndis:NDIS.dll
 0003:000001a4       __imp_NdisFreeMemory       100251a4     ndis:NDIS.dll
 0003:000001a8       __imp_NdisAllocateMemoryWithTag 100251a8     ndis:NDIS.dll
 0003:000001ac       __imp_NdisSetTimer         100251ac     ndis:NDIS.dll
 0003:000001b0       __imp_NdisQueryPacket      100251b0     ndis:NDIS.dll
 0003:000001b4       __imp_NdisInitializeWrapper 100251b4     ndis:NDIS.dll
 0003:000001b8       __imp_NdisMRegisterMiniport 100251b8     ndis:NDIS.dll
 0003:000001bc       __imp_NdisTerminateWrapper 100251bc     ndis:NDIS.dll
 0003:000001c0       __imp_NdisAllocateSpinLock 100251c0     ndis:NDIS.dll
 0003:000001c4       __imp_NdisReleaseSpinLock  100251c4     ndis:NDIS.dll
 0003:000001c8       __imp_NdisInitializeTimer  100251c8     ndis:NDIS.dll
 0003:000001cc       __imp_NdisMRegisterAdapterShutdownHandler 100251cc     ndis:NDIS.dll
 0003:000001d0       __imp_NdisMSetAttributesEx 100251d0     ndis:NDIS.dll
 0003:000001d4       __imp_NdisCancelTimer      100251d4     ndis:NDIS.dll
 0003:000001d8       __imp_NdisWaitEvent        100251d8     ndis:NDIS.dll
 0003:000001dc       __imp_NdisFreeEvent        100251dc     ndis:NDIS.dll
 0003:000001e0       __imp_NdisMSleep           100251e0     ndis:NDIS.dll
 0003:000001e4       __imp_NdisMDeregisterAdapterShutdownHandler 100251e4     ndis:NDIS.dll
 0003:000001e8       __imp_NdisFreeSpinLock     100251e8     ndis:NDIS.dll
 0003:000001ec       __imp_NdisWriteErrorLogEntry 100251ec     ndis:NDIS.dll
 0003:000001f0       __imp_NdisRegisterAdapter  100251f0     ndis:NDIS.dll
 0003:000001f4       __imp_NdisDeregisterAdapter 100251f4     ndis:NDIS.dll
 0003:000001f8       __imp_NdisSetEvent         100251f8     ndis:NDIS.dll
 0003:000001fc       \177NDIS_NULL_THUNK_DATA   100251fc     ndis:NDIS.dll
 0003:00000200       __imp_htonl                10025200     ws2:WS2.dll
 0003:00000204       __imp_htons                10025204     ws2:WS2.dll
 0003:00000208       \177WS2_NULL_THUNK_DATA    10025208     ws2:WS2.dll
 0003:0000020c       __xc_a                     1002520c     corelibc:crt0init.obj
 0003:00000218       __xc_z                     10025218     corelibc:crt0init.obj
 0003:0000021c       __xi_a                     1002521c     corelibc:crt0init.obj
 0003:00000220       __xi_z                     10025220     corelibc:crt0init.obj
 0003:00000224       __xp_a                     10025224     corelibc:crt0init.obj
 0003:00000228       __xp_z                     10025228     corelibc:crt0init.obj
 0003:0000022c       __xt_a                     1002522c     corelibc:crt0init.obj
 0003:00000230       __xt_z                     10025230     corelibc:crt0init.obj
 0003:00000238       ?g_IsSavePowerInD2@@3HA    10025238     swicom.obj
 0003:0000023c       ?gIsPowerManagedSupported@@3HA 1002523c     swicom.obj
 0003:00000240       ?InitCommandNames@@3PAPA_WA 10025240     swiroutines.obj
 0003:00000268       ?gdwResumeDetectInterval@@3KA 10025268     swiusb.obj
 0003:0000026c       ?g_bFirstTime@@3HA         1002526c     swiusb.obj
 0003:00000270       ?gArpResponseFrame@@3PAEA  10025270     swiusb.obj
 0003:000002a0       ?gDHCPDiscoveryFrame@@3PAEA 100252a0     swiusb.obj
 0003:000003f8       ?gDHCPRequestFrame@@3PAEA  100253f8     swiusb.obj
 0003:00000550       ?HighestAcceptableMax@@3T_LARGE_INTEGER@@A 10025550     wrpdata.obj
 0003:00000558       __security_cookie_complement 10025558     corelibc:seccook.obj
 0003:0000055c       __security_cookie          1002555c     corelibc:seccook.obj
 0003:00000568       ?g_dwLastDeviceResumedTickCount@@3KA 10025568     CEPowerControl.obj
 0003:0000056c       ?gPrintCount@@3IA          1002556c     dpwce.obj
 0003:00000570       ?gwszSWIUSBKey@@3PA_WA     10025570     swicom.obj
 0003:00000770       ?pOpenPortList@@3PAPAUVSP_OPEN_INFO@@A 10025770     swicom.obj
 0003:00000790       ?CSDisplayRawData@@3UCRITICAL_SECTION@@A 10025790     swicom.obj
 0003:000007a4       ?hDllInstance@@3PAXA       100257a4     swicom.obj
 0003:000007a8       ?guiCOMPortOpenCount@@3IA  100257a8     swicom.obj
 0003:000007ac       ?gDevicePwrState@@3W4_CEDEVICE_POWER_STATE@@A 100257ac     swicom.obj
 0003:000007b0       ?g_IsNMEAInProgress@@3HA   100257b0     swicom.obj
 0003:000007b4       ?gIsUseUnAttendedMode@@3HA 100257b4     swicom.obj
 0003:000007b8       ?bValidInstance@@3EA       100257b8     swicom.obj
 0003:000007bc       ?alreadyAttached@@3HA      100257bc     swicom.obj
 0003:000007c0       ?gMemoryCounter@@3KA       100257c0     swiroutines.obj
 0003:000007c4       ?gdwLastFreeSize@@3KA      100257c4     swiroutines.obj
 0003:000007c8       ?g_IsTerminalSuspended@@3HA 100257c8     swiusb.obj
 0003:000007cc       ?gUseNdisConfiguration@@3KA 100257cc     swiusb.obj
 0003:000007d0       ?CSUSBDeviceState@@3UCRITICAL_SECTION@@A 100257d0     swiusb.obj
 0003:000007e4       ?CSComPortOpenCount@@3UCRITICAL_SECTION@@A 100257e4     swiusb.obj
 0003:000007f8       ?CSSWIUsbMemoryControl@@3UCRITICAL_SECTION@@A 100257f8     swiusb.obj
 0003:0000080c       ?bWindowsMobile@@3KA       1002580c     swiusb.obj
 0003:00000810       ?gTlpContext@@3UTLP_CONTEXT@@A 10025810     swiusb.obj
 0003:00000e08       ?gdwIdleTimeout@@3KA       10025e08     swiusb.obj
 0003:00000e0c       ?gQmiFiltering@@3KA        10025e0c     swiusb.obj
 0003:00000e10       ?gQmiFilterCnt@@3KA        10025e10     swiusb.obj
 0003:00000e14       ?gQmiFilter@@3PAKA         10025e14     swiusb.obj
 0003:00000e50       ?gdwDefaultTransferSize@@3KA 10025e50     swiusb.obj
 0003:00000e54       ?dwThreadId@@3KA           10025e54     swiusb.obj
 0003:00000e58       ?hActivityThread@@3PAXA    10025e58     swiusb.obj
 0003:00000e5c       ?gdwMaxAllocateSizePerChunk@@3KA 10025e5c     swiusb.obj
 0003:00000e60       ?gEnableDataBundle@@3KA    10025e60     swiusb.obj
 0003:00000e64       ?gDeviceRemoteWakeupReg@@3KA 10025e64     swiusb.obj
 0003:00000e68       ?ghDeviceInstalledEvent@@3PAXA 10025e68     swiusb.obj
 0003:00000e6c       ?hDeviceCloseEvent@@3PAXA  10025e6c     swiusb.obj
 0003:00000e70       ?hUSBResumeEvent@@3PAXA    10025e70     swiusb.obj
 0003:00000e74       ?hUSBSuspendEvent@@3PAXA   10025e74     swiusb.obj
 0003:00000e78       ?hUSBActivityEvent@@3PAXA  10025e78     swiusb.obj
 0003:00000e7c       ?hHostJustResumedEvent@@3PAXA 10025e7c     swiusb.obj
 0003:00000e80       ?hPortRemoteWakeup@@3PAXA  10025e80     swiusb.obj
 0003:00000e84       ?hSendArpResponseEvent@@3PAXA 10025e84     swiusb.obj
 0003:00000e88       ?hSendDHCPDiscoveryEvent@@3PAXA 10025e88     swiusb.obj
 0003:00000e8c       ?hSendDHCPRequestEvent@@3PAXA 10025e8c     swiusb.obj
 0003:00000e90       ?g_IsRemoteWakeUpCallbackSupported@@3HA 10025e90     swiusb.obj
 0003:00000e94       ?ghModemPresent@@3PAXA     10025e94     swiusb.obj
 0003:00000e98       ?ghModemAbsent@@3PAXA      10025e98     swiusb.obj
 0003:00000e9c       ?gQmiCtlMsg@@3U_QMICTL_MSG@@A 10025e9c     swiusb.obj
 0003:00000eb0       ?gModem@@3U_SW_MODEM@@A    10025eb0     swiusb.obj
 0003:000019e8       __onexitend                100269e8     <common>
 0003:000019ec       __onexitbegin              100269ec     <common>
 0003:000019f0       _exitflag                  100269f0     <common>
 0003:000019f4       _pRawDllMain               100269f4     <common>

 entry point at        0001:00014448

 Static symbols

 0001:000017d8       __unwind$38487             100027d8 f   commdevice.obj
 0001:000017f0       __unwind$38488             100027f0 f   commdevice.obj
 0001:0000241c       __unwind$27643             1000341c f   commentry.obj
 0001:00004ce8       ?EventIOControl@@YAHPAUQMI_OPEN_INFO@@KPAEK1KPAK@Z 10005ce8 f   qmicom.obj
 0001:00004e8c       ?MdmIOControl@@YAHPAUQMI_OPEN_INFO@@KPAEK1KPAK@Z 10005e8c f   qmicom.obj
 0001:00005f30       __unwind$37988             10006f30 f   swdcom.obj
 0001:00005f40       __unwind$37989             10006f40 f   swdcom.obj
 0001:00007560       ?ProcessExiting@@YAHPAUVSP_OPEN_INFO@@@Z 10008560 f   swicom.obj
 0001:000080f8       ?NopIOControl@@YAHPAUQMI_OPEN_INFO@@KPAEK1KPAK@Z 100090f8 f   swicom.obj
 0001:000080f8       ?NopIOControl@@YAHPAUVSP_OPEN_INFO@@KPAEK1KPAK@Z 100090f8 f   swicom.obj
 0001:00008320       ?EventIOControl@@YAHPAUVSP_OPEN_INFO@@KPAEK1KPAK@Z 10009320 f   swicom.obj
 0001:000084c4       ?MdmIOControl@@YAHPAUVSP_OPEN_INFO@@KPAEK1KPAK@Z 100094c4 f   swicom.obj
 0001:0000a848       __unwind$41298             1000b848 f   swiusb.obj
 0001:0000ad24       __unwind$41411             1000bd24 f   swiusb.obj
 0001:0000aec8       __unwind$41480             1000bec8 f   swiusb.obj
 0001:0000b1c8       ?TransmitBytes@@YAHPAUSW_CHANNEL@@PAEI@Z 1000c1c8 f   swiusb.obj
 0001:0000b37c       ?TransmitBytesDirectIp@@YAHPAUSWD_CHANNEL@@PAEI@Z 1000c37c f   swiusb.obj
 0001:0000b7ac       ?InterruptThread@@YAXPAPAX@Z 1000c7ac f   swiusb.obj
 0001:0000bd74       ?InterruptDirectIpThread@@YAXPAPAX@Z 1000cd74 f   swiusb.obj
 0001:0000ce90       ?ParseTlpTransfer@@YAXPAEIPAXP6AX0I1@Z@Z 1000de90 f   swiusb.obj
 0001:0000d018       ?EthernetFrameHandlerMiniport@@YAXPAEIPAX@Z 1000e018 f   swiusb.obj
 0001:0000d02c       ?EthernetFrameHandlerRil@@YAXPAEIPAX@Z 1000e02c f   swiusb.obj
 0001:0000d1bc       ?EthernetFrameHandlerRilPacket@@YAXPAUSWD_CHANNEL@@PAPAUrilndispacket_tag@@@Z 1000e1bc f   swiusb.obj
 0001:0000d4a0       ?BulkInDirectIpNoTlpThread@@YAXPAPAX@Z 1000e4a0 f   swiusb.obj
 0001:0000db40       ?TransmitChannelBytesDirectIp@@YAHPAUSWD_CHANNEL@@PAEI@Z 1000eb40 f   swiusb.obj
 0001:0000dbb8       ?BulkOutThread@@YAXPAPAX@Z 1000ebb8 f   swiusb.obj
 0001:0000dd88       ?BulkOutDirectIpThread@@YAXPAPAX@Z 1000ed88 f   swiusb.obj
 0001:0000e038       ?ParseAndAddToReadQueue@@YAXPAEIPAUSW_CHANNEL@@@Z 1000f038 f   swiusb.obj
 0001:0000e0b4       ?BulkInThread@@YAXPAPAX@Z  1000f0b4 f   swiusb.obj
 0001:0000e708       ?BulkInDirectIpThread@@YAXPAPAX@Z 1000f708 f   swiusb.obj
 0001:0000ed9c       ?BulkOutMiniportThread@@YAXPAPAX@Z 1000fd9c f   swiusb.obj
 0001:00011750       ?ReadConfigurationInfo@@YAHPAUsAdapterConfig@@PAX1PAE@Z 10012750 f   wrp.obj
 0001:00012d84       ?OidFillOidList@@YAHPAEKPAK1@Z 10013d84 f   wrpoid.obj
 0001:0001459c       doexit                     1001559c f   corelibc:crt0dat.obj
 0001:00014924       ?CanThisExceptionObjectBeDestructed@@YAEPAUEHExceptionRecord@@E@Z 10015924 f   LIBCMT:frame_ce.obj
 0001:00014c70       ?CallCatchBlock@@YAPAXPAUEHExceptionRecord@@PAKPAU_CONTEXT@@PBU_s_FuncInfo@@PAXHK@Z 10015c70 f   LIBCMT:frame_ce.obj
 0001:00015008       ?BuildCatchObject@@YAXPAUEHExceptionRecord@@PAKPBU_s_HandlerType@@PBU_s_CatchableType@@@Z 10016008 f   LIBCMT:frame_ce.obj
 0001:000151dc       ?FindHandler@@YAEPAUEHExceptionRecord@@PAKPAU_CONTEXT@@PAU_DISPATCHER_CONTEXT@@PBU_s_FuncInfo@@H@Z 100161dc f   LIBCMT:frame_ce.obj
 0001:00015b04       ??__EgModem@@YAXXZ         10016b04 f   swiusb.obj
 0001:00015b50       ??__FgModem@@YAXXZ         10016b50 f   swiusb.obj

 Exports

  ordinal    name

        1    ?DriverEntry@@YAJPAU_CEDRIVER_OBJECT@@PAU_UNICODE_STRING@@@Z (long __cdecl DriverEntry(struct _CEDRIVER_OBJECT *,struct _UNICODE_STRING *))
               exported name: DriverEntry
        2    ?QMI_Close@@YAHPAUQMI_OPEN_INFO@@@Z (int __cdecl QMI_Close(struct QMI_OPEN_INFO *))
               exported name: QMI_Close
        3    ?QMI_Deinit@@YAHPAUQMI_PORT_MDD@@@Z (int __cdecl QMI_Deinit(struct QMI_PORT_MDD *))
               exported name: QMI_Deinit
        4    ?QMI_IOControl@@YAHPAUQMI_OPEN_INFO@@KPAEK1KPAK@Z (int __cdecl QMI_IOControl(struct QMI_OPEN_INFO *,unsigned long,unsigned char *,unsigned long,unsigned char *,unsigned long,unsigned long *))
               exported name: QMI_IOControl
        5    ?QMI_Init@@YAPAXPB_WPBX@Z (void * __cdecl QMI_Init(wchar_t const *,void const *))
               exported name: QMI_Init
        6    ?QMI_Open@@YAPAXPAXKK@Z (void * __cdecl QMI_Open(void *,unsigned long,unsigned long))
               exported name: QMI_Open
        7    ?QMI_Read@@YAKPAXPAEK@Z (unsigned long __cdecl QMI_Read(void *,unsigned char *,unsigned long))
               exported name: QMI_Read
        8    ?QMI_Seek@@YAKPAXJK@Z (unsigned long __cdecl QMI_Seek(void *,long,unsigned long))
               exported name: QMI_Seek
        9    ?QMI_Write@@YAKPAXPAEK@Z (unsigned long __cdecl QMI_Write(void *,unsigned char *,unsigned long))
               exported name: QMI_Write
       10    ?SWD_Close@@YAHPAUSWD_OPEN_INFO@@@Z (int __cdecl SWD_Close(struct SWD_OPEN_INFO *))
               exported name: SWD_Close
       11    ?SWD_Deinit@@YAHPAUSWD_MDD@@@Z (int __cdecl SWD_Deinit(struct SWD_MDD *))
               exported name: SWD_Deinit
       12    ?SWD_IOControl@@YAHPAUSWD_OPEN_INFO@@KPAEK1KPAK@Z (int __cdecl SWD_IOControl(struct SWD_OPEN_INFO *,unsigned long,unsigned char *,unsigned long,unsigned char *,unsigned long,unsigned long *))
               exported name: SWD_IOControl
       13    ?SWD_Init@@YAPAXPB_WPBX@Z (void * __cdecl SWD_Init(wchar_t const *,void const *))
               exported name: SWD_Init
       14    ?SWD_Open@@YAPAXPAXKK@Z (void * __cdecl SWD_Open(void *,unsigned long,unsigned long))
               exported name: SWD_Open
       15    ?SWD_Read@@YAKPAXPAEK@Z (unsigned long __cdecl SWD_Read(void *,unsigned char *,unsigned long))
               exported name: SWD_Read
       16    ?SWD_Seek@@YAKPAXJK@Z (unsigned long __cdecl SWD_Seek(void *,long,unsigned long))
               exported name: SWD_Seek
       17    ?SWD_Write@@YAKPAXPAEK@Z (unsigned long __cdecl SWD_Write(void *,unsigned char *,unsigned long))
               exported name: SWD_Write
       18    ?SWI_Close@@YAHPAUVSP_OPEN_INFO@@@Z (int __cdecl SWI_Close(struct VSP_OPEN_INFO *))
               exported name: SWI_Close
       19    ?SWI_Deinit@@YAHPAUVSP_PORT_MDD@@@Z (int __cdecl SWI_Deinit(struct VSP_PORT_MDD *))
               exported name: SWI_Deinit
       20    ?SWI_IOControl@@YAHPAUVSP_OPEN_INFO@@KPAEK1KPAK@Z (int __cdecl SWI_IOControl(struct VSP_OPEN_INFO *,unsigned long,unsigned char *,unsigned long,unsigned char *,unsigned long,unsigned long *))
               exported name: SWI_IOControl
       21    ?SWI_Init@@YAPAXPB_WPBX@Z (void * __cdecl SWI_Init(wchar_t const *,void const *))
               exported name: SWI_Init
       22    ?SWI_Open@@YAPAXPAXKK@Z (void * __cdecl SWI_Open(void *,unsigned long,unsigned long))
               exported name: SWI_Open
       23    ?SWI_PowerDown@@YAHPAX@Z (int __cdecl SWI_PowerDown(void *))
               exported name: SWI_PowerDown
       24    ?SWI_PowerUp@@YAHPAX@Z (int __cdecl SWI_PowerUp(void *))
               exported name: SWI_PowerUp
       25    ?SWI_Read@@YAKPAXPAEK@Z (unsigned long __cdecl SWI_Read(void *,unsigned char *,unsigned long))
               exported name: SWI_Read
       26    ?SWI_Seek@@YAKPAXJK@Z (unsigned long __cdecl SWI_Seek(void *,long,unsigned long))
               exported name: SWI_Seek
       27    ?SWI_Write@@YAKPAXPAEK@Z (unsigned long __cdecl SWI_Write(void *,unsigned char *,unsigned long))
               exported name: SWI_Write
       28    ?WMP_Close@@YAHK@Z (int __cdecl WMP_Close(unsigned long))
               exported name: WMP_Close
       29    ?WMP_Deinit@@YAHK@Z (int __cdecl WMP_Deinit(unsigned long))
               exported name: WMP_Deinit
       30    ?WMP_IOControl@@YAHKKPAEK0KPAK@Z (int __cdecl WMP_IOControl(unsigned long,unsigned long,unsigned char *,unsigned long,unsigned char *,unsigned long,unsigned long *))
               exported name: WMP_IOControl
       31    ?WMP_Init@@YAKPB_WPBX@Z (unsigned long __cdecl WMP_Init(wchar_t const *,void const *))
               exported name: WMP_Init
       32    ?WMP_Open@@YAKKKK@Z (unsigned long __cdecl WMP_Open(unsigned long,unsigned long,unsigned long))
               exported name: WMP_Open
       33    ?WMP_PowerDown@@YAXK@Z (void __cdecl WMP_PowerDown(unsigned long))
               exported name: WMP_PowerDown
       34    ?WMP_PowerUp@@YAXK@Z (void __cdecl WMP_PowerUp(unsigned long))
               exported name: WMP_PowerUp
       35    ?WMP_Read@@YAKKPAXK@Z (unsigned long __cdecl WMP_Read(unsigned long,void *,unsigned long))
               exported name: WMP_Read
       36    ?WMP_Seek@@YAKKJG@Z (unsigned long __cdecl WMP_Seek(unsigned long,long,unsigned short))
               exported name: WMP_Seek
       37    ?WMP_Write@@YAKKPBXK@Z (unsigned long __cdecl WMP_Write(unsigned long,void const *,unsigned long))
               exported name: WMP_Write
       38    USBDeviceAttach
       39    USBInstallDriver
